:100000000C94F8230C9429240C9429240C9429246E
:100010000C9429240C9491560C9429240C94292492
:100020000C9429240C9429240C9429240C9429241C
:100030000C9429240D94C9AB0C9429240C942924E4
:100040000C9429240D94A5250C9429240C9429247E
:100050000C9429240C9429240D94DA3B0D94F8A3D4
:100060000C9429240C949C320C9429240C9429245B
:100070000C9429240C9429240C9429240C942924CC
:100080000C9429240C9429240C9429240C942924BC
:100090000C9429240C9429240C9429240C942924AC
:1000A0000C9429240C9429240C9429240C9429249C
:1000B0000C9429240C9429240C9429240C9429248C
:1000C0000C9429240C9429240C9429240C94E532B2
:1000D0000C9429240C9429240C9429240C9429246C
:1000E0000C942924B50163015901D5019501C3017F
:1000F000810155015D01D701870133013F0157019E
:1001000085019D01C101A90183019701B101AD01E3
:10011000BF017D014301E701A301E301D101910189
:1001200079019301DB013501BD01E9018D01E50193
:1001300091018F0145016D018901E101C701B30101
:1001400077019B017F016901D9014D014B015B01E1
:10015000CD01DF019B015F0153016501036EDB36B9
:100160003D9A9999993DABAAAA2A3E000000803F8A
:10017000084AD73B3BCE016E84BCBFFDC12F3D6C0E
:1001800074319ABD56833DDA3D00C77F11BED9E474
:10019000BB4C3E916BAAAABE000000803F072C7AA0
:1001A000A5BA6CC590DA3B9365FC8BBC53F810FD87
:1001B0003C5692834DBD879D3AB63DCBC9BF5BBED1
:1001C00073DA0FC93F05A84CCDB2D44EB93836A961
:1001D000020C50B9918688083CA6AAAA2ABE000043
:1001E00000803F07634236B79BD8A71A3968561874
:1001F000AEBAAB558C1D3CB7CC5763BD6DEDFD75EC
:100200003EF6177231BF000000803F08000000BEBC
:10021000922449123EABAAAA2ABECDCCCC4C3E00B9
:10022000000080BEABAAAAAA3E00000000BF0000EA
:1002300000803F0000000000084178D3BB4387D115
:10024000133D190E3CC3BD4282AD2B3E68EC827655
:10025000BED98FE1A93E4C80EFFFBE01C4FF7F3FB6
:100260000000000000000D94F33C0D947BA50D945C
:10027000D14B0D94C3A60D944F690D94A24E0D94CD
:100280000D3D0D94A7620D9439A50D94BCA50D9458
:10029000BB6A0D9431790D940BA60D9407A60D94AD
:1002A000DF990D940E7D0D9423A60D94DD3C0D94E5
:1002B0001B3D0D94893C0D9411A60D94DF3C0D94CB
:1002C0001FA60D94C46A0D946D3C0D9427A60D9441
:1002D000CD6A0D94FDA50D9407030D94C6A50D944C
:1002E000A8590D94314D0D945A4C0D9406710D94EE
:1002F000EEA50D9461A50D9420930D94A46E0D941C
:10030000F9A50D94D93C0D94556E0D943B3D0D947B
:10031000E53C0D94F2A50D946B640D949EA50D948F
:10032000B2A50D94D0A50D9469A50D94B13C0D9482
:100330007A6E0D94A28A0D942CA60D941D6E0D94C8
:10034000194A0D94D66A0D9443A50D94B06D0D9481
:10035000AE5F0D94406E0D9476280D94846E0D94CE
:100360006F4C0D947F6E0D94E8A50D945F3C0D9439
:10037000FB840D94AC6C0D94C4480D9485A50D942C
:10038000946E0D942D6E0D94BF3C0D94806B0D9466
:10039000E4A50D94E9730D94694C0D9415A60D9484
:1003A000C55C0D9457A50D94A57B0D94973C0D94B9
:1003B000E33C0D9403A60D9471A50D94AF510D94DB
:1003C00019A60D94F5A50D944DA50D94A8A50D9411
:1003D0003EA50D948FA548617264636F64656420C7
:1003E00044656661756C742053657474696E6773D7
:1003F000204C6F616465640053746F726564207390
:10040000657474696E677320726574726965766568
:100410006400202020452F44203D20002020204D36
:10042000393030204B004C696E6561722061647612
:10043000616E63652073657474696E67733A004614
:10044000696C616D656E742073657474696E677331
:100450003A2044697361626C6564002020204D324B
:10046000303020440046696C616D656E74207365A0
:100470007474696E67733A002020204D3230392041
:1004800053004175746F2D526574726163743A2024
:10049000533D3020746F2064697361626C652C2059
:1004A0003120746F20696E74657270726574206596
:1004B0007874727564652D6F6E6C79206D6F7665DA
:1004C00073206173207265747261637473206F723C
:1004D000207265636F76657269657300204600203F
:1004E00020204D3230382053005265636F7665729C
:1004F0003A20533D4578747261206C656E6774686C
:1005000020286D6D2920463A537065656420286D5A
:100510006D2F6D2900205A002046002020204D32EA
:100520003037205300526574726163743A20533D32
:100530004C656E67746820286D6D2920463A5370AB
:1005400065656420286D6D2F6D29205A3A205A4C1C
:1005500069667420286D6D29002044002049002020
:1005600020204D33303420500050494420686561CC
:10057000746265642073657474696E67733A0020F1
:1005800044002049002020204D33303120500050BD
:1005900049442073657474696E67733A00205A0089
:1005A00020590020204D323036205800486F6D65AC
:1005B000206F666673657420286D6D293A002045AA
:1005C00000205A00205900205800204200205400EA
:1005D00020204D323035205300416476616E6365D2
:1005E00064207661726961626C65733A20533D4D97
:1005F000696E20666565647261746520286D6D2F73
:1006000073292C20543D4D696E2074726176656C9F
:1006100020666565647261746520286D6D2F73298D
:100620002C20423D6D696E696D756D207365676D37
:10063000656E742074696D6520286D73292C2058AF
:100640003D6D6178696D756D205859206A65726BD2
:1006500020286D6D2F73292C20205A3D6D617869FB
:100660006D756D205A206A65726B20286D6D2F7331
:10067000292C2020453D6D6178696D756D204520E0
:100680006A65726B20286D6D2F732900205400203D
:10069000204D323034205300416363656C657261D4
:1006A00074696F6E3A20533D616363656C65726176
:1006B00074696F6E2C20543D72657472616374208E
:1006C000616363656C65726174696F6E00204500DB
:1006D000205A0020590020204D3230312058004D42
:1006E0006178696D756D20416363656C65726174D5
:1006F000696F6E20286D6D2F7332293A00204500F6
:10070000205A0020590020204D3230332058004D0F
:100710006178696D756D2066656564726174657375
:1007200020286D6D2F73293A00204500205A0020A3
:10073000590020204D3932205800537465707320C1
:1007400070657220756E69743A0053657474696ED1
:1007500067732053746F72656400454550524F4D66
:10076000204572726F72000020006D657368206210
:100770006564206C6576656C696E673A20002900B7
:100780002C20002C2000706879736963616C2063F1
:100790006F6F7264696E617465733A202800290076
:1007A0002C20002C2000776F726C6420636F6F72B6
:1007B00064696E617465733A202800204600204504
:1007C000004731205A004D3234004D323620532537
:1007D0006C75004D3130362053004731204625647A
:1007E0000047312045312046343830004731205A07
:1007F0000020463230303000205900473120580068
:100800004D383300506F736974696F6E2072656183
:10081000642066726F6D20656570726F6D3A004D71
:100820003233202573002E67636F0046656564725E
:100830006174653A007265636F7665725F6D6163BE
:1008400068696E655F73746174655F616674657213
:100850005F706F7765725F70616E69632C20696E7F
:10086000697469616C20007265636F7665725F6D93
:10087000616368696E655F73746174655F616674F6
:1008800065725F706F7765725F70616E69632C204F
:10089000696E697469616C20007265636F76657258
:1008A0005F6D616368696E655F73746174655F61D4
:1008B000667465725F706F7765725F70616E696391
:1008C0002C20696E697469616C20006375727265B1
:1008D0006E745F706F736974696F6E5B5A5F4158B5
:1008E00049535D3A0043757272656E7420706F7380
:1008F0006974696F6E20595F415849533A004375D6
:100900007272656E7420706F736974696F6E2058AF
:100910005F415849533A00416674657220776169B6
:1009200074696E6720666F722074656D703A004757
:100930003120452D312046343830004731204535AF
:100940002046313230004D3833004D31393020539C
:100950002564004D3130392053256400473238205A
:10096000582059004731205A32352046383030005F
:100970004D31343020532564004D3130342053251F
:100980006400494E54340055564C4F202D20656E5E
:100990006400737470730055564C4F0020423A0047
:1009A00020453A00543A005A206C6976652061640B
:1009B0006A757374206F7574206F662072616E673C
:1009C000652E2053657474696E6720746F20302E15
:1009D00020436C69636B20746F20636F6E74696E63
:1009E00075652E005A206C6976652061646A75739E
:1009F00074206F7574206F662072616E67652E209B
:100A000053657474696E6720746F20300020573A04
:100A10000020453A00543A004B494C4C3A200041E2
:100A200075746F0020452F443D00416476616E630C
:100A300065204B3D002228322900443130303100FE
:100A400044313030300047323820590047323820A6
:100A500058005400496E76616C6964205420636FBD
:100A600064652E00496E76616C6964204D20636F69
:100A700064652E004D3232302053256900203A2023
:100A800000004C414E472053454C20464F524345B1
:100A900044002228312900205A3A0020593A0020E7
:100AA000453A00205A3A0020593A00583A002000AE
:100AB0002E0020423A0020453A00543A0020413AA4
:100AC0000020503A002042403A0020403A00202FB7
:100AD000003A00205400202F0020423A00202F002E
:100AE0006F6B20543A002569206D696E2C202569B2
:100AF0002073656300496E76616C6964204D2063E4
:100B00006F6465004D65736820626564206C65766E
:100B1000656C696E67206E6F7420616374697665B9
:100B20002E000A002020000A4D656173757265640D
:100B300020706F696E74733A000A5A20736561728F
:100B40006368206865696768743A20002C004E75F8
:100B50006D20582C593A2000476F20686F6D652032
:100B600066696E6973686564004D657368206265C7
:100B700064206C6576656C696E6720616374697664
:100B80006174656400557073616D706C6520666991
:100B90006E697368656400426564206C6576656C97
:100BA000696E6720636F7272656374696F6E206629
:100BB000696E697368656400206D6963726F6E7336
:100BC0000045786365737369766520626564206C9F
:100BD0006576656C696E6720636F727265637469B0
:100BE0006F6E3A200042656420636F7272656374B1
:100BF000696F6E2064617461206E6F742076616C21
:100C000069640A0042656420636F72726563746987
:100C10006F6E20646174612076616C69640A0062A1
:100C200061627973746570206170706C69656400CD
:100C3000636C65616E2075702066696E69736865A6
:100C40006420004D4553485F484F4D455F5A5F5300
:100C500045415243483A20004D65736820626564FF
:100C6000206C6576656C696E67207768696C6520B5
:100C70006C6F6F702066696E69736865642E000022
:100C8000206F66667365743A20006D657368206234
:100C90006564206C6576656C696E673A20000A00B1
:100CA000593A200000583A20003A206E6F20787997
:100CB00020636C616D70696E670A003A2078792054
:100CC000636C616D7065642E0A00002C2063616C9A
:100CD0006962726174696F6E207A3A2000426564BD
:100CE000206C6576656C696E672C20706F696E7418
:100CF0003A2000005A206A69747465722064617435
:100D0000612066726F6D205A2063616C2E206E6FB9
:100D1000742076616C69642E0A005A206A697474C2
:100D2000657220646174612066726F6D205A206361
:100D3000616C2E2076616C69642E0A004E6F206310
:100D40006C616D70696E6720666F72206669727380
:100D5000742063616C6962726174696F6E20706F78
:100D6000696E742E0A0046697273742063616C693F
:100D700062726174696F6E20706F696E7420636C4B
:100D8000616D7065642E0A00473238205730003A92
:100D9000200054656D7065726174757265206361C1
:100DA0006C6962726174696F6E20646F6E652E206B
:100DB000436F6E74696E7565207769746820707210
:100DC000657373696E6720746865206B6E6F622E41
:100DD0000000205A20736869667420286D6D293AD6
:100DE0000050494E44412074656D706572617475A0
:100DF00072653A2000002F3600537465703A200067
:100E000000205A20736869667420286D6D293A00A5
:100E100050494E44412074656D70657261747572FD
:100E2000653A20002F362028736B6970706564293D
:100E300000537465703A2000005A45524F3A200022
:100E40000073746172742074656D7065726174757D
:100E500072653A200050494E44412070726F6265BD
:100E60002063616C6962726174696F6E2073746172
:100E7000727400473238205730000A00205A3A2056
:100E80000020593A200020583A20004732382C20C0
:100E900066696E616C20004732382C2066696E618D
:100EA0006C20004732382C2066696E616C20004748
:100EB00032382C20696E697469616C2000473238C1
:100EC0002C20696E697469616C20004439393900DD
:100ED0004D3239002055706C6F616420696E20704E
:100EE000726F677265737300696E697469616C20F3
:100EF0007A737465707320616674657220726573AD
:100F000065743A2000696E697469616C207A737443
:100F1000657073206F6E20706F7765722075703A00
:100F20002000466163746F72792052455345540026
:100F300020202020334420205072696E7465727323
:100F400020202020002020204F726967696E616C8C
:100F5000205072757361202020004F637420313758
:100F6000203230313700436F6D70696C65643A2010
:100F700000286E6F6E652C2064656661756C742048
:100F8000636F6E66696729004F63742031372032C2
:100F90003031372032303A34303A333900737461AB
:100FA00072740020202020334420205072696E7417
:100FB00065727320202020002020204F726967690D
:100FC0006E616C2050727573612020200025002016
:100FD00020202020200020202020202000455241D9
:100FE00053494E4720616C6C206461746100466116
:100FF00063746F7279205245534554004D3630303A
:1010000000FFFFFF0000A0400000A04000000040E3
:1010100000007F4300005E439AD951430000000066
:10102000000040C19A99193E00007F4300005243DE
:101030000000524300000000000040C19A99193E90
:101040006563686F3A004572726F723A0000002162
:1010500010422063308440A550C660E770088129A3
:10106000914AA16BB18CC1ADD1CEE1EFF13112103B
:101070000273325222B5529442F772D662399318F3
:10108000837BB35AA3BDD39CC3FFF3DEE362244347
:101090003420040114E664C774A44485546AA54B43
:1010A000B528850995EEE5CFF5ACC58DD5533672DB
:1010B0002611163006D776F6669556B4465BB77A93
:1010C000A719973887DFF7FEE79DD7BCC7C448E567
:1010D000588668A7784008611802282338CCC9EDE3
:1010E000D98EE9AFF9488969990AA92BB9F55AD47B
:1010F0004AB77A966A711A500A333A122AFDDBDC33
:10110000CBBFFB9EEB799B588B3BBB1AABA66C8786
:101110007CE44CC55C222C033C600C411CAEED8F82
:10112000FDECCDCDDD2AAD0BBD688D499D977EB61A
:101130006ED55EF44E133E322E511E700E9FFFBED2
:10114000EFDDDFFCCF1BBF3AAF599F788F8891A9A5
:1011500081CAB1EBA10CD12DC14EF16FE18010A17C
:1011600000C230E3200450254046706760B9839880
:1011700093FBA3DAB33DC31CD37FE35EF3B10290CC
:1011800012F322D2323542145277625672EAB5CB4C
:10119000A5A89589856EF54FE52CD50DC5E234C31C
:1011A00024A01481046674476424540544DBA7FA20
:1011B000B79987B8975FE77EF71DC73CD7D326F26C
:1011C000369106B01657667676154634564CD96D6C
:1011D000C90EF92FE9C899E9898AB9ABA9445865BC
:1011E0004806782768C018E1088238A3287DCB5CC0
:1011F000DB3FEB1EFBF98BD89BBBAB9ABB754A540C
:101200005A376A167AF10AD01AB32A923A2EFD0F8B
:10121000ED6CDD4DCDAABD8BADE89DC98D267C075B
:101220006C645C454CA23C832CE01CC10C1FEF3E5F
:10123000FF5DCF7CDF9BAFBABFD98FF89F176E36AB
:101240007E554E745E932EB23ED10EF01E7C3C3E17
:101250005E2B3D3F2F5B5D3B2C2A225C004D3834DA
:1012600020582059205A2045004D3234004D323349
:10127000202573006175746F25692E67000A002FA1
:10128000000A002E0044656C6574696F6E2066610B
:10129000696C65642C2046696C653A200046696C6F
:1012A000652064656C657465643A002E002E002E1E
:1012B000002E004E6F772066726573682066696C39
:1012C000653A20004E6F7720646F696E672066690B
:1012D0006C653A20002220706F73002220706172CA
:1012E000656E743A2200535542524F5554494E454B
:1012F0002043414C4C207461726765743A2200743B
:101300007279696E6720746F2063616C6C207375ED
:10131000622D67636F64652066696C657320776909
:10132000746820746F6F206D616E79206C657665CE
:101330006C732E204D4158206C6576656C20697366
:101340003A00256920686F757273202569206D69E0
:101350006E757465730054494D454F55543A004DB0
:101360003131300046756C6C2052582042756666EB
:1013700065720022206661696C65643A2042756678
:101380006665722066756C6C2100456E71756569C5
:101390006E6720746F207468652066726F6E743A91
:1013A0002022002200456E717565696E6720746F9A
:1013B000207468652066726F6E743A2022002220C5
:1013C0006661696C65643A2042756666657220667E
:1013D000756C6C2100220050727573612069332096
:1013E0004D4B332072656164792E007A5F6D696EB2
:1013F0003A20007A5F6D61783A20005A204F666685
:1014000073657400795F6D696E3A2000795F6D6174
:10141000783A200059657300785F6D696E3A200054
:10142000785F6D61783A2000205761746368646F5B
:101430006720526573657400496E666F207363722E
:1014400065656E0057616974696E6720666F72200A
:101450006E6F7A7A6C6520616E64206265642063C9
:101460006F6F6C696E67005761697420666F7220D8
:10147000757365722E2E2E00557365642064757227
:10148000696E67207072696E7400556E6C6F61646E
:101490002066696C616D656E7400556E6C6F616479
:1014A000696E672066696C616D656E7400556E6B60
:1014B0006E6F776E20636F6D6D616E643A202200EF
:1014C00054756E650053442063617264205B466C02
:1014D00073684169725D0053442063617264205BEC
:1014E0006E6F726D616C5D0054656D702E2063616E
:1014F0006C2E205B4F4E5D0054656D702E20636135
:101500006C2E205B4F46465D0054656D70657261C0
:10151000747572652063616C6962726174696F6E63
:101520002069732066696E69736865642E20436C58
:1015300069636B20746F20636F6E74696E75652EBE
:101540000054656D702E2063616C2E2020202020B9
:1015500020202020200054656D70657261747572C2
:101560006500537570706F72740053746F702070E3
:1015700072696E740053544F505045442E200053EE
:101580007465707261746520746F6F206869676834
:101590003A2000546F74616C207072696E7420740C
:1015A000696D65203A00546F74616C2066696C61E6
:1015B0006D656E74203A005072696E742074696DA6
:1015C000653A20200046696C616D656E7420757304
:1015D00065643A202000537461746973746963739D
:1015E0002020004572726F72202D2073746174691F
:1015F00063206D656D6F7279206861732062656527
:101600006E206F7665727772697474656E005370C0
:101610006565640020536F6674776172652052655A
:10162000736574004D6F646520202020205B736912
:101630006C656E745D004D6F6465205B68696768FA
:1016400020706F7765725D0053686F7720656E64F8
:101650002073746F7073005365742074656D7065CA
:101660007261747572653A0053657474696E67735C
:1016700000576972696E67206572726F72005365F8
:101680006C6620746573742073746172742020001A
:10169000506C6561736520636865636B203A005325
:1016A000656C662074657374204F4B004E6F742018
:1016B000636F6E6E6563746564004D6F746F720066
:1016C0004865617465722F546865726D6973746FD3
:1016D000720046616E20746573740053656C6674A5
:1016E000657374206661696C65642020004C6566D2
:1016F0007420686F74656E642066616E3F00536588
:101700006C6674657374206572726F722021004577
:101710006E6473746F70206E6F7420686974004516
:101720006E6473746F707300456E6473746F7000D1
:1017300046726F6E74207072696E742066616E3FBF
:1017400000436865636B696E67205A20617869732E
:10175000202000436865636B696E672059206178BB
:101760006973202000436865636B696E67205820A9
:1017700061786973202000436865636B696E672038
:10178000686F74656E64202000436865636B696EE2
:101790006720656E6473746F707300436865636B74
:1017A000696E6720626564202020202000416C6CF7
:1017B00020636F7272656374202020202020004215
:1017C0006564202F204865617465720041786973F3
:1017D000206C656E67746800417869730053656CAE
:1017E000667465737420202020202020202000575C
:1017F000726974696E6720746F2066696C653A203F
:1018000000766F6C756D652E696E6974206661690E
:101810006C6564002053697A653A20004361726404
:101820002072656D6F766564005344207072696E36
:1018300074696E67206279746520006F70656E2030
:101840006661696C65642C2046696C653A20006F9E
:1018500070656E526F6F74206661696C65640043D9
:1018600061726420696E736572746564005344200C
:10187000696E6974206661696C0046696C652073E5
:10188000656C65637465640046696C65206F70659E
:101890006E65643A20006572726F722077726974A7
:1018A000696E6720746F2066696C6500534420631D
:1018B000617264206F6B0043616E6E6F7420656EA1
:1018C000746572207375626469723A2000526573A0
:1018D000756D696E67207072696E740052657375FC
:1018E0006D696E67207072696E7400526573756DF4
:1018F00065207072696E7400526573656E643A207B
:101900000043726173682064657465637465642E56
:1019100020436F6E74696E7565207072696E7469AC
:101920006E673F00426C61636B6F7574206F636319
:1019300075727265642E205265636F7665722070D1
:1019400072696E743F005265636F766572696E6787
:10195000207072696E742020202000686F77746F89
:101960002E707275736133642E636F6D00666F72D3
:10197000756D2E707275736133642E636F6D0070B8
:101980007275736133642E636F6D005072696E748B
:1019900020706175736564005072696E74206162B5
:1019A0006F72746564005072696E74657220646948
:1019B00073636F6E6E656374656400616E6420703E
:1019C0007265737320746865206B6E6F620050726D
:1019D000656865617420746865206E6F7A7A6C65DD
:1019E00021005072656865617400506F77657255AB
:1019F0007000506C65617365207761697400202008
:101A0000506C616E6E65724275666665724279747D
:101A100065733A200050494E44412048656174691D
:101A20006E67005049442063616C2E2020202020E6
:101A3000202020202020005049442063616C2E206B
:101A400066696E6973686564005049442063616C1F
:101A50006962726174696F6E0050617573652070A0
:101A600072696E7400506C616365206120736865F3
:101A70006574206F6620706170657220756E646594
:101A80007220746865206E6F7A7A6C652064757256
:101A9000696E67207468652063616C696272617445
:101AA000696F6E206F6620666972737420342070CF
:101AB0006F696E74732E20496620746865206E6F9E
:101AC0007A7A6C65206361746368657320746865F5
:101AD0002070617065722C20706F776572206F6660
:101AE0006620746865207072696E74657220696D15
:101AF0006D6564696174656C792E006F6B004F666B
:101B000066004E6F206D6F76652E004E6F20534439
:101B10002063617264004E6F7A7A6C650046696C6E
:101B2000616D656E74206E6F74206C6F61646564A6
:101B300000436F6C6F72206E6F7420636C6561720E
:101B4000004E6F00506C656173652075706772613F
:101B500064652E004E6577206669726D77617265E7
:101B60002076657273696F6E20617661696C61625F
:101B70006C653A004D6F7665205A004D6F76652092
:101B800059004D6F7665205800457874727564650C
:101B900072004D6F76652061786973004D657368DA
:101BA00020426564204C6576656C696E6700436110
:101BB0006C6962726174696F6E00206F6620390013
:101BC0004D6561737572696E6720726566657265D1
:101BD0006E636520686569676874206F662063615D
:101BE0006C6962726174696F6E20706F696E7400E7
:101BF0004D61696E004D32323120496E76616C69FB
:101C00006420657874727564657220004D323138D5
:101C100020496E76616C69642065787472756465BC
:101C20007220004D32303020496E76616C6964203C
:101C3000657874727564657220005265706F727495
:101C4000696E6720656E6473746F7020737461745D
:101C50007573004649524D574152455F4E414D45BF
:101C60003A4D61726C696E2056312E302E323B2017
:101C7000537072696E7465722F6772626C206D6149
:101C80007368757020666F722067656E36204649EE
:101C9000524D574152455F55524C3A6874747073B7
:101CA0003A2F2F6769746875622E636F6D2F70729B
:101CB00075736133642F50727573612D69332D50C4
:101CC0006C75732F2050524F544F434F4C5F564505
:101CD0005253494F4E3A312E30204D414348494EE0
:101CE000455F545950453A507275736120693320ED
:101CF0004D4B332045585452554445525F434F5540
:101D00004E543A3120555549443A30303030303015
:101D100030302D303030302D303030302D303030CC
:101D2000302D3030303030303030303030300A000C
:101D30004D31303920496E76616C69642065787464
:101D4000727564657220004D31303520496E7661C0
:101D50006C696420657874727564657220004D3119
:101D6000303420496E76616C6964206578747275D0
:101D700064657220004C6F6F73652070756C6C65C4
:101D800079004C6F61642066696C616D656E7400EA
:101D90004C6F6164696E672066696C616D656E7415
:101DA000004C6F6164696E6720636F6C6F720053E3
:101DB000656C656374206C616E6775616765004B67
:101DC000494C4C45442E2000496E76616C69642074
:101DD000657874727564657200496E7365727420FB
:101DE00066696C616D656E74005072696E74204630
:101DF000414E3A20004E6F7A7A6C652046414E3A49
:101E000000457874727564657220696E666F002093
:101E10006F66203900496D70726F76696E67206257
:101E200065642063616C6962726174696F6E2070B1
:101E30006F696E740043616C6962726174696E6788
:101E4000205A0043616C6962726174696F6E20642C
:101E50006F6E650043616C696272617465205A003F
:101E600048656174696E6720646F6E652E00486511
:101E70006174696E670046696C2E2073656E736FBE
:101E80007220205B6F6E5D0046696C2E2073656E5C
:101E9000736F72205B6F66665D0020467265652019
:101EA0004D656D6F72793A2000466C6F7700466918
:101EB0006E697368696E67206D6F76656D656E74A7
:101EC0007300206F66203400536561726368696E29
:101ED00067206265642063616C6962726174696F16
:101EE0006E20706F696E7400497465726174696FF9
:101EF0006E2000446F6E6520736176696E672066A0
:101F0000696C652E00446F6E65207072696E74692D
:101F10006E672066696C6500497320636F6C6F7231
:101F200020636C6561723F004368616E676520667F
:101F3000696C616D656E740046616E2073706565D5
:101F40006400656E717565696E672022004578745E
:101F50007275646572002045787465726E616C20DC
:101F60005265736574005072696E74657220737483
:101F70006F707065642064756520746F206572727F
:101F80006F72732E204669782074686520657272BE
:101F90006F7220616E6420757365204D3939392068
:101FA000746F20726573746172742E202854656D8D
:101FB00070657261747572652069732072657365EE
:101FC000742E2053657420697420616674657220D4
:101FD00072657374617274696E6729004E6F204C6C
:101FE000696E65204E756D62657220776974682030
:101FF000636865636B73756D2C204C617374204C42
:10200000696E653A20004E6F20436865636B737597
:102010006D2077697468206C696E65206E756D62DD
:1020200065722C204C617374204C696E653A2000F7
:1020300020746F6F206C6F6E672065787472757393
:10204000696F6E2070726576656E746564004C69A8
:102050006E65204E756D626572206973206E6F74B7
:10206000204C617374204C696E65204E756D6265FD
:10207000722B312C204C617374204C696E653A20B0
:10208000005072696E7465722068616C7465642EAC
:10209000206B696C6C28292063616C6C656421007D
:1020A00020636F6C6420657874727573696F6E203D
:1020B00070726576656E74656400636865636B73E2
:1020C000756D206D69736D617463682C204C61734C
:1020D00074204C696E653A20004552524F523A00C6
:1020E000456E642066696C65206C697374006F705E
:1020F000656E0054524947474552454400656E6439
:1021000073746F7073206869743A2000536C65654E
:10211000702E2E2E0044697361626C6520737465A5
:1021200070706572730043757272656E74004372ED
:10213000617368206465742E2020205B6F6E5D00E3
:102140004372617368206465742E20205B6F66663D
:102150005D0020436F756E7420583A20004368611B
:102160006E67656420636F72726563746C793F009B
:10217000436F6F6C646F776E00204C6173742055F1
:102180007064617465643A200043686F6F73652002
:1021900065787472756465723A004368616E67654C
:1021A000207375636365737321005072696E7420C8
:1021B00066726F6D2053440054656D702E2063610C
:1021C0006C6962726174696F6E0043616C696272FE
:1021D0006174696E67205A2E2E2E0043616C69620D
:1021E000726174650052657365742058595A206392
:1021F000616C6962722E0043616C69627261746520
:102200002058595A002042726F776E206F757420E3
:10221000526573657400426567696E2066696C6516
:10222000206C6973740058595A2063616C6962723A
:102230006174696F6E20636F6D70726F6D69736525
:10224000642E204C6566742066726F6E7420636124
:102250006C6962726174696F6E20706F696E742050
:102260006E6F7420726561636861626C652E0058E0
:10227000595A2063616C6962726174696F6E206380
:102280006F6D70726F6D697365642E2046726F6E2C
:10229000742063616C6962726174696F6E20706F23
:1022A000696E7473206E6F74207265616368616219
:1022B0006C652E0058595A2063616C6962726174B2
:1022C000696F6E20616C6C2072696768742E20588B
:1022D0002F5920617865732061726520736C69677E
:1022E00068746C7920736B657765642E20476F6F17
:1022F00064206A6F62210058595A2063616C6962D8
:10230000726174696F6E20616C6C207269676874A9
:102310002E20536B65772077696C6C206265206393
:102320006F72726563746564206175746F6D61743A
:102330006963616C6C792E0058595A2063616C692D
:1023400062726174696F6E206661696C65642E20CB
:102350004265642063616C6962726174696F6E20AA
:10236000706F696E7420776173206E6F7420666F72
:10237000756E642E0058595A2063616C69627261EF
:1023800074696F6E206F6B2E20582F59206178650D
:1023900073206172652070657270656E6469637523
:1023A0006C61722E20436F6E67726174756C61741C
:1023B000696F6E73210058595A2063616C696272AB
:1023C0006174696F6E206661696C65642E20506C63
:1023D0006561736520636F6E73756C7420746865D6
:1023E000206D616E75616C2E0058595A2063616CC6
:1023F0006962726174696F6E206661696C65642ED2
:10240000204C6566742066726F6E742063616C691F
:1024100062726174696F6E20706F696E74206E6F86
:102420007420726561636861626C652E0058595A48
:102430002063616C6962726174696F6E20666169A4
:102440006C65642E2046726F6E742063616C6962E5
:10245000726174696F6E20706F696E7473206E6F35
:102460007420726561636861626C652E0042656408
:10247000206C6576656C696E67206661696C656461
:102480002E2053656E736F7220646973636F6E6E76
:102490006563746564206F72206361626C6520629D
:1024A000726F6B656E2E2057616974696E67206666
:1024B0006F722072657365742E00426564206C65CE
:1024C00076656C696E67206661696C65642E205361
:1024D000656E736F72206469646E742074726967CC
:1024E0006765722E20446562726973206F6E206E7C
:1024F0006F7A7A6C653F2057616974696E672066F0
:102500006F722072657365742E00426564206C657D
:1025100076656C696E67206661696C65642E205310
:10252000656E736F72207472696767657265642087
:10253000746F6F20686967682E2057616974696ECF
:102540006720666F722072657365742E0042656441
:102550002048656174696E670042656420646F6E2F
:102560006500526967687420736964655B756D5DA9
:102570000052657365740052656172207369646509
:10258000205B756D5D00426564206C6576656C202E
:10259000636F7272656374004C656674207369645E
:1025A00065205B756D5D0046726F6E7420736964A3
:1025B000655B756D5D004265640044697374616EAE
:1025C0006365206265747765656E20746970206F3D
:1025D0006620746865206E6F7A7A6C6520616E641F
:1025E0002074686520626564207375726661636536
:1025F00020686173206E6F74206265656E2073655C
:1026000074207965742E20506C6561736520666F47
:102610006C6C6F7720746865206D616E75616C2CD1
:1026200020636861707465722046697273742073E8
:10263000746570732C2073656374696F6E204669CE
:10264000727374206C617965722063616C69627267
:102650006174696F6E2E004C6976652061646A75DD
:102660007374205A0041646A757374696E67205AE6
:10267000004175746F20686F6D6500207C20417586
:1026800074686F723A2000416C6C00416374697623
:10269000652045787472756465723A2000D713EB33
:1026A00013F313FB1304140C14141418142014281B
:1026B0001438144414671478148A149A14AD14C08E
:1026C00014C514D714E814F81409154115561562E9
:1026D000156A1575157F159315A615B715C515D669
:1026E00015E3150E161416241636164816571668D6
:1026F0001671167E1690169F16AC16BA16C016D214
:1027000016DB16ED16FE160F171F17281730174188
:102710001753176517771789179B17AD17BF17CC76
:1027200017D817DD17EF17011814181C1829183BB4
:10273000184F185F186D187A1888189618AC18B7C3
:1027400018CD18DC18EB18F8180119241946195B74
:10275000196D197F198B199819A619BB19CE19E291
:1027600019EA19F219FE19151A231A371A491A59B2
:102770001A651AFB1AFE1A021B0B1B161B1D1B31B6
:102780001B411B441B541B741B7B1B821B891B920C
:102790001B9C1BAE1BBA1BC01BF01BF51B0C1C2388
:1027A0001C3A1C531C301D471D5E1D751D821D905B
:1027B0001DA11DAF1DBF1DC81DD91DE91DF51D01A2
:1027C0001E0F1E151E351E431E541E601E6E1E76E5
:1027D0001E881E9A1EA91EAE1EC21EC81EE81EF32B
:1027E0001E051F181F281F381F421F4D1F561F662A
:1027F0001FDC1F062030204E208120A020BA20D9C7
:1028000020E020EE20F320FD200C21152126212E92
:1028100021402152215D217021792189219A21AA0B
:1028200021B821CA21DB21E521F721052216222624
:10283000226F22B422F72238237523B623E9232DF1
:10284000246D24BA240A254D255925622571257742
:102850002586259825A725B625BA255726652671EC
:10286000267B2687268B26457872656D65207370DA
:10287000616E206F6620746865205A2076616C75E1
:1028800065732100626F74746F6D00746F70000067
:10289000506F696E742068656967687420746F6F23
:1028A00020736D616C6C3A20007269676874006C0B
:1028B0006566740000506F696E742077696474688F
:1028C00020746F6F20736D616C6C3A2000002C20B7
:1028D000003A200046696E616C2063616C63756C20
:1028E000617465642062656420706F696E74200095
:1028F00000793A000044697374616E636520667202
:102900006F6D206D696E3A000043616C63756C6198
:1029100074696F6E206F6620746865206D616368EE
:10292000696E6520736B657720616E64206F6666E3
:10293000736574206661696C65642E00002C20004C
:102940003A200046696E616C206D65617375726531
:10295000642062656420706F696E742000002066D8
:1029600061696C65642E204C6F776572696E6720B3
:102970007A20746F20002C20697465726174696F0D
:102980006E2000496D70726F76696E6720626564B3
:1029900020706F696E742000002C207A002C206952
:1029A0007465726174696F6E2000496D70726F7624
:1029B000696E672062656420706F696E7420000024
:1029C0006C6F776572207468616E20596D696E2E28
:1029D000205920636F6F7264696E61746520636C47
:1029E000616D70696E672077617320757365642E01
:1029F0000043616C6962726174696F6E20706F6907
:102A00006E742000417420595F4D494E5F504F5302
:102A100000417420593000496D70726F76696E679D
:102A200020626564206F666673657420616E642041
:102A3000736B657700002C20002C200020004D6572
:102A40006173757265642000002C200041646A7512
:102A50007374656420706F736974696F6E3A2000D7
:102A6000002C20683A002C20646D61783A00506197
:102A7000727469616C20706F696E7420657374691B
:102A80006D617465642072616469757320746F6F21
:102A900020736D616C6C3A20000050617274696142
:102AA0006C20706F696E74206469616D6574657205
:102AB00020746F6F20736D616C6C3A2000746F70BE
:102AC000007269676874006C656674007269676893
:102AD00074006C65667400746F70006661696C6583
:102AE00064202D206E6F7420666F756E640A00720C
:102AF00069676874006C65667400002C2000496E7C
:102B0000697469616C20706F736974696F6E3A20C3
:102B10000066696E642062656420696E6475637422
:102B2000696F6E2073656E736F7220706F696E745B
:102B3000207A005920736561726368696E6720723C
:102B4000616469757320686967686572207468617B
:102B50006E20585F4D41582E20436C616D70696E38
:102B6000672077617320646F6E652E00592073654E
:102B700061726368696E6720726164697573206C45
:102B80006F776572207468616E20595F4D494E2ED3
:102B900020436C616D70696E672077617320646F8C
:102BA0006E652E005820736561726368696E6720D8
:102BB00072616469757320686967686572207468FA
:102BC000616E20585F4D41582E20436C616D7069D5
:102BD0006E672077617320646F6E652E00582073D6
:102BE0006561726368696E672072616469757320DC
:102BF0006C6F776572207468616E20585F4D494E26
:102C00002E20436C616D70696E672077617320645C
:102C10006F6E652E00536176696E67206265642071
:102C200063616C6962726174696F6E20766563744A
:102C30006F727320746F20454550524F4D005065A0
:102C40007270656E646963756C6172697479005A3B
:102C500065726F20706F696E7420636F7272656346
:102C600074696F6E3A005920766563746F72206CD8
:102C7000656E6774683A005820766563746F7220D9
:102C80006C656E6774683A00203C20005741524ED4
:102C9000494E473A2046726F6E7420706F696E74A9
:102CA000206E6F7420726561636861626C652E20AE
:102CB0005920636F6F7264696E6174653A000070C9
:102CC000745B315D3A0070745B305D3A00004D65B5
:102CD0006173757265643A000063757272656E7433
:102CE0005F706F736974696F6E5B5A5F41584953C7
:102CF0005D3A000063757272656E745F706F736920
:102D000074696F6E5B595F415849535D3A000063C7
:102D1000757272656E745F706F736974696F6E5BE4
:102D2000585F415849535D3A00417420592D340091
:102D300041742059300000636E74725B315D3A005B
:102D400000636E74725B305D3A00007665635F7994
:102D50005B315D3A00007665635F795B305D3A0018
:102D6000007665635F785B315D3A00007665635F8E
:102D7000785B305D3A00566563746F72733A200079
:102D8000497465726174696F6E3A2000496E7661AC
:102D90006C69642062656420636F72726563746934
:102DA0006F6E206D61747269782E20526573657440
:102DB00074696E6720746F206964656E74697479D4
:102DC0002E00496E76616C69642062656420636FD1
:102DD0007272656374696F6E206D61747269782EAA
:102DE00020582F59206178657320617265206661D3
:102DF000722066726F6D206265696E672070657201
:102E000070656E646963756C61722E00496E7661DF
:102E10006C69642062656420636F727265637469B3
:102E20006F6E206D61747269782E205368696674C4
:102E3000206F7574206F662072616E67652E005A70
:102E400065726F20706F696E7420636F7272656354
:102E500074696F6E3A00496E76616C6964206265D0
:102E60006420636F7272656374696F6E206D617444
:102E70007269782E204C656E677468206F662074C6
:102E80006865205920766563746F72206F757420B1
:102E90006F662072616E67652E00592076656374D7
:102EA0006F72206C656E6774683A00496E76616C6B
:102EB00069642062656420636F7272656374696F10
:102EC0006E206D61747269782E204C656E6774682F
:102ED000206F6620746865205820766563746F7271
:102EE000206F7574206F662072616E67652E0058C2
:102EF00020766563746F72206C656E6774683A0043
:102F0000556E646566696E65642062656420636FF2
:102F10007272656374696F6E206D61747269782E68
:102F200000000043616C63756C617465206F6666B8
:102F300073657420616E6420736B657720726574AD
:102F400075726E696E6720726573756C743A0000F5
:102F500000292C206572726F723A20002C20002903
:102F60003B207461726765743A2028002C20002988
:102F70003B206D656173757265642D636F72726558
:102F8000637465643A2028002C20006D65617375B8
:102F90007265643A202800706F696E7420230044C3
:102FA0006966666572656E63652061667465722028
:102FB000636F7272656374696F6E3A2000002C2033
:102FC0000063656E7465722C2061646A7573746544
:102FD000643A2000002C20005920766563746F72DB
:102FE0002C2061646A75737465643A2000002C209B
:102FF000005820766563746F722C2061646A757363
:103000007465643A200000636E74725B315D3A004F
:1030100000636E74725B305D3A0046696E616C20CD
:10302000636E74722076616C7565733A00000000FF
:1030300077793A0000636E74725B315D3A00005735
:1030400065696768745F793A000077783A000063D1
:103050006E74725B305D3A00005765696768745F33
:10306000783A000056657279206C6974746C65203A
:10307000736B65772064657465637465642E204F97
:103080007274686F676F6E616C697A696E672074BD
:10309000686520617865732E00004D61782E20658B
:1030A00072726F72206575636C696469616E3A0053
:1030B0004D61782E206572726F7220593A004D6111
:1030C000782E206572726F7220583A004D61782E0A
:1030D000206572726F72733A0000002C2065727264
:1030E0006F7220593A20002C206572726F7220583E
:1030F0003A20006572726F723A200029002C20007D
:10310000293B207461726765743A2028002C2000E6
:10311000293B20636F727265637465643A202800EE
:103120002C20006D656173757265643A202800007B
:103130002C206572726F72203E206D61782E2065A2
:1031400072726F72206575636C696469616E00509C
:103150006F696E74206E6F74206F6E206669727373
:103160007420726F77002C206572726F7220592064
:103170003E206D61782E206572726F722059002C8E
:10318000206572726F722058203E206D61782E206B
:103190006572726F722058002C20776569677468B9
:1031A00020593A2000506F696E74206F6E20666956
:1031B00072737420726F77003A00706F696E7420BA
:1031C00023004572726F7220616674657220636FAE
:1031D0007272656374696F6E3A2000002C20006380
:1031E000656E746572206E65772C20696E766572E7
:1031F0007465643A2000002C2000592076656374C1
:103200006F72206E65772C20696E766572746564C6
:103210003A2000002C20005820766563746F7220DD
:103220006E65772C20696E7665727465643A20004D
:10323000002C2000636F7272656374696F6E206189
:103240006E676C65733A2000002C2000636F727209
:10325000656374656420616E676C65733A20000075
:103260002C2000636F7272656374656420782F7917
:103270003A2000002C20002C20002C20003B206352
:103280006F7272656374696F6E20766563746F72B6
:103290003A2000697465726174696F6E3A200000AB
:1032A000292C206572726F723A20002C2000293B75
:1032B000207461726765743A2028002C2000206D0C
:1032C000656173757265643A202800706F696E7469
:1032D000202300002C200063656E7465722C206929
:1032E0006E697469616C3A2000002C2000592076C8
:1032F0006563746F722C20696E697469616C3A2021
:1033000000002C20005820766563746F722C2069B1
:103310006E697469616C3A200063616C63756C61FD
:103320007465206D616368696E6520736B657720D5
:10333000616E64206F6666736574204C53000000F4
:10334000E44200000000000057430000C0420000BB
:10335000E44200004043000040410000C042000041
:103360004041000000000000E442000000000000B6
:10337000574300000000000057430000C042000017
:10338000E4420000C042000040410000C042000092
:103390004041000040430000E44200004043000080
:1033A0005743000040435A00205A3A005900205920
:1033B0003A00580020583A0024F4D43050C38E20EC
:1033C000C2A24017828B7011127A910D816CD90ABA
:1033D000A861E108C7586607615143061E4B5D05A9
:1033E000C145A7041A411104093D980371393103FD
:1033F0004036DB0265339102D4305402802E1D0228
:10340000632CEE01752AC501B028A00110278101A7
:103410008F2564012B244B01E0223401AC211F01D4
:103420008D200D01801FFC00841EED00971DDF0024
:10343000B81CD200E61BC600201BBC00641AB200F8
:10344000B219A8000A19A0006A189900D1179100B2
:1034500040178B00B516840031167E00B315790035
:103460003A157300C7146F0058146A00EE13660013
:103470008813630025135E00C7125B006C125700AF
:1034800015125400C111510070114F0021114B0051
:10349000D61049008D10470046104400021042002B
:1034A000C00F4000800F3E00420F3C00060F3B0063
:1034B000CB0E3800930E37005C0E3500270E34001B
:1034C000F30D3200C10D3100900D3000600D2E0063
:1034D000320D2D00050D2C00D90C2B00AE0C29004F
:1034E000850C29005C0C2700350C27000E0C2600EB
:1034F000E80B2400C40B2400A00B23007D0B230049
:103500005A0B2100390B2100180B2000F80A1F006C
:10351000D90A1E00BB0A1E009D0A1D00800A1D005C
:10352000630A1C00470A1B002C0A1B00110A1A0020
:10353000F7091A00DD091900C4091900AB091900BF
:10354000920917007B091800630917004C0916003F
:1035500036091600200916000A091500F50815009D
:10356000E0081400CC081400B8081400A4081400E3
:10357000900813007D0812006B0813005808120011
:103580004608120034081100230811001208110027
:1035900001081100F0071000E0071000D00710002C
:1035A000C0071000B0070F00A107100091070E0020
:1035B00083070F0074070F0065070E0057070E0002
:1035C00049070E003B070D002E070E0020070D00D7
:1035D00013070D0006070D00F9060C00ED060D009F
:1035E000E0060C00D4060C00C8060C00BC060C005B
:1035F000B0060C00A4060B0099060C008D060B000B
:1036000082060B0077060B006C060B0061060A00B1
:1036100057060B004C060A0042060A0038060A004C
:103620002E060A0024060A001A060A0010060900DF
:1036300007060A00FD050900F4050900EB0509006D
:10364000E2050900D9050900D0050900C7050900F0
:10365000BE050900B5050800AD050800A50509006F
:103660009C050800940508008C05080084050800E6
:103670007C050800740508006C0507006505080056
:103680005D050700560508004E05070047050700C1
:103690004005080038050700310507002A05070026
:1036A000230507001C050600160507000F05070087
:1036B0000805060002050700FB040600F5040700E4
:1036C000EE040600E8040600E2040700DB0406003E
:1036D000D5040600CF040600C9040600C304060092
:1036E000BD040600B7040600B1040500AC040600E2
:1036F000A6040600A00405009B040600950405002E
:10370000900406008A040500850405008004060074
:103710007A04050075040500700405006B040500BB
:1037200066040500610405005C04050057040500FB
:10373000520405004D04050048040500430405003B
:103740003E0404003A04050035040500300404007A
:103750002C04050027040400230405001E040400B3
:103760001A04040016040500110404000D040400EA
:10377000090405000404040000040400FC03040020
:10378000F8030400F4030400F0030400EC03040055
:10379000E8030400E4030400E0030400DC03040085
:1037A000D8030400D4030400D0030400CC030400B5
:1037B000C8030300C503030024F404D9201BC40C70
:1037C0005C0E9804C4095F0265077101F405F900F5
:1037D000FB04B30048048700C10369005803550087
:1037E00003034500BE023A008402310053022A005E
:1037F0002902250004022000E4011C00C801190070
:10380000AF0117009801140084011300710110002A
:103810006101100051010E0043010D0036010B0043
:103820002B010B0020010B00150109000C01090000
:1038300003010800FB000800F3000800EB0007008C
:10384000E4000600DE000600D8000600D2000600F4
:10385000CC000500C7000500C2000500BD00040043
:10386000B9000400B5000400B1000400AD0004007C
:10387000A9000400A5000300A20003009F000400AB
:103880009B000300980003009500020093000300D2
:10389000900003008D0002008B00030088000200EE
:1038A0008600020084000300810002007F00020005
:1038B0007D0002007B000200790002007700010019
:1038C0007600020074000200720001007100020024
:1038D0006F0002006D0001006C0002006A00010030
:1038E0006900020067000100660001006500010038
:1038F000640002006200010061000100600001003C
:103900005F0002005D0001005C0001005B0001003F
:103910005A00010059000100580001005700010041
:103920005600010055000100540001005300000042
:10393000530001005200010051000100500001003D
:103940004F0001004E0000004E0001004D0001003C
:103950004C0001004B0000004B0001004A00010038
:103960004900010048000000480001004700010034
:10397000460000004600010045000000450001002F
:103980004400010043000000430001004200000029
:103990004200010041000000410001004000010020
:1039A0003F0000003F0001003E0000003E0001001B
:1039B0003D0000003D0001003C0000003C00000014
:1039C0003C0001003B0000003B0001003A00000009
:1039D0003A00010039000000390001003800000001
:1039E00038000000380001003700000037000100F7
:1039F00036000000360000003600010035000000EF
:103A000035000000350001003400000034000000E3
:103A100034000100330000003300000033000100D7
:103A200032000000320000003200010031000000CE
:103A300031000000310001003000000030000000C3
:103A4000300001002F0000002F0000002F000000B8
:103A50002F0001002E0000002E0000002E000100AB
:103A60002D0000002D0000002D0000002D000100A1
:103A70002C0000002C0000002C0000002C00010095
:103A80002B0000002B0000002B0000002B00010089
:103A90002A0000002A0000002A0000002A0001007D
:103AA0002900000029000000290000002900000072
:103AB0002900010028000000280000002800000064
:103AC0002800000028000100270000002700000057
:103AD000270000002700000027000100260000004A
:103AE000260000002600000026000000260001003D
:103AF0002500000025000000250000002500000032
:103B00002500000025000100240000002400000022
:103B10002400000024000000240001002300000015
:103B20002300000023000000230000002300000009
:103B300023000000230001002200000022000000FA
:103B400022000000220000002200000022000100EC
:103B500021000000210000002100000021000000E1
:103B600021000000210000002100010020000000D1
:103B700020000000200000002000000020000000C5
:103B80002000000020000000200001001F000000B5
:103B90001F0000001F0000001F0000001F000000A9
:103BA0001F0000001F0001001E0000001E0000009A
:103BB0001E0000001E0000004572723A204D494E62
:103BC00054454D50204245440054656D7065726106
:103BD000747572652068656174656420626564202F
:103BE0007377697463686564206F66662E204D493B
:103BF0004E54454D50207472696767657265642044
:103C000021004572723A204D415854454D50204292
:103C100045440054656D7065726174757265206805
:103C20006561746564206265642073776974636894
:103C30006564206F66662E204D415854454D5020D6
:103C40007472696767657265642021004572723A13
:103C5000204D494E54454D50003A204578747275B8
:103C6000646572207377697463686564206F666643
:103C70002E204D494E54454D50207472696767653A
:103C80007265642021004572723A204D41585445B6
:103C90004D50003A204578747275646572207377D0
:103CA000697463686564206F66662E204D415854C0
:103CB000454D502074726967676572656420210004
:103CC00020484F54454E4420544845524D414C20C5
:103CD00052554E41574159002048454154424544B0
:103CE00020544845524D414C2052554E4157415960
:103CF00000544845524D414C2052554E4157415970
:103D00000042454420544845524D414C2052554EA6
:103D1000415741590020544845524D414C2052557D
:103D20004E41574159202820505245484541542082
:103D3000484F54454E44290020544845524D414C6B
:103D40002052554E41574159202820505245484550
:103D50004154204845415442454429005052454869
:103D6000454154204552524F520042454420505242
:103D70004548454154204552524F52004572723ACF
:103D8000205052494E542046414E204552524F52E7
:103D9000004552524F523A205072696E742066614B
:103DA0006E207370656564206973206C6F7765722F
:103DB000207468656E20657870656374656400457D
:103DC00072723A20455854522E2046414E20455298
:103DD000524F52004552524F523A204578747275F4
:103DE0006465722066616E20737065656420697316
:103DF000206C6F776572207468656E2065787065D9
:103E00006374656400202D20496E76616C696420BE
:103E10006578747275646572206E756D6265722066
:103E20002100504944204175746F74756E65206699
:103E3000696E6973686564212050757420746865C3
:103E4000206C617374204B702C204B6920616E6470
:103E5000204B6420636F6E7374616E74732066729E
:103E60006F6D2061626F766520696E746F20436F9D
:103E70006E66696775726174696F6E2E680050496D
:103E800044204175746F74756E65206661696C6558
:103E900064212074696D656F75740020403A006F6D
:103EA0006B20543A006F6B20423A00504944204145
:103EB00075746F74756E65206661696C6564212028
:103EC00054656D706572617475726520746F6F20D2
:103ED0006869676800204B643A2000204B693A20EB
:103EE00000204B703A200020436C6173736963209B
:103EF00050494420002054753A2000204B753A2048
:103F000000206D61783A2000206D696E3A20002013
:103F1000643A200020626961733A200010137D002A
:103F20002015780060177300C0196E00401C6900EE
:103F3000E01E640080215F0040245A00F0265500F6
:103F400090295000202C4B00802E4600C0304100AC
:103F5000D0323C00B034370050363200C0372D002C
:103F600000392800103A2300F03A1E00B03B190037
:103F7000503C1400D03C0F00303D0A00803D05004D
:103F8000C03D0000F03DFBFF103EF6FF303EF1FF6C
:103F9000403EECFF503EE7FF603EE2FF703EDDFF3B
:103FA000703ED8FF1000C90210012C01400122010F
:103FB00070011801B0010E01F00104015002FA0075
:103FC000B002F0003003E600D003DC009004D20021
:103FD0007005C800A006BE000008B400B009AA0021
:103FE000D00BA000600E960060118C0000158200BE
:103FF00020197800C01D6E00A0226400B0275A006E
:10400000902C500000314600E0343C001038320063
:10401000903A2800603C1E00A03D1400803E0A003B
:10402000203F000070012C0190012701B001220106
:10403000C0011D01F00118011002130130020E0130
:104040006002090190020401C002FF000003FA00AF
:104050004003F5008003F000D003EB002004E600ED
:104060007004E100E004DC004005D700C005D20088
:104070004006CD00D006C8008007C3003008BE004F
:10408000F008B900C009B400B00AAF00B00BAA0034
:10409000D00CA500000EA000500F9B00C010960091
:1040A0005012910000148C00C0158700B0178200D8
:1040B000B0197D00D01B7800001E730040206E00F8
:1040C00090226900F024640040275F0090295A0084
:1040D000E02B5500102E500020304B0010324600CF
:1040E000E033410090353C00103737007038320023
:1040F000A0392D00B03A2800A03B2300603C1E00F0
:10410000103D1900903D1400103E0F00703E0A0053
:10411000C03E0500003F0000544D43204452495624
:104120004552204F56455254454D502000436F6E26
:1041300074696E7565207769746820616E6F746844
:10414000657220626F7764656E3F00473736004DB9
:104150003435205A004D3435004738300020003EB9
:10416000003E0020003E003E00005365766572650B
:1041700020736B65773A0000536C6967687420732D
:104180006B65773A002D2D2D2D2D2D2D2D2D2D2DBF
:104190002D2D2D2D2D2D2D2D2D004E2F41004D651A
:1041A00061737572656420736B65773A20004E2FDA
:1041B00041006D6D000052696768743A0043656E96
:1041C0007465723A004C6566743A005920646973EC
:1041D00074616E63652066726F6D206D696E3A0062
:1041E0004D373031004D373032004D3530300047DB
:1041F00031205A31352046313530300047393100D1
:10420000473120583530205931393020453020464B
:104210003730303000473930004D373032004D37BD
:1042200030322043004D3730322055004D37303288
:10423000004731205A31352046313530300047397A
:104240003100473120583530205931393020453040
:10425000204637303030004D383300473930004D7C
:104260003834004D31303420533000473930004766
:1042700031204531004D3832004D3833004D31305A
:104280003620532564004D32323020532564003AE5
:10429000200020202020202020202020202020203E
:1042A000202020202000203A200020202020202034
:1042B000202020202020202020202020202000201E
:1042C00020202020202020202020202000257300D6
:1042D0002020002D2D3A2D2D002000200020004C04
:1042E000002020002046002D2D2D003E5553420079
:1042F0005344002D2D0025202020202000202000C8
:104300002020000120002020202D2D2D2000202005
:104310005A002020000120004D36303000464C4528
:1043200058202D20203233302F353000505020209F
:10433000202D20203235342F313030004849505361
:10434000202D20203232302F313030005045542083
:10435000202D20203234302F393000504C41202085
:104360002D20203231352F35350041425320202D6C
:1043700020203235352F313030004D3234004D326F
:104380003320257300052E2E00580059005A004591
:1043900078747275646572004739390044697361D5
:1043A000626C65206661726D206D6F64653F0044CC
:1043B000697361626C65206661726D206D6F646502
:1043C000004661726D206E756D626572004D383405
:1043D000005072696E742066616E3A00457874729E
:1043E000756465722066616E3A0041786973206C6D
:1043F000656E67746820646966666572656E63657C
:104400003A004D6561737572656420617869732047
:104410006C656E6774683A004D3834004732382056
:1044200057005A30005A3100593000593100583085
:1044300000583100456E642073746F707320646996
:104440006167004D343400473238205700436865B7
:10445000636B2066616E73205B4449535D00436863
:1044600065636B2066616E73205B454E5D0054652D
:104470006D7065726174757265730058595A206366
:10448000616C2E2064657461696C73002D2D2D2D77
:104490002D2D2D2D2D2D2D2D00466C61736841691C
:1044A0007220495020416464723A002D2D2D2D2D2B
:1044B0002D2D2D2D2D2D2D004F63742031372032C1
:1044C00030313700446174653A20002D2D2D2D2D9B
:1044D0002D2D2D2D2D2D2D00453344763666756CF2
:1044E0006C0045494E595F30346100315F37356D9E
:1044F0006D5F4D4B33002D2D2D2D2D2D2D2D2D2D63
:104500002D2D0020332E302E31322D524332206299
:10451000313030004669726D776172653A0025640A
:104520002E25642E25642E2564004661726D206E52
:10453000756D62657200007263006265746100618E
:104540006C70686100646576005052555341334485
:10455000465700332E302E31322D524332000000A8
:104560000A0B02090C0D0E080703040100000000ED
:10457000000000000000000000000000000000003B
:1045800000000000000000000000121110000000F8
:10459000000000000000000000000000000000001B
:1045A000000000000000000000000000000000000B
:1045B00000000000010210202008081020401020F8
:1045C00040800201020108040201010204081020D7
:1045D00040808040201008040201800402018040D5
:1045E000201008040201080402010102040810203E
:1045F0004080010204081020408010080408801048
:104600002040044080102040048005050505070572
:1046100008080808020202020A0A0808040404043E
:10462000010101010101010103030303030303036A
:10463000040707070C0C0C0C0C0C0C0C02020202F9
:1046400006060606060606060B0B0B0B0B0B0B0BE2
:1046500007070A0A0A0A0A0A0505050404040808E5
:10466000000020002300260029002C002F0032002B
:1046700000010000030106010901000022002500DD
:1046800028002B002E00310034000201000005013B
:1046900008010B0100002100240027002A002D0042
:1046A0003000330001010000040107010A01024E3D
:1046B000414E494E495459494E46CDCCCC3D0AD77E
:1046C000233C17B7D13877CC2B329595E6241FB110
:1046D0004F0A000020410000C84200401C4620BC98
:1046E000BE4CCA1B0E5AAEC59D7400407A10F35AD8
:1046F00000A0724E18090010A5D4E80000E8764822
:10470000170000E40B54020000CA9A3B000000E1CD
:10471000F505000080969800000040420F00000060
:10472000A08601000000102700000000E803000040
:1047300000006400000000000A000000000001000A
:10474000000000002C76D888DC674F0823DFC1DF2B
:10475000AE59E1B1B796E5E3E453C63AE65199762E
:1047600096E8E6C28426EB898C9B62ED407C6FFC68
:10477000EFBC9C9F40F2BAA56FA5F490055A2AF7AA
:104780005C936B6CF9676DC11BFCE0E40D47FEF5B3
:1047900020E6B500D0ED902E03009435770500801B
:1047A000841E080000204E0A000000C80C3333337A
:1047B000330F986E12831141EF8D2114893BE6551A
:1047C00016CFFEE6DB18D1844B381BF77C1D901DFD
:1047D000A4BBE424203284725E228100C9F124EC5F
:1047E000A1E53D27AF9438BB6B01AB013B01D694EB
:1047F00011241FBECFEFD1E2DEBFCDBF00E00CBF62
:1048000019E0A0E0B2E0E8E0F8E703E00BBF02C087
:1048100007900D92AA3AB107D9F72BE1AAEAB9E0BD
:1048200001C01D92A93EB207E1F717E4CEEED7E42E
:1048300000E006C022970109FE010BBF0F9474B27D
:10484000C43ED10780E00807A9F70F9429AC0D9466
:10485000F2BB0C940000CF92DF92EF92FF920F9385
:104860001F93CF93DF938C01D42EC62FD72FD60E54
:10487000DC1671F1F801E080F180C990C7010F9456
:10488000B6B8C816F1F06C2DC7010F94E6B8C70191
:104890000F94B6B88C15A9F0EAE5F7E08491882367
:1048A00041F09091C00095FFFCCF8093C6003196F7
:1048B000F5CF8091C00085FFFCCF8AE08093C600D1
:1048C00007C0F80180819181019691838083D0CFC8
:1048D000DF91CF911F910F91FF90EF90DF90CF90DC
:1048E0000895EF92FF920F931F93CF93DF931F9240
:1048F000CDB7DEB78C017B01460FF8018081918135
:1049000049830F94B6B8F70181937F01F801808144
:10491000918101969183808349814E11EECF0F9052
:10492000DF91CF911F910F91FF90EF900895FF922B
:104930000F931F93CF93DF93CDB7DEB72C970FB6AE
:10494000F894DEBF0FBECDBF8C01F62E80E390E35E
:10495000A0E3B0E08D839E83AF83B8871C870B876D
:1049600044E0BE016B5F7F4FCE010B9674DF40E1E8
:1049700065E479E1CE010B966EDF40E165E579E112
:10498000CE010B9668DF40E165E379E1CE010B963D
:1049900062DF44E06DE279E1CE010B965CDF44E03A
:1049A00069E279E1CE010B9656DF44E061E379E1FB
:1049B000CE010B9650DF44E065E179E1CE010B9624
:1049C0004ADF44E065E679E1CE010B9644DF44E03E
:1049D00069E179E1CE010B963EDF44E06DE179E1DA
:1049E000CE010B9638DF44E061E279E1CE010B960F
:1049F00032DF44E065E279E1CE010B962CDF4CE03A
:104A00006BEE7AE0CE010B9626DF44E064EE7AE0AE
:104A1000CE010B9620DF44E06CE972E0CE010B96EC
:104A20001ADF44E068E972E0CE010B9614DF44E03F
:104A300064E972E0CE010B960EDF44E06CE872E0B0
:104A4000CE010B9608DF44E068E872E0CE010B96D9
:104A500002DF44E064E872E0CE010B96FCDE80E207
:104A600090E09A87898742E0BE01675F7F4FCE0161
:104A70000B96F1DE41E060EE7AE0CE010B96EBDEC4
:104A800044E06FE172E0CE010B96E5DE44E067E1C1
:104A900072E0CE010B96DFDE44E06BED7AE0CE01F2
:104AA0000B96D9DE44E067ED7AE0CE010B96D3DEBB
:104AB00044E063E172E0CE010B96CDDE41E067E0B9
:104AC0007BE0CE010B96C7DE44E06FE372E0CE01DF
:104AD0000B96C1DE89E08F1560F444E064E673E173
:104AE000CE010B96B8DE44E060E673E1CE010B9692
:104AF000B2DE46E551E360E070E049835A836B83A0
:104B00007C831C870B8744E0BE016F5F7F4FCE0123
:104B10000B96A1DEE0E4F0E18491882341F09091CE
:104B2000C00095FFFCCF8093C6003196F5CFEAE434
:104B3000F7E08491882341F09091C00095FFFCCF6D
:104B40008093C6003196F5CF8091C00085FFFCCFE1
:104B50008AE08093C6002C960FB6F894DEBF0FBE95
:104B6000CDBFDF91CF911F910F91FF9008951F93BB
:104B7000CF93DF93182FC0E4D0E1FE018491882306
:104B800041F09091C00095FFFCCF8093C600319614
:104B9000F5CFEAE3F7E08491882341F09091C000DB
:104BA00095FFFCCF8093C6003196F5CF8091C00071
:104BB00085FFFCCF8AE08093C600FE018491E0E48B
:104BC000F0E1882349F09091C00095FFFCCF8093DD
:104BD000C60031968491F5CF409145195091461900
:104BE000609147197091481982E397E00E94923AC8
:104BF0004091491950914A1960914B1970914C1983
:104C00008FE297E00E94923A40914D1950914E19CF
:104C100060914F19709150198CE297E00E94923A7E
:104C20004091511950915219609153197091541932
:104C300089E297E00E94923A8091C00085FFFCCF04
:104C40008AE08093C600FE018491E0E4F0E18823CD
:104C500049F09091C00095FFFCCF8093C60031963B
:104C60008491F5CFEFE0F7E08491882341F09091B3
:104C7000C00095FFFCCF8093C6003196F5CF8091A0
:104C8000C00085FFFCCF8AE08093C600FE018491BE
:104C9000E0E4F0E1882349F09091C00095FFFCCF5B
:104CA0008093C60031968491F5CF4091551950916B
:104CB0005619609157197091581986E097E00E9433
:104CC000923A4091591950915A1960915B1970911B
:104CD0005C1983E097E00E94923A40915D195091EF
:104CE0005E1960915F197091601980E097E00E94F1
:104CF000923A4091611950916219609163197091D3
:104D000064198DEF96E00E94923A8091C00085FF71
:104D1000FCCF8AE08093C600FE018491E0E4F0E1DC
:104D2000882349F09091C00095FFFCCF8093C60086
:104D300031968491F5CFEFEDF6E08491882341F030
:104D40009091C00095FFFCCF8093C6003196F5CFBF
:104D50008091C00085FFFCCF8AE08093C600FE01F1
:104D60008491E0E4F0E1882349F09091C00095FF40
:104D7000FCCF8093C60031968491F5CF40913519D0
:104D800050913619609137197091381986ED96E077
:104D90000E94A33A4091391950913A1960913B19F8
:104DA00070913C1983ED96E00E94A33A40913D1921
:104DB00050913E1960913F197091401980ED96E035
:104DC0000E94A33A409141195091421960914319B0
:104DD000709144198DEC96E00E94A33A8091C00036
:104DE00085FFFCCF8AE08093C600FE018491E0E459
:104DF000F0E1882349F09091C00095FFFCCF8093AB
:104E0000C60031968491F5CFE8E9F6E084918823D5
:104E100041F09091C00095FFFCCF8093C600319681
:104E2000F5CF8091C00085FFFCCF8AE08093C6005B
:104E3000FE018491E0E4F0E1882349F09091C00004
:104E400095FFFCCF8093C60031968491F5CF4091B9
:104E50002D1950912E1960912F19709130198FE8EA
:104E600096E00E94923A4091291950912A19609136
:104E70002B1970912C198CE896E00E94923A80913F
:104E8000C00085FFFCCF8AE08093C600FE018491BC
:104E9000E0E4F0E1882349F09091C00095FFFCCF59
:104EA0008093C60031968491F5CFE9EDF5E08491C9
:104EB000882341F09091C00095FFFCCF8093C600FD
:104EC0003196F5CF8091C00085FFFCCF8AE08093BA
:104ED000C600FE018491E0E4F0E1882349F090915E
:104EE000C00095FFFCCF8093C60031968491F5CF2A
:104EF00040913119509132196091331970913419E0
:104F000080ED95E00E94923A409115195091161942
:104F100060911719709118198DEC95E00E94923AE2
:104F200040916519509166196091671970916819DF
:104F30008AEC95E00E94A33A4091191950911A19F0
:104F400060911B1970911C1987EC95E00E94923AB0
:104F500040911D1950911E1960911F1970912019CF
:104F600084EC95E00E94923A4091211950912219C7
:104F7000609123197091241981EC95E00E94923A76
:104F8000409125195091261960912719709128197F
:104F90008EEB95E00E94923A8091C00085FFFCCF95
:104FA0008AE08093C600FE018491E0E4F0E188236A
:104FB00049F09091C00095FFFCCF8093C6003196D8
:104FC0008491F5CFECEAF5E08491882341F090914B
:104FD000C00095FFFCCF8093C6003196F5CF80913D
:104FE000C00085FFFCCF8AE08093C600FE0184915B
:104FF000E0E4F0E1882349F09091C00095FFFCCFF8
:105000008093C60031968491F5CF4091EB0A509180
:10501000EC0A6091ED0A7091EE0A83EA95E00E9435
:10502000923A4091EF0A5091F00A6091F10A709122
:10503000F20A80EA95E00E94923A4091F30A509178
:10504000F40A6091F50A7091F60A8DE995E00E94E4
:10505000923A8091C00085FFFCCF8AE08093C60021
:10506000FE018491E0E4F0E1882349F09091C000D2
:1050700095FFFCCF8093C60031968491F5CFEFE881
:10508000F5E08491882341F09091C00095FFFCCF1A
:105090008093C6003196F5CF8091C00085FFFCCF8C
:1050A0008AE08093C600FE018491E0E4F0E1882369
:1050B00049F09091C00095FFFCCF8093C6003196D7
:1050C0008491F5CF40919C0250919D0260919E0287
:1050D00070919F0285E895E00E94923A6091980253
:1050E0007091990280919A0290919B020F94133EC5
:1050F000AB01BC0182E895E00E94923A6091940273
:105100007091950280919602909197020F941F3EA4
:10511000AB01BC018FE795E00E94923A8091C000FC
:1051200085FFFCCF8AE08093C600FE018491E0E415
:10513000F0E1882349F09091C00095FFFCCF809367
:10514000C60031968491F5CFE9E6F5E08491882395
:1051500041F09091C00095FFFCCF8093C60031963E
:10516000F5CF8091C00085FFFCCF8AE08093C60018
:10517000FE018491E0E4F0E1882349F09091C000C1
:1051800095FFFCCF8093C60031968491F5CF409176
:105190008C0250918D0260918E0270918F028FE58A
:1051A00095E00E94923A6091880270918902809104
:1051B0008A0290918B020F94133EAB01BC018CE5E7
:1051C00095E00E94923A60918402709185028091EC
:1051D0008602909187020F941F3EAB01BC0189E5C6
:1051E00095E00E94923A8091C00085FFFCCF8AE052
:1051F0008093C600FE018491E0E4F0E1882349F049
:105200009091C00095FFFCCF8093C60031968491A9
:10521000F5CFE5E2F5E08491882341F09091C0005C
:1052200095FFFCCF8093C6003196F5CF8091C000EA
:1052300085FFFCCF8AE08093C600FE018491E0E404
:10524000F0E1882349F09091C00095FFFCCF809356
:10525000C60031968491F5CF40911F0250912002F3
:1052600060912102709122028BE195E00E94923AB6
:1052700020E030E040E752E460911702709118029C
:105280008091190290911A020F9429B0AB01BC01D0
:1052900088E195E00E94923A4091DB0A5091DC0A45
:1052A0006091DD0A7091DE0A85E195E00E94923AF4
:1052B0008091C00085FFFCCF8AE08093C600FE018C
:1052C0008491E0E4F0E1882349F09091C00095FFDB
:1052D000FCCF8093C60031968491F5CFE9EEF4E0DF
:1052E0008491882341F09091C00095FFFCCF80937A
:1052F000C6003196F5CF8091C00085FFFCCF8AE0D3
:105300008093C600FE018491E0E4F0E1882349F037
:105310009091C00095FFFCCF8093C6003196849198
:10532000F5CF4091D70A5091D80A6091D90A70916F
:10533000DA0A8FED94E00E94923A20E030E040E7F4
:1053400052E46091130270911402809115029091C1
:1053500016020F9429B0AB01BC018CED94E00E94C1
:10536000923A8091C00085FFFCCF8AE08093C6000E
:10537000FE018491E0E4F0E1882349F09091C000BF
:1053800095FFFCCF8093C60031968491F5CFE2E87B
:10539000F4E08491882341F09091C00095FFFCCF08
:1053A0008093C6003196F5CF8091C00085FFFCCF79
:1053B0008AE08093C600FE018491E0E4F0E1882356
:1053C00049F09091C00095FFFCCF8093C6003196C4
:1053D0008491F5CF4091E00A50E060E070E088E70A
:1053E00094E00E94A33A8091C00085FFFCCF8AE040
:1053F0008093C600FE018491E0E4F0E1882349F047
:105400009091C00095FFFCCF8093C60031968491A7
:10541000F5CF8091070B8823A1F1E5E6F4E08491B4
:10542000882341F09091C00095FFFCCF8093C60087
:105430003196F5CF8091C00085FFFCCF8AE0809344
:10544000C600FE018491E0E4F0E1882349F09091E8
:10545000C00095FFFCCF8093C60031968491F5CFB4
:1054600040913F025091400260914102709142028E
:105470008BE594E00E94923A8091C00085FFFCCFBA
:1054800011C0EFE3F4E08491882341F09091C000D3
:1054900095FFFCCF8093C6003196F5CF8091C00078
:1054A00085FFFCCF8AE08093C6001A3008F43EC026
:1054B000FE01C491E0E4F0E1CC2349F08091C0000A
:1054C00085FFFCCFC093C6003196C491F5CFE6E2CC
:1054D000F4E08491882341F09091C00095FFFCCFC7
:1054E0008093C6003196F5CF8091C00085FFFCCF38
:1054F0008AE08093C60040916413509165136091D7
:105500006613709167138CE194E00E94923A409187
:10551000601350916113609162137091631382E183
:1055200094E0DF91CF911F910C94923ADF91CF914B
:105530001F910895AF92BF92CF92DF92EF92FF92A8
:105540000F931F93CF93DF93CDB7DEB7E0970FB6DE
:10555000F894DEBF0FBECDBF80E1E1EDF2E0DE01E9
:10556000919601900D928A95E1F780E1E1EEF2E0EB
:10557000DE01519601900D928A95E1F780E1E1EF0D
:10558000F2E0DE01119601900D928A95E1F76E012D
:1055900081E2C80ED11C85E4E82E89E1F82E8E0147
:1055A0000F5E1F4F65E579E1AE014F5F5F4F95E3F9
:1055B000A92E99E1B92E20E030E0F6018191919178
:1055C000A191B1916F01F70181939193A193B1934F
:1055D0007F01F80181919191A191B1918F01FB011E
:1055E00081939193A193B193BF01FA01819191911C
:1055F000A191B191AF01F50181939193A193B193E1
:105600005F012F5F3F4F24303105B9F60F94CB1A5D
:1056100080E090E4ACE9B4E480932D1990932E19C6
:10562000A0932F19B09330198093291990932A19B8
:10563000A0932B19B0932C19109231191092321992
:10564000109233191092341980E29EE4A0E0B0E089
:105650008093651990936619A0936719B0936819A0
:1056600010921519109216191092171910921819F4
:1056700080E090E0A0E7B1E48093191990931A19A3
:10568000A0931B19B0931C1980931D1990931E1998
:10569000A0931F19B09320198DEC9CECACECBEE3E9
:1056A0008093211990932219A0932319B093241960
:1056B00080E090E0A0E2B0E4809325199093261951
:1056C000A0932719B09328191092F30A1092F40AA4
:1056D0001092F50A1092F60A1092EF0A1092F00A50
:1056E0001092F10A1092F20A1092EB0A1092EC0A50
:1056F0001092ED0A1092EE0A8DE39AE0A1E8B1E46F
:1057000080939C0290939D02A0939E02B0939F026F
:105710006DEC7CEC84E99FE30F940D3E609398025E
:105720007093990280939A0290939B0265E87BEEB6
:1057300080E692E40F94193E609394027093950270
:1057400080939602909397020F943E2D80E090E014
:10575000A0E8BFE38093900290939102A0939202FD
:10576000B09393021092E00A80E090E0A0E4B0E4ED
:1057700080931F0290932002A0932102B0932202F3
:1057800040E050E064E372E4409317025093180243
:105790006093190270931A021092DB0A1092DC0ACD
:1057A0001092DD0A1092DE0A1092D70A1092D80ADF
:1057B0001092D90A1092DA0A40E050E060E071E4F9
:1057C00040931302509314026093150270931602D3
:1057D0001092070B80933F0290934002A0934102E6
:1057E000B09342020E94244DE0E4F0E184918823CA
:1057F00041F09091C00095FFFCCF8093C600319698
:10580000F5CFE6EDF3E08491882341F09091C0005C
:1058100095FFFCCF8093C6003196F5CF8091C000F4
:1058200085FFFCCF8AE08093C600E0960FB6F8941F
:10583000DEBF0FBECDBFDF91CF911F910F91FF90C3
:10584000EF90DF90CF90BF90AF9008951F93CF93CC
:10585000DF93CDB7DEB72C970FB6F894DEBF0FBE3F
:10586000CDBF162F9C878B8786E591E3A0E0B0E043
:1058700089839A83AB83BC8344E0BE016B5F7F4F17
:10588000CE010B962ED843E050E0BE016B5F7F4FF8
:10589000CE0101960F9425B6892B09F0FFC040E197
:1058A00065E479E1CE010B961CD840E165E579E12C
:1058B000CE010B9616D840E165E379E1CE010B9657
:1058C00010D80F94CB1A44E06DE279E1CE010B962B
:1058D00008D844E069E279E1CE010B9602D844E0B1
:1058E00061E379E1CE010B960E94712444E065E109
:1058F00079E1CE010B960E94712444E065E679E1DE
:10590000CE010B960E94712444E069E179E1CE0159
:105910000B960E94712444E06DE179E1CE010B9673
:105920000E94712444E061E279E1CE010B960E946D
:10593000712444E065E279E1CE010B960E94712466
:105940004CE06BEE7AE0CE010B960E94712444E0AD
:1059500064EE7AE0CE010B960E94712444E06CE97B
:1059600072E0CE010B960E94712444E068E972E077
:10597000CE010B960E94712444E064E972E0CE01EE
:105980000B960E94712444E06CE872E0CE010B9605
:105990000E94712444E068E872E0CE010B960E94F8
:1059A000712444E064E872E0CE010B960E947124F9
:1059B00042E0BE01675F7F4FCE010B960E947124CB
:1059C00041E060EE7AE0CE010B960E94712444E043
:1059D0006FE172E0CE010B960E94712444E067E112
:1059E00072E0CE010B960E94712444E06BED7AE0E8
:1059F000CE010B960E94712444E067ED7AE0CE015F
:105A00000B960E94712444E063E172E0CE010B9694
:105A10000E94712441E067E07BE0CE010B960E947A
:105A2000712444E06FE372E0CE010B960E94712472
:105A30001A3070F044E064E673E1CE010B960E94E8
:105A4000712444E060E673E1CE010B960E9471245C
:105A50000E94244D0F943E2DE0E4F0E184918823D0
:105A600041F09091C00095FFFCCF8093C600319625
:105A7000F5CFE8EFF3E08491882341F09091C000E6
:105A800095FFFCCF8093C6003196F5CF8091C00082
:105A900085FFFCCF8AE08093C60001C04BDD2C96C9
:105AA0000FB6F894DEBF0FBECDBFDF91CF911F912F
:105AB0000895682F772767FD709580914F1090911A
:105AC00050108C5A9F4E0F940AB6909346108093B4
:105AD000451021E0892B09F420E0822F0895809160
:105AE00045109091461060E070E001960D94B3B2BD
:105AF0008A3010F0895A01C0805D9091C00095FFF6
:105B0000FCCF8093C6000895CF93C82F82958F70E5
:105B1000EFDF8C2F8F70CF91EBCFCF93C82F892FD2
:105B2000F3DF8C2FCF91F0CFCF93DF93FB0120E0F9
:105B300030E0DC01ED018D918823A1F14115510583
:105B400019F02417350774F58032A1F38A3051F12A
:105B500090ED980F9A3020F4682F6295607F08C00E
:105B60009FE9980F9630A8F4682F6295607F605780
:105B7000CE0102967981A0EDA70FAA3018F4762FF6
:105B80007A2B0CC0AFE9A70FA63018F47755762B07
:105B900005C088279927821B930B05C071932F5F3F
:105BA0003F4FC7CFC901DF91CF910895E0914510D4
:105BB000F09146108181882371F069E573E08AEAEB
:105BC00099E0AED682E475DF882319F00C9400F0DA
:105BD00008950C9400000895CF93DF9364E673E07A
:105BE0008AEA99E09DD6F894C0E0D0E060E0CE016A
:105BF0000F94E6B82196C11580E1D807B9F77894DB
:105C0000DF91CF910895AF92BF92CF92DF92EF9242
:105C1000FF920F931F93CF93DF93CDB7DEB76097BB
:105C20000FB6F894DEBF0FBECDBF66E773E08AEA19
:105C300099E076D681E43DDF8823A9F08091451074
:105C400090914610FC012181283741F440E150E059
:105C500060E070E002960F941BB403C040DF0F9425
:105C600097AD7B0102C0E12CF12C83E422DF882375
:105C700031F035DF0F9497AD262F872F02C020E03B
:105C800080E2FFE1FF22022F182F013020E21207ED
:105C900010F000E010E2C8018E0D9F1D813090428F
:105CA00020F000E010E20E191F0988E502DF8823CA
:105CB00071F1809145109091461040E150E0BE0195
:105CC0006F5F7F4F019630DF8C01009701F1FE017D
:105CD0003196CF01800F911FD701E817F90719F00E
:105CE00021912D93FACF4AE050E0B8018AEA99E079
:105CF00076D66AE873E08AEA99E012D6C7010DDF2A
:105D00008091C00085FFFCCF8AE08093C60080E2CE
:105D1000B82E9AE0A92E0115110529F1C701FDDE63
:105D20008091C00085FFFCCFB092C6006701F0E112
:105D3000CF0ED11CF7012FEFE21AF20A8081909169
:105D4000C00095FFFCCFB092C600DEDE0150110905
:105D500019F0EC14FD0471F78091C00085FFFCCFB1
:105D6000A092C600D8CF60960FB6F894DEBF0FBEE3
:105D7000CDBFDF91CF911F910F91FF90EF90DF90FA
:105D8000CF90BF90AF900895AF92BF92CF92DF9225
:105D9000EF92FF920F931F93CF93DF93CDB7DEB7B0
:105DA00060970FB6F894DEBF0FBECDBF6BEA73E00D
:105DB0008AEA99E0B5D581E47CDE8823A9F0809158
:105DC000451090914610FC012181283741F440E1B3
:105DD00050E060E070E002960F941BB403C07FDED9
:105DE0000F9497AD7B0102C0E12CF12C83E461DEBE
:105DF000882331F074DE0F9497AD262F872F02C0D1
:105E000020E080E2FFE1FF22022F182F013020E284
:105E1000120710F000E010E2C8018E0D9F1D8130C6
:105E2000904220F000E010E20E191F0988E541DEE3
:105E30008823B1F1809145109091461040E150E0E7
:105E4000BE016F5F7F4F01966FDE8C01009741F1BD
:105E5000CE0101965C01C12CD12CC016D10661F097
:105E6000F50161915F01C6018E0D9F1D0F94E6B88B
:105E7000FFEFCF1ADF0AF1CF4AE050E0B8018AEA1B
:105E800099E0ADD562EC73E08AEA99E049D5C701A3
:105E900044DE8091C00085FFFCCF8AE08093C6007D
:105EA00020E2B22E3AE0A32E0115110531F1C7010F
:105EB00034DE8091C00085FFFCCFB092C600670140
:105EC00020E1C20ED11CC701EFEFEE1AFE0A0F94BB
:105ED000B6B89091C00095FFFCCFB092C60014DE1A
:105EE0000150110919F0EC14FD0469F78091C0000C
:105EF00085FFFCCFA092C600D7CF60960FB6F8946E
:105F0000DEBF0FBECDBFDF91CF911F910F91FF90EC
:105F1000EF90DF90CF90BF90AF900895CF92DF9237
:105F2000EF92FF92CF93DF9366EE73E08AEA99E0F7
:105F3000F7D480E5BEDD882309F46BC0D0DD0F9473
:105F400097AD6B017C018FEFC816D10411F008F0FA
:105F500060C086E4AEDD882379F0C1DD0F9497AD93
:105F60006115710511F460E004C06130710521F420
:105F700061E08C2D0F942DA686E59BDD8823B1F082
:105F8000AEDD0F9497AD6115710511F460E005C0A9
:105F90006130710509F03DC061E08C2DDF91CF913A
:105FA000FF90EF90DF90CF900D9466A68C2D0F940C
:105FB0009BA6C1E0D0E0892B11F4C0E0D0E0E6EF71
:105FC000F3E08191882339F09091C00095FFFCCFD8
:105FD0008093C600F6CF4AE050E0B6018AEA99E025
:105FE000ACD4E4EDF5E08191882339F09091C000C4
:105FF00095FFFCCF8093C600F6CF4AE050E0BE018B
:106000008AEA99E0DF91CF91FF90EF90DF90CF90F7
:106010009BC4DF91CF91FF90EF90DF90CF900895D8
:10602000CF93DF93EC0160E08E810F9466A681E050
:1060300090E00F94A8A461E08E810F9466A681E0A1
:1060400090E00F94A8A460E08E810F9466A684E689
:1060500090E0DF91CF910D94A8A4CF92DF92EF92C0
:10606000FF920F931F93CF93DF937C01C0E0D0E0AA
:10607000C62ED12C87010C0F1D1F61E0F80187810E
:106080000F942DA6B6010C2E02C0759567950A9443
:10609000E2F76170F80187810F9466A62196C430FB
:1060A000D10541F7C701DF91CF911F910F91FF906B
:1060B000EF90DF90CF90B4CFCF92DF92EF92FF922C
:1060C0000F931F93CF93DF937C01C0E0D0E0C62EE7
:1060D000D12C87010C0F1D1F61E0F80187810F94FF
:1060E0002DA6B6010C2E02C0759567950A94E2F7AD
:1060F0006170F80187810F9466A62196C830D1059A
:1061000041F7C701DF91CF911F910F91FF90EF9061
:10611000DF90CF9085CF1F93CF93DF93EC01162FA5
:10612000642F8C810F9466A68D818F3F19F060E0FB
:106130000F9466A68F85612F84FF05C0CE01DF9185
:10614000CF911F91B9CF70E084E0759567958A95DE
:10615000E1F7CE0182DF612FCE01DF91CF911F9158
:106160007CCF40E0D8CF61E0FCDF80E496E00D9486
:10617000A8A462E0F6DF80E496E00D94A8A4CF9393
:10618000DF93CDB7DEB728970FB6F894DEBF0FBE0A
:10619000CDBF28E0E1E0F3E0DE01119601900D9221
:1061A0002A95E1F7FC012389421710F04FEF420FC7
:1061B000FE013196E40FF11DE40FF11D2081260F41
:1061C0002068622F28960FB6F894DEBF0FBECDBFB1
:1061D000DF91CF91C6CFFC016089262F2460208BF0
:1061E0006C60BFCFCF93DF93EC01423018F08F8506
:1061F00088608F874B8B1C8A222329F0413019F449
:106200008F8584608F8780E593EC0F94A8A460E06D
:106210008C810F9466A660E08E810F9466A68D81B6
:106220008F3F19F060E00F9466A66F8564FD19C07A
:1062300063E0CE0112DF84E991E10F94A8A463E04A
:10624000CE010BDF84E991E10F94A8A463E0CE01B5
:1062500004DF86E990E00F94A8A462E0CE01FDDEA1
:1062600013C06062CE017DDF84E991E10F94A8A4A0
:106270006F856062CE0175DF86E990E00F94A8A477
:106280006F856062CE016DDF6F856062CE0169DF70
:106290008CE390E00F94A8A484E0888BCE019BDF70
:1062A0008CE390E00F94A8A4CE015DDF88EB9BE027
:1062B0000F94A8A482E0898B66E0CE0152DF8CE3C4
:1062C00090E0DF91CF910D94A8A46F927F928F926E
:1062D000AF92CF92EF920F931F93CF93DF93CDB7EF
:1062E000DEB73C01162F842F5E854F85388999894A
:1062F000F301848325830683E782C086A186828694
:10630000538744873587968761E00F942DA6F30164
:1063100085818F3F19F061E00F942DA661E0F301B4
:1063200086810F942DA6112319F0F301178603C05F
:1063300080E1F301878720E041E060E1C301DF9164
:10634000CF911F910F91EF90CF90AF908F907F9052
:106350006F9048CF8F92AF92CF92EF920F93DC0164
:1063600013961C921E921297EEEFF3E0ED93FC93BE
:106370001F921F921F921F928C2CAE2CC02EE22EC9
:10638000042F2FEF462F61E0A0DF0F900F900F90AA
:106390000F900F91EF90CF90AF908F900895CF9383
:1063A000DF93EC01423018F08F8588608F874B8B2C
:1063B0001C8A222329F0413019F48F8584608F874D
:1063C00080E593EC0F94A8A460E08C810F9466A6FE
:1063D00060E08E810F9466A68D818F3F19F060E09A
:1063E0000F9466A66F8564FD19C063E0CE0135DEAB
:1063F00084E991E10F94A8A463E0CE012EDE84E944
:1064000091E10F94A8A463E0CE0127DE86E990E035
:106410000F94A8A462E0CE0120DE13C06062CE011A
:10642000A0DE84E991E10F94A8A46F856062CE019B
:1064300098DE86E990E00F94A8A46F856062CE0193
:1064400090DE6F856062CE018CDE8CE390E00F946D
:10645000A8A484E0888BCE01BEDE8CE390E00F948C
:10646000A8A4CE0186DE80E496E00F94A8A482E082
:10647000898B66E0CE0175DE8CE390E00F94A8A4D2
:1064800040E068E0CE017BDE62E279E0CE010F946D
:1064900001A741E068E0CE0172DE62E279E0CE0160
:1064A0000F9401A742E066E0CE0169DE60E279E088
:1064B000CE01DF91CF910D9401A7CF92DF92EF92A1
:1064C000FF920F931F93CF93DF931F921F92CDB72D
:1064D000DEB78C01677088E0689FB00111246064AA
:1064E000C80149835A833DDE4981C42E5A81D52E85
:1064F000E12CF12CD6016D916D01D801ED91FC914B
:106500000190F081E02DC8011995BFEFEB1AFB0A4D
:10651000E8E0EE16F10471F70F900F90DF91CF9144
:106520001F910F91FF90EF90DF90CF90089541E081
:10653000F2DD81E090E008951F920F920FB60F9266
:1065400011240BB60F922F933F934F935F936F934A
:106550008F939F93EF93FF93CF93DF931F92CDB7CA
:10656000DEB78091C00084FF04C08091C60089839B
:1065700019C06091C60020912B0A30912C0AC901E4
:1065800001968F77992740912D0A50912E0A8417F2
:10659000950741F0F901E555F64F608390932C0A79
:1065A00080932B0A0F90DF91CF91FF91EF919F91F4
:1065B0008F916F915F914F913F912F910F900BBEF3
:1065C0000F900FBE0F901F9018951F920F920FB64D
:1065D0000F9211240BB60F922F933F934F935F931B
:1065E0006F938F939F93EF93FF93CF93DF931F92BC
:1065F000CDB7DEB780912F0A9091300A019709F547
:106600008091D00084FF04C08091D600898319C096
:106610006091D60020912B0A30912C0AC901019675
:106620008F77992740912D0A50912E0A841795074C
:1066300041F0F901E555F64F608390932C0A809361
:106640002B0A0F90DF91CF91FF91EF919F918F9146
:106650006F915F914F913F912F910F900BBE0F90D3
:106660000FBE0F901F901895CF92DF92EF92FF927E
:106670006A017B01411581EE58076105710509F436
:1066800063C082E08093C00060E079E08DE390E039
:10669000A70196010F943CB22150310941095109DB
:1066A000CA01B90122E030E040E050E00F943CB272
:1066B00091E03093C5002093C4008091C1008061B7
:1066C0008093C1008091C10088608093C100809157
:1066D000C10080688093C100992341F082E08093DB
:1066E000D00060E079E08DE390E006C01092D00029
:1066F00060E874E88EE190E0A70196010F943CB247
:106700002150310941095109CA01B90122E030E0A3
:1067100040E050E00F943CB23093D5002093D40079
:106720008091D10080618093D1008091D1008860F8
:106730008093D1008091D10080688093D100FF9038
:10674000EF90DF90CF9008951092C00090E020E18C
:1067500030E0AFCF20912D0A30912E0A80912B0A84
:1067600090912C0A8217930771F0F901E555F64FC5
:1067700080812F5F3F4F2F77332730932E0A20934E
:106780002D0A90E008958FEF9FEF089580912D0AD4
:1067900090912E0A90932C0A80932B0A08954F9281
:1067A0005F926F927F928F929F92AF92BF92CF92A1
:1067B000DF92EF92FF920F931F93CF93DF93CDB7AA
:1067C000DEB7A0970FB6F894DEBF0FBECDBF5C0159
:1067D0004115510561057105E9F420E030E040E321
:1067E00050E060E070E0A0960FB6F894DEBF0FBEF8
:1067F000CDBFDF91CF911F910F91FF90EF90DF9070
:10680000CF90BF90AF909F908F907F906F905F9050
:106810004F905BC08E010F5F1F4FC12CD12C7601B2
:106820004801422E512C612C712C8FEFC81AD80AC6
:10683000E80AF80ACB01BA01A30192010F941AB237
:10684000CA01F80161938F01A901BC0141155105ED
:106850006105710551F7F1E0CF1AD108E108F1089F
:10686000F401EC0DFD1D80818A3010F440E301C07D
:1068700047E3480F552747FD5095652F752F20E0BA
:1068800030E0C50122D081E0C81AD108E108F10842
:10689000EFEFCE16DE06EE06FE0611F7A0960FB657
:1068A000F894DEBF0FBECDBFDF91CF911F910F9146
:1068B000FF90EF90DF90CF90BF90AF909F908F9020
:1068C0007F906F905F904F9008952115310539F4B6
:1068D0008091C00085FFFCCF4093C60008952A3008
:1068E000310509F43FC05BCF9A01462F552747FD7C
:1068F0005095652F752FE9CFCF93DF93EC0120E002
:1069000030E04DE050E060E070E0DFDF20E030E0BC
:106910004AE050E060E070E0CE01DF91CF91D5CF4A
:10692000FB012191BF01222339F03091C00035FFD6
:10693000FCCF2093C600F4CFDFCF9A01AB016627CE
:1069400057FD6095762FC1CFCF93DF93EC019A016D
:10695000AB01662757FD6095762FB7DFCE01DF913B
:10696000CF91CACFCF92DF92EF92FF92CF93DF9376
:10697000EC016A017B0177FF0FC020E030E04DE2BF
:1069800050E060E070E0A1DFF094E094D094C09417
:10699000C11CD11CE11CF11C2AE0B701A601CE01EB
:1069A000DF91CF91FF90EF90DF90CF90F8CE21153F
:1069B000310539F48091C00085FFFCCF4093C600BB
:1069C0000895EDCECF93DF93EC019A01462F50E06E
:1069D00060E070E0ECDFCE01DF91CF918DCF9A01C6
:1069E000AB0160E070E0E3CFCF93DF93EC019A015D
:1069F000AB0160E070E0DBDFCE01DF91CF917CCFB7
:106A0000CF93DF93EC01D3DFCE01DF91CF9174CF31
:106A10008F929F92AF92BF92CF92DF92EF92FF92AE
:106A20001F93CF93DF93EC016A017B01122F20E0CB
:106A300030E0A901C701B6010F9428AD87FF0CC053
:106A400020E030E04DE250E060E070E0CE013DDF5C
:106A5000F7FAF094F7F8F094B12C60E070E080E081
:106A60009FE3B11641F020E030E040E251E40F94A2
:106A70002FADB394F6CF9B01AC01C701B6010F94C3
:106A800038AC6B017C010F949CAD4B015C010F9401
:106A9000C8AD9B01AC01C701B6010F9437AC6B01C7
:106AA0007C012AE0B501A401CE0179DE112361F059
:106AB000E4E1F7E08191882339F09091C00095FFDF
:106AC000FCCF8093C600F6CF112319F120E030E00F
:106AD00040E251E4C701B6010F9429B06B017C017B
:106AE0000F9497AD4B01AA2497FCA094BA2CB50142
:106AF000A401CE0137DFC501B4010F94CAAD9B01DB
:106B0000AC01C701B6010F9437AC6B017C01115089
:106B1000DBCFDF91CF911F91FF90EF90DF90CF906F
:106B2000BF90AF909F908F90089572CFCF93DF93D7
:106B3000EC016EDFCE01DF91CF91DECEFC016591DD
:106B40007591859194910895EF92FF920F931F9301
:106B5000CF93DF93EC01CC0FDD1FCC0FDD1FCE01F7
:106B6000845E9F4EEBDF9E012950354F79018E01E7
:106B70000551154FF80120813181428153810F94D5
:106B800038ACF7016083718382839383CE018C5C80
:106B90009F4ED4DF9E01215D3D4F7901F801208198
:106BA0003181428153810F9438ACF7016083718346
:106BB00082839383CE01885D9F4EC0DFCD5DDD4F24
:106BC000F80120813181428153810F9438AC688370
:106BD00079838A839B83DF91CF911F910F91FF90DF
:106BE000EF900895CF93C82F40910E0250910F025D
:106BF00060911002709111024093AE0A5093AF0A57
:106C00006093B00A7093B10A2091490230914A0210
:106C100030936D0B20936C0B24E630E030934A02E6
:106C2000209349020F9442A46093A90A7093AA0A80
:106C30008093AB0A9093AC0A8C2FCF910D947B1C60
:106C400080E00F947B1C8091AE0A9091AF0AA091D6
:106C5000B00AB091B10A80930E0290930F02A093F4
:106C60001002B093110280916C0B90916D0B909378
:106C70004A02809349020F9442A46093A90A709338
:106C8000AA0A8093AB0A9093AC0A0895682F7727DD
:106C900067FD709580914F10909150108C5A9F4EC7
:106CA0000F940AB6909346108093451021E0892BEB
:106CB00009F420E0822F089520914F103091501058
:106CC000BC01C9018C5A9F4E0F9442B69093461056
:106CD0008093451021E0892B09F420E0822F08954C
:106CE00080914510909146104AE050E060E070E0DD
:106CF00001960D941BB40F931F93CF93DF930091D4
:106D000045101091461065E470E0C8010F940AB672
:106D1000EC01009751F460E070E0C8010196DF914A
:106D2000CF911F910F910D94B3B2188280914510AD
:106D30009091461060E070E001960F94B3B225E4A4
:106D40002883DF91CF911F910F9108958091451075
:106D50009091461060E070E001960D94B3B22F92CE
:106D60003F924F925F926F927F928F929F92AF92DB
:106D7000BF92CF92DF92EF92FF920F931F93CF9328
:106D8000DF93CDB7DEB760970FB6F894DEBF0FBEC6
:106D9000CDBF1C012A013B014801590120E030E030
:106DA0004CE052E4C301B2010F9437AC25E535E560
:106DB00047E052E40F942FAD6B017C010F9405AEB8
:106DC0000F9497AD8B0177FF12C020E030E040E8D0
:106DD0005FE3C701B6010F9457AF18160CF05DC002
:106DE000C12CD12CE0E8EE2EEFE3FE2E56C066302B
:106DF0007105DCF02AEA3AE24CE453E4C301B20143
:106E00000F9437AC25E535E547E052E40F942FADFC
:106E10006B017C0120E030E0A9010F9428AD87FFD1
:106E20003FC0C12CD12C76013BC0882777FD8095CF
:106E3000982F0F94CAAD25E535E547E052E40F944D
:106E400029B020E030E04CE052E40F9438AC9B01D4
:106E5000AC01C301B2010F9437AC25E535E547E03D
:106E600052E40F942FAD6B017C0120E030E0A901CA
:106E70000F9428AD87FD17C020E030E040E85FE3C5
:106E8000C701B6010F9457AF181684F4C12CD12C4A
:106E900070E8E72E7FE3F72E09C000E010E006C09F
:106EA00005E010E003C0C12CD12C760120E030E0D9
:106EB00040EC50E4C501B4010F9437AC2BEA3AEA38
:106EC00042E052E40F942FAD2B013C010F9405AE2C
:106ED0000F9497AD788B6F8777FF12C020E030E07A
:106EE00040E85FE3C301B2010F9457AF18160CF0EE
:106EF0005FC0412C512C60E8662E6FE3762E58C09F
:106F0000AF85B8891697E4F026E535E549E253E404
:106F1000C501B4010F9437AC2BEA3AEA42E052E4DF
:106F20000F942FAD2B013C0120E030E0A9010F941C
:106F300028AD87FD40C0E5E0F0E0F88BEF8746C064
:106F4000882777FD8095982F0F94CAAD2BEA3AEAEF
:106F500042E052E40F9429B020E030E040EC50E4ED
:106F60000F9438AC9B01AC01C501B4010F9437AC50
:106F70002BEA3AEA42E052E40F942FAD2B013C0198
:106F800020E030E0A9010F9428AD87FD1CC020E06F
:106F900030E040E85FE3C301B2010F9457AF181629
:106FA000ACF4412C512C50E8652E5FE3752E0EC0D9
:106FB000188A1F860BC0412C512C320125E030E08D
:106FC000388B2F8703C0412C512C3201A701960129
:106FD00060E070E080E89FE30F9437AC69837A83C8
:106FE0008B839C83C80101969E838D83AF85B8896E
:106FF0001196BA87A987A301920160E070E080E84A
:107000009FE30F9437AC6B877C878D879E8747E023
:107010002F853889429FF001439FF00D1124F88796
:10702000EF83E00FF11FEE0FFF1FEE0FFF1FE20DCA
:10703000F31D218132814381548169817A818B8161
:107040009C810F9429B04B015C01EF81F8858D8103
:107050009E81E80FF91FEE0FFF1FEE0FFF1FE20DDD
:10706000F31D2181328143815481C701B6010F9400
:1070700029B09B01AC01C501B4010F9438AC9B0150
:10708000AC016B857C858D859E850F9429B04B0165
:107090005C0127E0E985FA852E9FD0012F9FB00D76
:1070A0001124B887AF83FD01E00FF11FEE0FFF1F22
:1070B000EE0FFF1FE20DF31D2181328143815481C8
:1070C00069817A818B819C810F9429B069837A834D
:1070D0008B839C83AF81B8858D819E81A80FB91F5A
:1070E000AA0FBB1FAA0FBB1FA20DB31D11962D9196
:1070F0003D914D915C911497C701B6010F9429B051
:107100009B01AC0169817A818B819C810F9438ACA1
:107110009B01AC01C301B2010F9429B09B01AC01EA
:10712000C501B4010F9438AC60960FB6F894DEBF79
:107130000FBECDBFDF91CF911F910F91FF90EF90C8
:10714000DF90CF90BF90AF909F908F907F906F9087
:107150005F904F903F902F9008954F925F926F9263
:107160007F929F92AF92BF92CF92DF92EF92FF9267
:107170000F931F93CF93DF937C015B018A01E90199
:1071800090907D12911014C0FC0180819181A281A8
:10719000B381FA0180839183A283B383FB01808151
:1071A0009181A281B38188839983AA83BB837FC0A5
:1071B00091FE55C0FC012081318142815381609153
:1071C0006D1270916E1280916F12909170120F94E7
:1071D00029B02B013C01F50120813181428153818D
:1071E0006091711270917212809173129091741269
:1071F0000F9429B09B01AC01C301B2010F9438ACCC
:10720000F8016083718382839383F7012081318148
:10721000428153816091751270917612809177123C
:10722000909178120F9429B06B017C01F5012081B7
:107230003181428153816091791270917A128091EB
:107240007B1290917C120F9429B09B01AC01C70175
:10725000B6010F9438AC688379838A839B8390FE50
:1072600026C02091551230915612409157125091DC
:107270005812F80160817181828193810F9438AC3A
:10728000F801608371838283938320915912309136
:107290005A1240915B1250915C12688179818A8107
:1072A0009B810F9438AC688379838A839B83DF91B9
:1072B000CF911F910F91FF90EF90DF90CF90BF90F3
:1072C000AF909F907F906F905F904F9008952F9216
:1072D0003F924F925F926F927F928F929F92AF9266
:1072E000BF92CF92DF92EF92FF920F931F93CF93B3
:1072F000DF93CDB7DEB728970FB6F894DEBF0FBE89
:10730000CDBF8C011B019E012F5F3F4FAE014B5F34
:107310005F4F23DF20E030E0A9016D817E818F8106
:1073200098850F9428AD87FF07C01D821E821F829B
:107330001886FF24F39401C0F12C20E030E040E4F3
:1073400051EC69817A818B819C810F9428AD87FFF4
:107350000AC080E090E0A0E4B1EC89839A83AB831B
:10736000BC83FF24F39420E030E04FE753E46D81C9
:107370007E818F8198850F9457AF181654F480E062
:1073800090E0AFE7B3E48D839E83AF83B887FF249B
:10739000F39420E030E042E553E469817A818B8107
:1073A0009C810F9457AF18164CF480E090E0A2E552
:1073B000B3E489839A83AB83BC8303C0FF2009F4C1
:1073C00083C0C980DA80EB80FC808D809E80AF8096
:1073D000B88470907D1271100BC0F8018082918288
:1073E000A282B382F101C082D182E282F3826AC0BA
:1073F00070FE1CC0209155123091561240915712C8
:1074000050915812C501B4010F9437AC4B015C0187
:107410002091591230915A1240915B1250915C1296
:10742000C701B6010F9437AC6B017C0171FE4AC0F5
:1074300020915D1230915E1240915F125091601266
:10744000C501B4010F9429B02B013C0120916112B8
:10745000309162124091631250916412C701B601DB
:107460000F9429B09B01AC01C301B2010F9438AC59
:10747000F801608371838283938320916512309138
:1074800066124091671250916812C501B4010F94C1
:1074900029B04B015C012091691230916A12409130
:1074A0006B1250916C12C701B6010F9429B09B0169
:1074B000AC01C501B4010F9438ACF1016083718354
:1074C00082839383FF24F3948F2D28960FB6F8942C
:1074D000DEBF0FBECDBFDF91CF911F910F91FF9007
:1074E000EF90DF90CF90BF90AF909F908F907F9064
:1074F0006F905F904F903F902F900895CF93DF93C0
:107500001F92CDB7DEB7BE016F5F7F4F0F94C0589B
:107510000F90DF91CF910895682F87EF9FE00D9432
:10752000C8B80895FC012491222341F03091C00095
:1075300035FFFCCF2093C6000196F4CF22E030E067
:107540008AEA99E0F2CAFC012491222341F03091A9
:10755000C00035FFFCCF2093C6000196F4CF2AE08F
:1075600030E08AEA99E023CACF9362E074E08AEAC5
:1075700099E0D6D9C1E0C093A0026FEF89E69FE001
:107580000F94C8B8C093CD02CF91089562E174E022
:107590008AEA99E0C5D91092A00260E089E69FE0EE
:1075A0000F94C8B81092CD020895CF9363E274E0AF
:1075B0008AEA99E0B5D9109246131092451383E0F8
:1075C0000F942D266093910A7093920A8093930AE8
:1075D0009093940A1092900AC1E0C0930702C0935E
:1075E00006021092950A6FEF87E69FE00F94C8B8E5
:1075F000C093CE02CF91089562E374E08AEA99E0E5
:107600008FD91092070260E087E69FE00F94C8B818
:107610001092CE020895EF92FF920F931F93CF9393
:10762000DF931F92CDB7DEB789830F948154898190
:10763000823009F468C0B4F5882309F442C081306F
:1076400009F0F4C09FB7F8948091020184608093A0
:1076500002019FBFEFEFF1EE24E0E150F040204047
:10766000E1F700C000009FB7F894809102018B7F82
:10767000809302019FBF40E050E0BA018DEE9FE091
:107680000F94DAB840E050E0BA0181EF9FE00F9428
:10769000DAB80F90DF91CF911F910F91FF90EF908B
:1076A0000D943179833009F45CC0843009F0BEC098
:1076B0000F90DF91CF911F910F91FF90EF900D945C
:1076C000A0819FB7F89480910201846080930201A9
:1076D0009FBF2FEF81EE94E0215080409040E1F772
:1076E00000C000009FB7F894809102018B7F8093C7
:1076F00002019FBF0F90DF91CF911F910F91FF90DB
:10770000EF900D9429550F94295580EF05DF1092C5
:10771000841B1092831B6091851B84EC9FE00F9467
:10772000C8B863E87BE181EC9FE00F94AD549FB74C
:10773000F894809102018460809302019FBF8FEFD3
:1077400091EEE4E081509040E040E1F700C000009D
:107750009FB7F894809102018B7F809302019FBFB5
:1077600065C08EEE9FE00F9480694DED5FE062E0B2
:1077700081E00F9497859FB7F8948091020184600F
:10778000809302019FBFFFEF21EE84E0F150204083
:107790008040E1F700C000009FB7F894809102019B
:1077A0008B7F809302019FBF10928F0A10928E0AE6
:1077B00046ED5FE063E083E00F94978540918E0A89
:1077C00050918F0A63E083E00F948C54E12CF12CEC
:1077D00009E210E06FEFC7010F94E6B8C701B801E6
:1077E0000F9407B2892BD9F480918E0A90918F0A59
:1077F000019690938F0A80938E0A4FEC5FE063E0CE
:1078000083E00F94978540918E0A50918F0A63E030
:1078100083E00F948C548DEC9FE00F9480699FEF70
:10782000E91AF90AE114E0E1FE06A1F60F90DF91F2
:10783000CF911F910F91FF90EF90089580E1E7EFB6
:10784000FAE0A2ECBAE001900D928A95E1F7089572
:107850004F925F926F927F928F929F92AF92BF9260
:10786000CF92DF92EF92FF92CF93DF9300D01F92DF
:10787000CDB7DEB70F94CC258BE408DA882391F0DE
:107880003ADA6B017C0120E030E0A9010F9457AF98
:1078900087FD08C0C0926413D0926513E09266130E
:1078A000F092671382E5F2D9882359F024DA6B014C
:1078B0007C0120E030E0A9010F9428AD87FF83C050
:1078C00006C0C12CD12C60E8E62E6FEBF62E84E4C6
:1078D000DDD9882321F00FDA4B015C0106C0812C31
:1078E000912C50E8A52E5FEBB52E87E5CFD98823E4
:1078F00021F001DA2B013C0106C0412C512C40E85B
:10790000642E4FEB742E88E4C1D9882331F0F3D96B
:1079100069837A838B839C8308C080E090E0A0E831
:10792000BFEB89839A83AB83BC8320E030E0A9015D
:10793000C501B4010F9457AF87FD45C020E030E08A
:10794000A901C301B2010F9457AF87FD3CC020E0ED
:1079500030E0A90169817A818B819C810F9457AFB6
:1079600087FD31C020E030E0A901C501B4010F94CA
:1079700028AD882391F120E030E040E05FE3C501CD
:10798000B4010F9429B06B017C0129813A814B81AC
:107990005C81C301B2010F9429B04B015C01A701C6
:1079A0009601C701B6010F9429B02BED3FE049E4E1
:1079B00050E40F9429B09B01AC01C501B4010F94B0
:1079C0002FAD6B017C0120E030E0A901C701B601B9
:1079D0000F9457AF87FF04C00BC0C12CD12C760188
:1079E000C0926013D0926113E0926213F09263131D
:1079F000E0E4F0E18491882341F09091C00095FF8C
:107A0000FCCF8093C6003196F5CFEAE2FAE084918C
:107A1000882341F09091C00095FFFCCF8093C60071
:107A20003196F5CF409164135091651360916613C0
:107A30007091671322E030E08AEA99E076D880916D
:107A4000C00085FFFCCF8AE08093C600E4E2FAE044
:107A50008491882341F09091C00095FFFCCF8093E2
:107A6000C6003196F5CFC0906013D0906113E090BE
:107A70006213F090631320E030E0A901C701B60162
:107A80000F9428AD882361F022E030E0B701A60111
:107A90008AEA99E04AD88091C00085FFFCCF11C0E6
:107AA000EFE1FAE08491882341F09091C00095FFC6
:107AB000FCCF8093C6003196F5CF8091C00085FF42
:107AC000FCCF8AE08093C6000F900F900F900F902C
:107AD000DF91CF91FF90EF90DF90CF90BF90AF906C
:107AE0009F908F907F906F905F904F9008952F920E
:107AF0003F924F925F926F927F928F929F92AF923E
:107B0000BF92CF92DF92EF92FF920F931F93CF938A
:107B1000DF931F92CDB7DEB7E3E2F8E2859194914F
:107B2000EDDC81E00F947B1C8983E3E0F0E1E491DC
:107B30008E2F992781950CF490951C0184E00F9469
:107B40004D41AFEFBAE01D921D921D921C9213970A
:107B5000EBEFFAE02081318142815381A7EFBAE057
:107B60006D917D918D919C91E3E0CE2EEBE0DE2E28
:107B7000E12CF12C87010F94061960DE88E190E179
:107B80000E949E352DEC3CEC4CE85FE30F9429B04D
:107B90004B015C01B101882777FD8095982F0F94E8
:107BA000CAAD9B01AC01C501B4010F9429B0EAEC48
:107BB000FAE020813181428153810F9438AC2B014E
:107BC0003C01AAECBAE06D937D938D939C9313973F
:107BD000E3E5F2E0608171818281938160930E021E
:107BE00070930F02809310029093110220E030E016
:107BF00040E752E40F942FAD4B015C01A6ECBAE0D4
:107C00002D913D914D915C91E2ECFAE060817181A2
:107C100082819381A3EEBAE0BF93AF93FEECCF2EA7
:107C2000FAE0DF2E830172010F94580C82E00F946A
:107C3000C23E0F94CC250F94CD4180E00F947B1C65
:107C4000AFEFBAE01D921D921D921C921397EBEFBD
:107C5000FAE02081318142815381A7EFBAE06D9132
:107C60007D918D919C91A3E0CA2EABE0DA2EE12CA0
:107C7000F12C87010F940619E1DD2AE0229DC00155
:107C8000239D900D1124BC01882777FD8095982FA6
:107C90000F94CAADEAECFAE0208131814281538130
:107CA0000F9438AC2B013C01AAECBAE06D937D93A4
:107CB0008D939C93139720E030E040E05FE3E3E591
:107CC000F2E060817181828193810F9429B0609389
:107CD0000E0270930F02809310029093110220E025
:107CE00030E040E752E40F942FAD4B015C01A6EC6D
:107CF000BAE02D913D914D915C91E2ECFAE060810A
:107D0000718182819381A3EEBAE0BF93AF93BEEC01
:107D1000CB2EBAE0DB2E830172010F94580C0F9426
:107D2000CC2589810F947B1C80E090E0AFE4B3E424
:107D3000EFEFFAE080839183A283B383ABEFBAE0E5
:107D40002D913D914D915C91E7EFFAE06081718159
:107D50008281938113E0C12E1BE0D12EE12CF12C06
:107D60000FE413E40F94061981E00F900F900F9029
:107D70000F900F90DF91CF911F910F91FF90EF9097
:107D8000DF90CF90BF90AF909F908F907F906F903B
:107D90005F904F903F902F9008952F923F924F9277
:107DA0005F926F927F928F929F92AF92BF92CF928B
:107DB000DF92EF92FF920F931F93CF93DF93CDB794
:107DC000DEB729970FB6F894DEBF0FBECDBF3C01DA
:107DD00081E00F947B1C8F8382E06816710408F0A9
:107DE00081C2F301EF5FFF4EE491D301AA0FBB1FE5
:107DF000AA0FBB1FBA83A983A55BBD4FBE83AD830A
:107E00008D919D910D90BC91A02D80930E02909329
:107E10000F02A0931002B093110281E0062C01C062
:107E2000880F0A94EAF70F944D41E981FA81E950ED
:107E3000F54FF987E8871082118212821382E09051
:107E4000FF0AF090000B0091010B1091020B2091A2
:107E5000FB0A3091FC0A4091FD0A5091FE0A6091A4
:107E6000F70A7091F80A8091F90A9091FA0AE3E012
:107E7000CE2EEBE0DE2E0F940619E981FA81EE5347
:107E8000F54F2F0180E090E0A0E4B0E4808391837F
:107E9000A283B38320E030E040E752E460910E0219
:107EA00070910F0280911002909111020F942FADEA
:107EB0004B015C01E090CA0AF090CB0A0091CC0A19
:107EC0001091CD0A2091C60A3091C70A4091C80A84
:107ED0005091C90A6091C20A7091C30A8091C40A84
:107EE0009091C50AF3EE2F2EFAE03F2E3F922F928B
:107EF000AEECCA2EAAE0DA2E0F94580C0F94CC25C3
:107F00000F94631C80E00F947B1CA885B9851D929B
:107F10001D921D921C921397E090FF0AF090000BA7
:107F20000091010B1091020B2091FB0A3091FC0A89
:107F30004091FD0A5091FE0A6091F70A7091F80A8B
:107F40008091F90A9091FA0AB3E0CB2EBBE0DB2EC8
:107F50000F94061980E090E0A0E8BFEBF201808367
:107F60009183A283B38320E030E040E752E4609144
:107F70000E0270910F0280911002909111020F94E5
:107F80002FAD4B015C01E090CA0AF090CB0A009142
:107F9000CC0A1091CD0A2091C60A3091C70A4091AF
:107FA000C80A5091C90A6091C20A7091C30A8091AF
:107FB000C40A9091C50A3F922F92EEECCE2EEAE0D1
:107FC000DE2E0F94580C0F94CC2581E00F947B1C6F
:107FD00089819A81805F9F4E0E949E352DEC3CECFA
:107FE0004CE85FEB0F9429B0D2016D937D938D9394
:107FF0009C93139720E030E040E752E460910E023A
:1080000070910F0280911002909111020F942FAD88
:108010004B015C01E090CA0AF090CB0A0091CC0AB7
:108020001091CD0A2091C60A3091C70A4091C80A22
:108030005091C90A6091C20A7091C30A8091C40A22
:108040009091C50A3F922F920F94580C0F94CC2513
:108050000F94631C80E00F947B1CE885F9851082E7
:10806000118212821382E090FF0AF090000B0091BF
:10807000010B1091020B2091FB0A3091FC0A4091F8
:10808000FD0A5091FE0A6091F70A7091F80A8091FA
:10809000F90A9091FA0AF3E0CF2EFBE0DF2E0F945D
:1080A000061980E090E0A0E2B1E4F20180839183C0
:1080B000A283B38320E030E040E752E460910E02F7
:1080C00070910F0280911002909111020F942FADC8
:1080D0004B015C01E090CA0AF090CB0A0091CC0AF7
:1080E0001091CD0A2091C60A3091C70A4091C80A62
:1080F0005091C90A6091C20A7091C30A8091C40A62
:108100009091C50A3F922F92AEECCA2EAAE0DA2EC9
:108110000F94580C0F94CC250F94631C81E00F949E
:108120007B1C80E090E0A0E7B1ECF20180839183BA
:10813000A283B38320E030E040E05FE3AD81BE8105
:108140006D917D918D919C910F9429B060930E0259
:1081500070930F02809310029093110220E030E0A0
:1081600040E752E40F942FAD4B015C01E090CA0A46
:10817000F090CB0A0091CC0A1091CD0A2091C60A4A
:108180003091C70A4091C80A5091C90A6091C20A49
:108190007091C30A8091C40A9091C50A3F922F92B0
:1081A0000F94580C0F94CC25C3010E94A435F30101
:1081B000E851F54F81E080830F94CD410F94631C0B
:1081C00080E00F947B1C2AE037ED43E25FE3E88513
:1081D000F98560817181828193810F9437ACA88584
:1081E000B9856D937D938D939C931397E090FF0ACF
:1081F000F090000B0091010B1091020B2091FB0AF3
:108200003091FC0A4091FD0A5091FE0A6091F70AF4
:108210007091F80A8091F90A9091FA0AB3E0CB2E96
:10822000BBE0DB2E0F9406192AE037ED43E25FE353
:10823000E885F98560817181828193810F9438ACE2
:10824000A885B9856D937D938D939C931397F201C7
:1082500060837183828393832AE939E949E95EE384
:1082600060910E0270910F028091100290911102A4
:108270000F9429B020E030E040E752E40F942FAD96
:108280004B015C01E090CA0AF090CB0A0091CC0A45
:108290001091CD0A2091C60A3091C70A4091C80AB0
:1082A0005091C90A6091C20A7091C30A8091C40AB0
:1082B0009091C50A3F922F92EEECCE2EEAE0DE2E90
:1082C0000F94580C0F94CC2510920E0210920F02AE
:1082D00010921002109211020FB6F894DEBF0FBE7A
:1082E000CDBF62C192E06916710409F05DC1E3E09F
:1082F000F0E174901092FF0A1092000B1092010BA3
:108300001092020B2091FB0A3091FC0A4091FD0A69
:108310005091FE0A6091F70A7091F80A8091F90A6B
:108320009091FA0AF3E0CF2EFBE0DF2EE12CF12C46
:1083300087010F94061988E190E10E949E354B0158
:108340005C01672D772767FD7095872F972F0F9416
:10835000CAAD2B013C0120E030E040EC5FE3C501F9
:10836000B4010F9429B0A30192010F9429B069833D
:108370007A838B839C836093CA0A7093CB0A809321
:10838000CC0A9093CD0A609153027091540280916F
:1083900055029091560260930E0270930F028093E3
:1083A00010029093110220E030E040E752E40F9475
:1083B0002FAD4B015C012091C60A3091C70A409154
:1083C000C80A5091C90A6091C20A7091C30A80918B
:1083D000C40A9091C50AA3EE2A2EAAE03A2E3F9233
:1083E0002F92BEECCB2EBAE0DB2EE980FA800B8117
:1083F0001C810F94580C0F94CC251092FF0A1092F8
:10840000000B1092010B1092020B2091FB0A30918D
:10841000FC0A4091FD0A5091FE0A6091F70A7091A2
:10842000F80A8091F90A9091FA0A13E0C12E1BE034
:10843000D12EE12CF12C87010F9406198CE090E1EC
:108440000E949E359058A30192010F9429B0698330
:108450007A838B839C836093CA0A7093CB0A809340
:10846000CC0A9093CD0A20E030E040E752E46091DE
:108470000E0270910F0280911002909111020F94E0
:108480002FAD4B015C012091C60A3091C70A409183
:10849000C80A5091C90A6091C20A7091C30A8091BA
:1084A000C40A9091C50A3F922F920EECC02E0AE0AA
:1084B000D02EE980FA800B811C810F94580C0F9408
:1084C000CC258CE090E10E949E359B01AC010F947D
:1084D00038ACA30192010F9429B02B013C016093A9
:1084E000CA0A7093CB0A8093CC0A9093CD0A20E0FD
:1084F00030E040E05FE3609153027091540280915C
:108500005502909156020F9429B060930E02709319
:108510000F02809310029093110220E030E040E7B8
:1085200052E40F942FAD4B015C012091C60A3091AB
:10853000C70A4091C80A5091C90A6091C20A709155
:10854000C30A8091C40A9091C50A3F922F92830179
:1085500072010F94580C0F94CC2582E090E00E9499
:10856000A4358091FF0A9091000BA091010BB0916E
:10857000020B8093CA0A9093CB0AA093CC0AB093C3
:10858000CD0A10920E0210920F0210921002109259
:1085900011020F94631C81E08093EA0A0F900F9000
:1085A0000F900F900F900F908F8129960FB6F8942F
:1085B000DEBF0FBECDBFDF91CF911F910F91FF9016
:1085C000EF90DF90CF90BF90AF909F908F907F9073
:1085D0006F905F904F903F902F900D947B1CCF92A7
:1085E000DF92EF92FF920F931F9328D980E090E0E3
:1085F000D4DB81E090E0D1DBE090FF0AF090000B4B
:108600000091010B1091020B2091FB0A3091FC0AA2
:108610004091FD0A5091FE0A6091F70A7091F80AA4
:108620008091F90A9091FA0AF3E0CF2EFBE0DF2E59
:108630000F9406191F910F91FF90EF90DF90CF904C
:108640000D94631C0F9442A46093A90A7093AA0A24
:108650008093AB0A9093AC0A089520E030E0A90122
:1086600068EB71E084E50F9490A869E170E080E028
:1086700090E00F9471A484E50F94B6AB64E170E0D0
:1086800080E090E00D9471A47F928F929F92AF92C0
:10869000BF92CF92DF92EF92FF920F931F93CF93EF
:1086A000DF9300D01F92CDB7DEB710927B1A1092E5
:1086B0007A1A1092791A1092781A0F94815484EDD4
:1086C0009EE00F9480698E010F5F1F4F7E0125E0B1
:1086D000E20EF11C8AEA99E00E94AA338F3FEFEF85
:1086E0009E07C1F3F80181938F01EE15FF0591F705
:1086F00089809A80AB80BC808091C00085FFFCCFD0
:108700008BE28093C600C12CD12C7601ABE27A2E8D
:108710008091330B882309F450C00DE41AE0C8148B
:10872000D904EA04FB04A1F08AEA99E00E94AA3382
:108730008F3FFFEF9F07C1F32FEFC21AD20AE20A61
:10874000F20AF80181938F01FAE00D381F0739F71B
:108750006DE47AE086E79BE00E9436AC8091C00031
:1087600085FFFCCF7092C6000F945137C814D9040E
:10877000EA04FB0469F671DF60E086E79BE00E9493
:1087800069AD1092330BEFEDF7E285919491FC0106
:108790002491222341F03091C00035FFFCCF20937B
:1087A000C6000196F4CF8091C00085FFFCCF8AE01F
:1087B0008093C60080E090E000C00F900F900F9073
:1087C0000F90DF91CF911F910F91FF90EF90DF906D
:1087D000CF90BF90AF909F908F907F9008950F940F
:1087E00042A46093A90A7093AA0A8093AB0A90935B
:1087F000AC0AE0914F10F0915010EF5AFF4E80817B
:108800008130B9F4E3E7F7E285919491FC0124917A
:10881000222341F03091C00035FFFCCF2093C600E9
:108820000196F4CF8091C00085FFFCCF8AE0809351
:10883000C60008958AEA99E00E94C633E7E4F7E2A9
:1088400085919491FC012491222341F03091C00044
:1088500035FFFCCF2093C6000196F4CF4091351030
:108860005091361060913710709138104F5F5F4F04
:108870006F4F7F4F2AE030E08AEA99E00E9465342A
:108880008091C00085FFFCCF8AE08093C600A7CF0F
:108890008F929F92AF92BF92CF92DF92EF92FF9210
:1088A0000F931F93CF93DF93B0ECEB2EB6E0FB2E2C
:1088B00007EF1AE0C2ECDAE08EE6C82E8BE0D82E85
:1088C000F70181917F010E944636882319F10E94A9
:1088D000A6364B015C01F6018081811103C06091D5
:1088E000AD0A01C061E070E080E090E00F94CAAD95
:1088F000F80120813181428153810F9429B09B017D
:10890000AC01C501B4010F9438AC688379838A83C4
:108910009B8309C0F80180819181A281B381888302
:108920009983AA83BB830C5F1F4F2496FFEFCF1A56
:10893000DF0A84ECE81686E0F80611F686E40E9469
:1089400046368823D9F00E94A6366B017C016093DD
:10895000B20A7093B30A8093B40A9093B50A20E0E8
:1089600030E0A9010F9457AF181644F4C0920E02DC
:10897000D0920F02E0921002F0921102DF91CF919B
:108980001F910F91FF90EF90DF90CF90BF90AF902D
:108990009F908F9008957CDF89E40E94463688235B
:1089A00059F00E94A6366093B60A7093B70A809376
:1089B000B80A9093B90A08C01092B60A1092B70A82
:1089C0001092B80A1092B90A8AE40E9446368823A7
:1089D00059F00E94A6366093BA0A7093BB0A80933E
:1089E000BC0A9093BD0A08951092BA0A1092BB0A6D
:1089F0001092BC0A1092BD0A0895CF92DF92EF92B6
:108A0000FF92CF93DF93EC01BC016C5F7F4F0E941C
:108A1000673920E030E0A901609137027091380297
:108A20008091390290913A020F9438AC6B017C012D
:108A30009B01AC01688579858A859B850F9428AD5B
:108A400087FF04C0C886D986EA86FB86C0902B02C1
:108A5000D0902C02E0902D02F0902E02A7019601FA
:108A6000688579858A859B850F9457AF181624F4FD
:108A7000C886D986EA86FB86DF91CF91FF90EF907A
:108A8000DF90CF9008952F923F924F925F926F9216
:108A90007F928F929F92AF92BF92CF92DF92EF928E
:108AA000FF920F931F93CF93DF93CDB7DEB7AB97B2
:108AB0000FB6F894DEBF0FBECDBF9F878E87798B30
:108AC000688B5B8B4A8B3D8B2C8B1F8B0E8BED82C7
:108AD000DC018D909D90AD90BC904090F70A509035
:108AE000F80A6090F90A7090FA0ADB018D919D9165
:108AF0000D90BC91A02D88879987AA87BB87C090CD
:108B0000FB0AD090FC0AE090FD0AF090FE0A20914A
:108B1000FF0A3091000B4091010B5091020BEA8942
:108B2000FB8960817181828193810F9437AC688F5A
:108B3000798F8A8F9B8F80917E12811173C0AE894D
:108B4000BF898D909D90AD90BC90EA89FB89E080B3
:108B5000F18002811381A889B9892D913D914D91B0
:108B60005C91EE85FF856081718182819381FE0138
:108B70003596FF93EF93CC88DD880F94580CEE85E3
:108B8000FF8580819181A281B3818093F70A9093C0
:108B9000F80AA093F90AB093FA0AE889F989808162
:108BA0009181A281B3818093FB0A9093FC0AA093E8
:108BB000FD0AB093FE0AEA89FB8980819181A28136
:108BC000B3818093FF0A9093000BA093010BB093A5
:108BD000020BEC89FD8980819181A281B381809310
:108BE000030B9093040BA093050BB093060B0F900F
:108BF0000F90AB960FB6F894DEBF0FBECDBFDF91DE
:108C0000CF911F910F91FF90EF90DF90CF90BF9089
:108C1000AF909F908F907F906F905F904F903F901C
:108C20002F900895A3019201C501B4010F9437ACB0
:108C30002B013C0120E030E0A9010F9457AF530114
:108C40004201181624F0B7FAB094B7F8B094A7010F
:108C50009601688579858A859B850F9437AC6887EE
:108C600079878A879B8720E030E0A9010F9457AF6E
:108C7000288539854A855B8518160CF05058C50142
:108C8000B4010F9438AC6B017C0120E030E0A90105
:108C90000F9457AF18160CF052CF20E030E040EFA1
:108CA00051E4C701B6010F942FAD0F9415AD0F9489
:108CB00097AD7D876C87623071050CF440CF2091B1
:108CC000030B3091040B4091050B5091060BAC89BE
:108CD000BD896D917D918D919C910F9437AC6C8F76
:108CE0007D8F8E8F9F8F22242394312C8C859D85A0
:108CF000AA2797FDA095BA2F88A799A7AAA7BBA7CF
:108D0000DE011596BF83AE83B101882777FD80957C
:108D1000982F0F94CAAD6B017C0168A579A58AA52F
:108D20009BA50F94CAAD9B01AC01C701B6010F947E
:108D30002FAD6B017C01EE89FF8980809180A2803C
:108D4000B3802C8D3D8D4E8D5F8D0F9429B09B018E
:108D5000AC016091030B7091040B8091050B909115
:108D6000060B0F9438AC69837A838B839C83288DA0
:108D7000398D4A8D5B8DC701B6010F9429B02091C2
:108D8000FF0A3091000B4091010B5091020B0F94A0
:108D900038AC68A379A38AA39BA3288539854A8523
:108DA0005B85C701B6010F9429B02091FB0A309171
:108DB000FC0A4091FD0A5091FE0A0F9438AC6CA356
:108DC0007DA38EA39FA3A3019201C701B6010F94B7
:108DD00029B02091F70A3091F80A4091F90A509190
:108DE000FA0A0F9438ACFF81FF932E812F93DE0196
:108DF00011966D01E8A0F9A00AA11BA12CA13DA12B
:108E00004EA15FA10F94580CBFEF2B1A3B0A0F9095
:108E10000F90EC85FD852E163F0609F075CF8FCE9D
:108E20004F925F926F927F928F929F92AF92BF927A
:108E3000CF92DF92EF92FF920F931F93CF93DF9326
:108E4000CDB7DEB728970FB6F894DEBF0FBECDBF03
:108E500082EC9AE0D2DD0F9442A46093A90A709349
:108E6000AA0A8093AB0A9093AC0A8091C20A9091AF
:108E7000C30AA091C40AB091C50A8D839E83AF83B3
:108E8000B8879C01AD016091F70A7091F80A809152
:108E9000F90A9091FA0A0F9428AD811197C0409079
:108EA000C60A5090C70A6090C80A7090C90AA30108
:108EB00092016091FB0A7091FC0A8091FD0A9091E9
:108EC000FE0A0F9428AD811181C020E030E040E718
:108ED00052E460910E0270910F0280911002909105
:108EE00011020F942FAD4B015C01E090CA0AF09083
:108EF000CB0A0091CC0A1091CD0A83EE9AE09F93A1
:108F00008F932EECC22E2AE0D22EA30192016D8106
:108F10007E818F8198850F94580C0F900F908091CF
:108F2000C20A9091C30AA091C40AB091C50A809365
:108F3000F70A9093F80AA093F90AB093FA0A80917D
:108F4000C60A9091C70AA091C80AB091C90A809335
:108F5000FB0A9093FC0AA093FD0AB093FE0A80914D
:108F6000CA0A9091CB0AA091CC0AB091CD0A809305
:108F7000FF0A9093000BA093010BB093020B80911A
:108F8000CE0A9091CF0AA091D00AB091D10A8093D5
:108F9000030B9093040BA093050BB093060B28963C
:108FA0000FB6F894DEBF0FBECDBFDF91CF911F91FA
:108FB0000F91FF90EF90DF90CF90BF90AF909F9078
:108FC0008F907F906F905F904F900895E090E30AAC
:108FD0006091490270914A02882777FD8095982F09
:108FE0000F94CAAD20910E0230910F0240911002F1
:108FF000509111020F9429B02EE333EC4EE259E365
:109000000F9429B069837A838B839C838E010F5FD1
:109010001F4F2EEC3AE04AEC5AE066EC7AE082EC24
:109020009AE031DD7CCF4F925F926F927F928F9268
:109030009F92AF92BF92CF92DF92EF92FF920F93E7
:109040001F93CF93C62FE091E30AF0E0882309F441
:10905000D9C0DF01A152B54F8C918111AFC1809170
:10906000F70A9091F80AA091F90AB091FA0A809350
:10907000C20A9093C30AA093C40AB093C50A809110
:10908000FB0A9091FC0AA091FD0AB091FE0A809320
:10909000C60A9093C70AA093C80AB093C90A8091E0
:1090A000FF0A9091000BA091010BB091020B8093ED
:1090B000CA0A9093CB0AA093CC0AB093CD0AC09071
:1090C000030BD090040BE090050BF090060BC092C0
:1090D000CE0AD092CF0AE092D00AF092D10AEE0FD7
:1090E000FF1FEE0FFF1FE55CFD4F208131814281A4
:1090F0005381662349F060911B0270911C0280919C
:109100001D0290911E0208C060911F027091200202
:1091100080912102909122020F942FAD9B01AC010E
:10912000C701B6010F9438AC6093030B7093040B26
:109130008093050B9093060B83E09BE00F94A51A98
:1091400080900E0290900F02A0901002B090110239
:1091500020E030E040E752E460911702709118027D
:109160008091190290911A020F9429B060930E0217
:1091700070930F028093100290931102E091E30A22
:10918000F0E0E152F54F81E080834ADE2091DB0A76
:109190003091DC0A4091DD0A5091DE0A6091FF0AAD
:1091A0007091000B8091010B9091020B0F9437ACE2
:1091B0007B018C016093FF0A7093000B8093010B7D
:1091C0009093020B2091FB0A3091FC0A4091FD0A1A
:1091D0005091FE0A6091F70A7091F80A8091F90A9D
:1091E0009091FA0AE3E0CE2EEBE0DE2E0F94061902
:1091F00017DE80920E0290920F02A0921002B0929F
:109200001102DCC0E152F54F8081882309F4D6C0F9
:109210008090F70A9090F80AA090F90AB090FA0AA4
:109220008092C20A9092C30AA092C40AB092C50A60
:109230004090FB0A5090FC0A6090FD0A7090FE0A74
:109240004092C60A5092C70A6092C80A7092C90A30
:109250006091FF0A7091000B8091010B9091020BBD
:109260006093CA0A7093CB0A8093CC0A9093CD0A7C
:109270000091030B1091040B2091050B3091060B0C
:109280000093CE0A1093CF0A2093D00A3093D10ACC
:109290002091DB0A3091DC0A4091DD0A5091DE0A10
:1092A0000F9438AC7B018C016093FF0A7093000B24
:1092B0008093010B9093020B33E0C32E3BE0D32E3F
:1092C000A3019201C501B4010F9406191091E30A9C
:1092D000CC2389F02091D30A3091D40A4091D50A49
:1092E0005091D60A60911B0270911C0280911D0260
:1092F00090911E0210C02091D70A3091D80A409157
:10930000D90A5091DA0A60911F027091200280916F
:109310002102909122020F9438AC24E0129FF001B8
:109320001124E55CFD4F20813181428153810F94EE
:109330002FAD9B01AC016091030B7091040B8091E8
:10934000050B9091060B0F9437AC6093030B709351
:10935000040B8093050B9093060B83E09BE00F9426
:10936000A51AC0900E02D0900F02E0901002F0906B
:10937000110220E030E040E752E460911302709166
:10938000140280911502909116020F9429B06093F7
:109390000E0270930F028093100290931102E091DD
:1093A000E30AF0E0E152F54F10823ADDC0920E027E
:1093B000D0920F02E0921002F0921102CF911F9111
:1093C0000F91FF90EF90DF90CF90BF90AF909F9064
:1093D0008F907F906F905F904F900895AF92BF9263
:1093E000CF92DF92EF92FF920F931F93CF93DF9371
:1093F000D82F2091BA0A3091BB0A4091BC0A5091F3
:10940000BD0A6091B60A7091B70A8091B80A90912E
:10941000B90A0F9464AFC62F172F082FF92E609149
:10942000490270914A02882777FD8095982F0F9402
:10943000CAAD20910E0230910F024091100250915E
:1094400011020F9429B020E030E040E752E40F947D
:109450002FAD20E030E048EC52E40F942FAD209186
:10946000E30A2F93DF93FF920F931F93CF935B0138
:109470006C01B2E0EB2E01E020E046EB5AE062EC3A
:109480007AE087EF9AE00F940A038091C20A9091E4
:10949000C30AA091C40AB091C50A8093F70A9093B9
:1094A000F80AA093F90AB093FA0A8091C60A90913B
:1094B000C70AA091C80AB091C90A8093FB0A909389
:1094C000FC0AA093FD0AB093FE0A8091CA0A90910B
:1094D000CB0AA091CC0AB091CD0A8093FF0A909359
:1094E000000BA093010BB093020B8091CE0A9091D8
:1094F000CF0AA091D00AB091D10A8093030B909328
:10950000040BA093050BB093060B0F9442A4609339
:10951000A90A7093AA0A8093AB0A9093AC0A0F90A1
:109520000F900F900F900F900F90DF91CF911F91A0
:109530000F91FF90EF90DF90CF90BF90AF90089584
:10954000EC01E8E1FAE08491882341F09091C000B9
:1095500095FFFCCF8093C6003196F5CF70E04AE0CE
:1095600050E08AEA99E00E94A434F8940F94EB2F1B
:10957000179A1092E80A169A1092E90A149AE6E4E9
:10958000F0E18491882341F09091C00095FFFCCFD9
:109590008093C6003196F5CFE9EFF7E2859194917B
:1095A000FC012491222341F03091C00035FFFCCF13
:1095B0002093C6000196F4CF8091C00085FFFCCFB8
:1095C0008AE08093C6002097C9F0FE018491FE01D5
:1095D000882349F09091C00095FFFCCF8093C6008E
:1095E00031968491F5CF8091C00085FFFCCF8AE051
:1095F0008093C600CE010E947E3A06C0E5EBF7E2FA
:10960000859194910F94BE557894C6E0D0E021974F
:1096100051F068EC70E080E090E00F9471A480E07D
:109620000F941757F4CFF894FFCFCF92DF92EF92B9
:10963000FF920F931F93CF93C82F80914B1090915F
:109640004C10039714F40E94BAB50F9442A40091F1
:10965000A50A1091A60A2091A70A3091A80AC090E5
:10966000A90AD090AA0AE090AB0AF090AC0A6C1953
:109670007D098E099F09061717072807390740F447
:10968000012B022B032B21F064E083EB98E058DFE1
:1096900040910A0250910B0260910C0270910D02F0
:1096A000452B462B472B19F10F9442A40091A90A90
:1096B0001091AA0A2091AB0A3091AC0A601B710B81
:1096C000820B930B00910A0210910B0220910C0265
:1096D00030910D02061717072807390740F49091BB
:1096E000691380916813981302C0CC2349F0CF917D
:1096F0001F910F91FF90EF90DF90CF900D94860A0D
:10970000179A1092E80A169A1092E90A149AEFCF63
:109710000F94EB2F8091970A81113DC081E08093D7
:10972000970A8091351090913610A0913710B09122
:1097300038108093311090933210A0933310B0936F
:109740003410E6E4F0E18491882341F09091C00068
:1097500095FFFCCF8093C6003196F5CFEFEEF7E290
:1097600085919491FC012491222341F03091C00015
:1097700035FFFCCF2093C6000196F4CF8091C00046
:1097800085FFFCCF8AE08093C600E3EDF6E2859189
:1097900094910D94985508958091970A0895CF93C8
:1097A000DF93EC018091E30A8093980A84E50E949C
:1097B0004636811102C080E084C00E94A6360F9414
:1097C0009CAD6093980A6623B1F3E0E4F0E18491E4
:1097D000882341F09091C00095FFFCCF8093C60094
:1097E0003196F5CFCD36D10509F435C064F4C836CD
:1097F000D105B1F0C936D10509F052C0E7EAF7E268
:10980000A591B49124C0CA3DD10509F432C0CD3D23
:10981000D10509F045C0EBE9F7E2A591B4913DC04F
:10982000E9EAF7E285919491FC012491222309F45D
:1098300037C03091C00035FFFCCF2093C6000196A1
:10984000F3CF9091C00095FFFCCF8093C6008D911F
:109850008111F7CF25C0E5EAF7E2A591B4918D918A
:109860008823F1F09091C00095FFFCCF8093C60053
:10987000F6CFEDE9F7E2A591B4918D91882381F0BF
:109880009091C00095FFFCCF8093C600F6CF9091D9
:10989000C00095FFFCCF8093C6008D918111F7CF5A
:1098A0006091980A70E04AE050E08AEA99E00E94EC
:1098B0009D348091C00085FFFCCF8AE08093C60074
:1098C00081E0DF91CF9108954F925F926F927F92E6
:1098D0008F929F92AF92BF92CF92DF92EF92FF92C0
:1098E000CF93DF9300D01F92CDB7DEB72B013C01A1
:1098F00029833A834B835C838DEE9FE00F94B6B847
:109900008F3F01F58EEE9FE00F94B6B88F3FD1F4F4
:109910008FEE9FE00F94B6B88F3FA1F480EF9FE0E9
:109920000F94B6B88F3F71F440E050E0BA018DEE6D
:109930009FE00F94DAB840E050E0BA0181EF9FE079
:109940000F94DAB881EF9FE00F94BEB84B015C0131
:109950008DEE9FE00F94BEB86B017C0169817A8126
:109960008B819C812CE330E040E050E00F941AB2F0
:10997000C20ED31EE41EF51EB701A6018DEE9FE0B8
:109980000F94DAB8C301B20128EE33E040E050E0B2
:109990000F941AB2BA01A901480D591D6A1D7B1D09
:1099A00081EF9FE00F94DAB810922D0B10922E0BDE
:1099B00010922F0B1092300B0F900F900F900F9072
:1099C000DF91CF91FF90EF90DF90CF90BF90AF905D
:1099D0009F908F907F906F905F904F900895CF925F
:1099E000DF92EF92FF922091070B2223F1F020E00B
:1099F00030E040E05FE30F9429B06B017C0120E090
:109A000030E0A9010F9428AD882379F0A7019601D1
:109A1000C701B6010F9429B02BED3FE049E450E4B3
:109A20000F9429B09B01AC0104C020E030E040E875
:109A30005FE360E070E080E89FE30F942FADFF905C
:109A4000EF90DF90CF90089560913F0270914002B7
:109A50008091410290914202C2DF60933B02709379
:109A60003C0280933D0290933E020895CF93DF9392
:109A7000EC010F94513781E0D8DD80E00F94175747
:109A8000209799F0C233D10540F062E370E080E0A6
:109A900090E00F9471A4E297ECCFBE0180E090E0DB
:109AA0000F9471A4C0E0D0E0E4CFDF91CF9108958E
:109AB0002F923F924F925F926F927F928F929F92DE
:109AC000AF92BF92CF92DF92EF92FF921F93CF930C
:109AD000DF934B015C01CC24CA94DC2C76015DE061
:109AE000252E5AE0352E68EE462E63E0562E612C68
:109AF000712C1AE08091D20A811126C12FEFC21673
:109B0000D206E206F20651F0F7FC1EC10F9442A401
:109B10006C197D09683B7B4008F016C10F9442A484
:109B2000681979098A099B09693E73408105910585
:109B300008F47FC08091851B811177C0E5E1FAE0D0
:109B40008491882341F09091C00095FFFCCF8093D1
:109B5000C6003196F5CFE091980A24E0E29FF0012B
:109B60001124EE58F54E408151816281738121E0CC
:109B700030E08AEA99E00E949535E1E1FAE08491CB
:109B8000882341F09091C00095FFFCCF8093C600E0
:109B90003196F5CF6091980A70E04AE050E08AEA89
:109BA00099E00E949D34F1018491EDE0FAE0882370
:109BB00049F09091C00095FFFCCF8093C60031968C
:109BC0008491F5CFF7FE03C0E0E3F9E025C00F94E0
:109BD00042A44B015C01C701B6016854744F8F4F1A
:109BE0009F4F681979098A099B09A30192010F9473
:109BF0001AB2BA01A9012AE030E08AEA99E00E948B
:109C000065348091C00085FFFCCF0DC09091C000ED
:109C100095FFFCCF8093C60081918111F7CF809191
:109C2000C00085FFFCCF1093C6000F9442A44B01E7
:109C30005C010F94513780E0F8DC80E00F941757F7
:109C4000FFEFCF16DF06EF06FF0609F046C0809152
:109C5000960AE091980AF0E0EF01CC0FDD1FCC0FDF
:109C6000DD1FCE58D54EEE0FFF1FE658F54E882368
:109C7000D1F080819181BC01882777FD8095982F54
:109C80000F94CAAD20E030E040E85FE30F9437ACBA
:109C90009B01AC01688179818A819B810F9457AFC8
:109CA00087FF4DC027CF80819181BC01882777FD38
:109CB0008095982F0F94CAAD20E030E040E85FE334
:109CC0000F9438AC9B01AC01688179818A819B81BA
:109CD0000F9428AD18169CF50DCFF7FC0BCFE09133
:109CE000980AF0E0EF01CC0FDD1FCC0FDD1FCE583E
:109CF000D54EEE0FFF1FE658F54E80819181BC01D5
:109D0000882777FD8095982F0F94CAAD9B01AC01F1
:109D1000688179818A819B810F9437AC0F9497ADCC
:109D200097FF07C090958095709561957F4F8F4FF5
:109D30009F4F66307105810591050CF4DBCE0F94C1
:109D400042A46B017C01D6CEDF91CF911F91FF9091
:109D5000EF90DF90CF90BF90AF909F908F907F90CB
:109D60006F905F904F903F902F900895CF93DF9327
:109D70001F921F92CDB7DEB7BE016F5F7F4F88EF96
:109D80009FE00F94BE5489819A818156904F803A0A
:109D90009F4020F11A821982E4EEF9E08491882331
:109DA00041F09091C00095FFFCCF8093C6003196A2
:109DB000F5CF8091C00085FFFCCF8AE08093C6007C
:109DC000BE016F5F7F4F88EF9FE00F94AD5487EA2D
:109DD00099E00F948C5A81E00F9484580F900F9063
:109DE000DF91CF9108952F923F924F925F926F92A1
:109DF0007F928F929F92AF92BF92CF92DF92EF921B
:109E0000FF920F931F93CF93DF93CDB7DEB7CA585E
:109E1000D2400FB6F894DEBF0FBECDBFC958DD4F9C
:109E2000688379838A839B83C757D240FE01E75FAB
:109E3000FD4F88E2DF011D928A95E9F7E850F24074
:109E400080E991E0DF019C011D9221503040E1F753
:109E5000C75ADD4F19821882C955D240CE01875AA0
:109E60009D4F5C014E019FE6891A9EEF990ADE0123
:109E7000AF51BE4F3D0190EBC92E9FE0D92E23E29A
:109E8000E22EF12C00E010E0C359DD4F8882CD5660
:109E9000D240CD58DD4F9882C357D240B7018827B2
:109EA00077FD8095982F0F94CAADD3016D937D9364
:109EB0008D939D933D01F501619171915F0188271B
:109EC00077FD8095982F0F94CAADD4016D937D9343
:109ED0008D939D934D010F5F1F4F0630110559F073
:109EE000B501C6010F94BE54B5E0EB0EF11CE2E0E3
:109EF000CE0ED11CD3CFCF51DE4F288139814A817C
:109F00005B81C15ED140C958DD4F688179818A810A
:109F10009B81C757D2400F9428AD87FD2BC3FE010C
:109F2000EF51FE4F7F016E01FFE2CF1AFEEFDF0A15
:109F30003E012BEB621A2DEF720AC359DD4F0881E7
:109F4000CD56D240CD58DD4F1881C357D24085E061
:109F500090E0CF58DD4F99838883C157D240CF58C6
:109F6000DD4FA881B981C157D2401197CF58DD4F3D
:109F7000B983A883C157D240F7012089318942892A
:109F8000538964897589868997890F9437AC4B0109
:109F90005C01D80150962D913D914D915C91539764
:109FA00054966D917D918D919C9157970F9437ACFC
:109FB000A50194010F942FADF601929382937293B1
:109FC00062936F01D301BE92AE929E928E923D013A
:109FD00004501109B4E0EB1AF108CF58DD4FE881C5
:109FE000F981C157D240EF2B09F0B9CF6E01FFECD8
:109FF000CF1AFDEFDF0A3E0127E4621A2EEF720A44
:10A000002E013DE3430E511CCE0101967C0101E07F
:10A0100010E0D6018D909D90AD90BC901397149652
:10A020002D913D914D915C911797C501B4010F940D
:10A0300038AC9B01AC010F9438ACF70164A775A74D
:10A0400086A797A70130110541F080A691A6A2A688
:10A05000B3A684829582A682B7820F5F1F4FD30179
:10A0600014962D913D914D915C91179718966D9195
:10A070007D918D919C911B970F9437AC20E030E03F
:10A0800040EC50E40F9429B0F20160837183828325
:10A090009383F4E0CF0ED11C2CE2E20EF11C34E0ED
:10A0A000630E711C88E2480E511C0530110509F041
:10A0B000B0CF8E010B5A1F4F6E0191E5C90ED11C16
:10A0C00022242394312C2C0E3D1EA8ED2A0E311C87
:10A0D000F801B8972081318142815381F801608174
:10A0E0007181828193810F942FAD4B015C01E12C32
:10A0F000F12C3601F8E26F1A710826014E0C5F1C34
:10A10000F301EE0DFF1D2481358146815781C50184
:10A11000B4010F9429B09B01AC01D20114966D914A
:10A120007D918D919C9117970F9437ACF2016483C8
:10A13000758386839783F4E0EF0EF11C24E1E21629
:10A14000F104D9F6045D1F4F38E2C30ED11C02158D
:10A15000130509F0BDCF1E0185EB280E311C6E01E1
:10A1600091EBC90ED11C3E01A7EE6A1AADEF7A0A37
:10A1700014E0E12EF12C270100E010E0812C912C5D
:10A18000A12CB12CF601E00FF11FD301A00FB11FDC
:10A190002D913D914D915C9160817181828193817E
:10A1A0000F9429B09B01AC01B401C5010F9438ACE8
:10A1B0004B015C01BFEF4B1A5B0A0C5F1F4FE5E0E0
:10A1C0004E165104F9F69B01AC01D1016D917D91C0
:10A1D0008D919C910F9437ACF601208131814281A1
:10A1E00053810F942FADD3016D937D938D939C93E9
:10A1F0001397B1E0EB1AF108E8E22E1A3108FCE2FD
:10A20000CF1AD10824E0621A7108E114F10409F0B0
:10A21000B2CFCB50DE4F88819981AA81BB81C55FC7
:10A22000D140C957DD4F88839983AA83BB83C75820
:10A23000D2408E01075F1D4FDE01AF5CBD4FC55898
:10A24000DD4FB983A883CB57D240C359DD4F288057
:10A25000CD56D240CD58DD4F3880C357D240FE0195
:10A26000EF51FE4FC358DD4FF983E883CD57D240FD
:10A27000C358DD4FA881B981CD57D240CD90DD9034
:10A28000ED90FD90C358DD4FB983A883CD57D240E0
:10A29000C958DD4F288139814A815B81C757D24037
:10A2A000C701B6010F9428AD1816B4F0C358DD4F9E
:10A2B000E881F981CD57D24020813181428153819B
:10A2C000C958DD4F688179818A819B81C757D24007
:10A2D0000F9428AD1816FCF4CF58DD4F2881398132
:10A2E000C157D2402430310509F01FC1C957DD4F95
:10A2F000288139814A815B81C758D240C958DD4FD6
:10A30000688179818A819B81C757D2400F9457AF6A
:10A3100018160CF00AC1D80114968D919D910D90DC
:10A32000BC91A02DC158DD4F88839983AA83BB833C
:10A33000CF57D240F8014080518062807380C55869
:10A34000DD4FA881B981CB57D2408D919D910D9061
:10A35000BC91A02DC359DD4F88839983AA83BB8309
:10A36000CD56D240D1018D919D910D90BC91A02DE3
:10A37000CD57DD4F88839983AA83BB83C358D240CE
:10A38000A7019601C958DD4F688179818A819B8137
:10A39000C757D2400F9437ACCD58DD4F68837983CF
:10A3A0008A839B83C357D24020E030E040E450E4EE
:10A3B0000F948CB06B017C01A3019201C158DD4F59
:10A3C000688179818A819B81CF57D2400F9437ACC5
:10A3D0004B015C0120E030E040EC50E4C359DD4F1C
:10A3E000688179818A819B81CD56D2400F9429B0B2
:10A3F0009B01AC01C501B4010F942FADA7019601DB
:10A400000F9429B06B017C0120E030E040E05FE375
:10A41000C301B2010F9429B04B015C01CD58DD4F4F
:10A42000288139814A815B81C357D240CA01B90171
:10A430000F9429B09B01AC01C501B4010F9429B060
:10A440009B01AC01C701B6010F9438AC6B017C01D4
:10A45000CD57DD4F288139814A815B81C358D24075
:10A46000F10164817581868197810F9437ACC3595E
:10A47000DD4F288139814A815B81CD56D2400F94CE
:10A480002FAD4B015C01C359DD4F288139814A81D1
:10A490005B81CD56D240CA01B9010F9438ACA301FB
:10A4A00092010F9429B02B013C01C359DD4F288143
:10A4B00039814A815B81CD56D240C158DD4F6881D8
:10A4C00079818A819B81CF57D2400F9429B09B011B
:10A4D000AC01C301B2010F9438AC20E030E040EC95
:10A4E00050E40F942FAD9B01AC01C501B4010F9452
:10A4F00037ACCD58DD4F288139814A815B81C35704
:10A50000D2400F9429B09B01AC01C701B6010F9452
:10A5100038ACCD57DD4F288139814A815B81C358E2
:10A52000D2400F9438AC4B015C01CF58DD4F2881ED
:10A530003981C157D2402F5F3F4FCF58DD4F39830C
:10A540002883C157D2400C5F1F4FC558DD4F88810B
:10A550009981CB57D2400496C558DD4F99838883A3
:10A56000CB57D24094E0290E311C2530310509F03B
:10A570007FCE04C0812C912CA12CB12CB401C5013B
:10A58000C657DD4F0FB6F894DEBF0FBECDBFDF91CB
:10A59000CF911F910F91FF90EF90DF90CF90BF90E0
:10A5A000AF909F908F907F906F905F904F903F9073
:10A5B0002F9008958091610B8823C9F086EA9FE06F
:10A5C0000F94B6B8882399F060916C1A70916D1A47
:10A5D00080916E1A90916F1A06DC20914D1930917E
:10A5E0004E1940914F19509150190D942FAD60E0C4
:10A5F00070E0CB0108954F925F926F927F928F929D
:10A600009F92AF92BF92CF92DF92EF92FF920F9301
:10A610001F93CF93DF93CDB7DEB728970FB6F8948B
:10A62000DEBF0FBECDBF0F94CC2580914902909123
:10A630004A0290936D0B80936C0BE091E30AF0E07B
:10A64000EE0FFF1FE658F54E60817181882777FD78
:10A650008095982F0F94CAAD6093550B7093560B4D
:10A660008093570B9093580B8091E10A9091E20AE6
:10A670009093540B8093530B0F9442A460933B0B25
:10A6800070933C0B80933D0B90933E0B8091F70AA7
:10A690009091F80AA091F90AB091FA0A89839A83F5
:10A6A000AB83BC838093430B9093440BA093450BE7
:10A6B000B093460B4090FB0A5090FC0A6090FD0A54
:10A6C0007090FE0A4092470B5092480B6092490BE3
:10A6D00070924A0B8091FF0A9091000BA091010BA0
:10A6E000B091020B8D839E83AF83B88780934B0B11
:10A6F00090934C0BA0934D0BB0934E0B6091030BBA
:10A700007091040B8091050B9091060B60934F0B99
:10A710007093500B8093510B9093520B20E030E0DC
:10A7200040E85FE30F9437AC6093030B7093040B26
:10A730008093050B9093060B83EE9AE09F938F9383
:10A74000812C912CB8ECAB2EB3E4BB2E13E0C12EC0
:10A750001BE0D12EED80FE800F811885A3019201B0
:10A7600069817A818B819C810F94580C20E030E0C4
:10A7700040EA51E46091FF0A7091000B8091010B57
:10A780009091020B0F9438AC2B013C010F900F906D
:10A7900020E030E042E553E40F9457AF18164CF038
:10A7A0004092FF0A5092000B6092010B7092020BD4
:10A7B0000CC080E090E0A2E5B3E48093FF0A9093A0
:10A7C000000BA093010BB093020BE090FF0AF090F6
:10A7D000000B0091010B1091020B2091FB0A3091AC
:10A7E000FC0A4091FD0A5091FE0A6091F70A7091AF
:10A7F000F80A8091F90A9091FA0AA3EE6A2EAAE06B
:10A800007A2E7F926F92812C912CB0E7AB2EB1E41F
:10A81000BB2EE3E0CE2EEBE0DE2E0F94580C109210
:10A820007B1A10927A1A10927D1A10927C1A10924A
:10A830007F1A10927E1A80E090E0A8E4B2E4809340
:10A84000F70A9093F80AA093F90AB093FA0A80E005
:10A8500090E0AEE3B3E48093FB0A9093FC0AA093EC
:10A86000FD0AB093FE0AE090FF0AF090000B009101
:10A87000010B1091020B7F926F92812C912CF8E4C6
:10A88000AF2EF2E4BF2E9C01AD01C501B4010F94BF
:10A89000580C1092E20A1092E10A0F900F900F905C
:10A8A0000F9028960FB6F894DEBF0FBECDBFDF9194
:10A8B000CF911F910F91FF90EF90DF90CF90BF90BD
:10A8C000AF909F908F907F906F905F904F900D947E
:10A8D000CC25E091E30A84E0E89FF0011124EE58D2
:10A8E000F54E4081518162817381E4EAF9E08491FF
:10A8F000882341F09091C00095FFFCCF8093C60063
:10A900003196F5CF22E030E08AEA99E00E94953551
:10A91000E0EAF9E08491882341F09091C00095FF2E
:10A92000FCCF8093C6003196F5CF6091E30A70E0CA
:10A930004AE050E08AEA99E00E949D34ECE9F9E0AF
:10A940008491882341F09091C00095FFFCCF8093C3
:10A95000C6003196F5CF4091601A5091611A60910E
:10A96000621A7091631A21E030E08AEA99E00E944D
:10A9700095358091C00085FFFCCF8AE08093C600AA
:10A980000895CF93DF9300D000D0CDB7DEB7179AEC
:10A990001092E80A169A1092E90AE7E9F9E0849120
:10A9A000882341F09091C00095FFFCCF8093C600B2
:10A9B0003196F5CF8091C00085FFFCCF8AE080936F
:10A9C000C60083E40F9469453C0120902D1030901F
:10A9D0002E1040902F10509030100F94331B281AD7
:10A9E000390A410851080E94F7BA281A390A410861
:10A9F000510857FE03C0212C312C2101909169137D
:10AA000080916813981799F0E091681327E5E29F09
:10AA1000F0011124E659FC4E20E030E040E752E41A
:10AA200062A173A184A195A10F9429B008C060917F
:10AA30000E0270910F0280911002909111020F94FA
:10AA400097AD7E836D830F94DD0A0E94A1B31092AF
:10AA5000780B789420E030E040E85FE36091030BEE
:10AA60007091040B8091050B9091060B0F9437ACFD
:10AA700069837A838B839C83E090FF0AF090000BBC
:10AA80000091010B1091020B2091FB0A3091FC0AFE
:10AA90004091FD0A5091FE0A6091F70A7091F80A00
:10AAA0008091F90A9091FA0AA3EEBAE0BF93AF93AE
:10AAB000812C912CE8ECAE2EE3E4BE2EDE01119643
:10AAC0006D010F94580C20E030E040E85FE36091A6
:10AAD000030B7091040B8091050B9091060B0F9462
:10AAE00037AC69837A838B839C832FE832EC45EF04
:10AAF0005FE36091FF0A7091000B8091010B9091D0
:10AB0000020B0F9438AC6B017C0167E074E06619AE
:10AB10007709F4E076956795FA95E1F780E090E0A3
:10AB20000F94C8AD20914D1930914E1940914F1995
:10AB3000509150190F942FAD9B01AC01C701B60184
:10AB40000F9438AC7B018C012091FB0A3091FC0AF8
:10AB50004091FD0A5091FE0A6091F70A7091F80A3F
:10AB60008091F90A9091FA0AA3EEBAE0BF93AF93ED
:10AB7000812C912CA0E2AA2EA2E4BA2EDE0111961D
:10AB80006D010F94580CB201A10181E99FE00F946F
:10AB9000DAB80F900F900F900F9005E71FE0F12C9F
:10ABA000B3E0EB2E80917E12882341F18F2D6E2D24
:10ABB0000F94E6B1B5E18B02F001112423E092027B
:10ABC000E00DF11D1124EE0FFF1FEE0FFF1FE258E5
:10ABD000FD4E20E030E04AE754E4618172818381D8
:10ABE00094810F9429B020E030E040E05FE30F94BF
:10ABF00038AC0F9405AE0F9497AD02C060E070E0E2
:10AC0000C8010F94E2B8F3940E5F1F4F89E0F81269
:10AC1000C9CFB30183E79FE00F94E2B84091F70AF0
:10AC20005091F80A6091F90A7091FA0A8DE99FE053
:10AC30000F94DAB84091FB0A5091FC0A6091FD0A2A
:10AC40007091FE0A81EA9FE00F94DAB84091FF0A02
:10AC50005091000B6091010B7091020B8DE89FE009
:10AC60000F94DAB8BE016B5F7F4F89E89FE00F94C5
:10AC7000AD54E091E30AF0E0EE0FFF1FE658F54E09
:10AC800060818CE89FE00F94C8B86091781A8BE8D7
:10AC90009FE00F94C8B86091E10A88E89FE00F94A4
:10ACA000C8B861E085EA9FE00F94C8B80F94CC253E
:10ACB000E2E9F9E08491882341F09091C00095FF8A
:10ACC000FCCF8093C6003196F5CF83E40F9469459D
:10ACD0004AE050E0BC018AEA99E00E94F434E7E8D7
:10ACE000F9E08491882341F09091C00095FFFCCF5A
:10ACF0008093C6003196F5CF8091C00085FFFCCFD0
:10AD00008AE08093C600F894FFCF6C987498EAE6C6
:10AD1000F0E080818160808380818D7F8083EC9AE8
:10AD200008951F920F920FB60F9211240BB60F9237
:10AD30002F933F934F935F936F937F938F939F9343
:10AD4000AF93BF93EF93FF93EC98E2E8F9E084911F
:10AD5000882341F09091C00095FFFCCF8093C600FE
:10AD60003196F5CF8091C00085FFFCCF8AE08093BB
:10AD7000C6008091780B811104DEFF91EF91BF91A5
:10AD8000AF919F918F917F916F915F914F913F9183
:10AD90002F910F900BBE0F900FBE0F901F90189524
:10ADA000BF92CF92DF92EF92FF920F931F93CF93B8
:10ADB000DF93CDB7DEB7E1970FB6F894DEBF0FBED5
:10ADC000CDBF88E89FE00F94B6B8B82EBE01605D95
:10ADD0007F4F89E89FE00F94BE54EBE2F8E0849146
:10ADE000882341F09091C00095FFFCCF8093C6006E
:10ADF0003196F5CF68A979A94AE050E08AEA99E04E
:10AE00000E94A4348E01015E1F4F85E9E82E8FE079
:10AE1000F82ED02EC12EC7010F94B6B8F801819339
:10AE20008F01FFEFEF1AFF0A8DE9E8168FE0F806B1
:10AE300091F71FA2ED2DFC2D8191882339F090917F
:10AE4000C00095FFFCCF8093C600F6CF66E278E0A5
:10AE50008D2D9C2D0F9465B5CF92DF928FE198E0F8
:10AE60009F938F938E010F5F1F4F1F930F930F942C
:10AE70008AB60F900F900F900F900F900F907E0159
:10AE800095E0E90EF11CF7018081882349F09927AC
:10AE900087FD90950F9454B5F70181937F01F3CF0F
:10AEA00060E0C8010E9417B481E99FE00F94BEB82A
:10AEB000F62EE72ED82EC92EE4E0F8E08491882300
:10AEC00041F09091C00095FFFCCF8093C600319671
:10AED000F5CF2AE030E04F2D5E2D6D2D7C2D8AEAD6
:10AEE00099E00E94003561E080E098E00E9417B48C
:10AEF0006BEF77E0C8010F9470B58DE99FE00F9478
:10AF0000BEB86CA77DA78EA79FA7CE018C960F9485
:10AF10000D5DBC01C8010F94FFB568EF77E0C80173
:10AF20000F9465B581EA9FE00F94BEB86CA77DA72A
:10AF30008EA79FA7CE018C960F940D5DBC01C80112
:10AF40000F94FFB561EF77E0C8010F9465B560E03D
:10AF5000C8010E9417B46CEE77E0C8010F9470B579
:10AF60008DE89FE00F94BEB86CA77DA78EA79FA722
:10AF7000CE018C960F940D5DBC01C8010F94FFB5F6
:10AF800060E0C8010E9417B461E081EE97E00E9482
:10AF900017B489A98F9388A98F938AED97E09F931F
:10AFA0008F931F930F930F948AB660E0C8010E949D
:10AFB00017B463ED77E0C8010F9470B58B2D90E066
:10AFC0009DA78CA7CE018C960F946F5FBC01C80122
:10AFD0000F94FFB560E0C8010E9417B4CF92DF92D2
:10AFE000EF92FF928AEC97E09F938F931F930F93BA
:10AFF0000F948AB660E0C8010E9417B461E086EC45
:10B0000097E00E9417B40FB6F894DEBF0FBECDBF15
:10B01000E1960FB6F894DEBF0FBECDBFDF91CF91A2
:10B020001F910F91FF90EF90DF90CF90BF90089508
:10B030004F925F926F927F92AF92BF92CF92DF92C8
:10B04000EF92FF920F931F93CF93DF93CDB7DEB7AD
:10B05000E0970FB6F894DEBF0FBECDBF2B013C01C9
:10B0600069017A0180914C0A8111E5C0F8940F942E
:10B07000131B80912D1090912E10A0912F10B09144
:10B0800030108093480A9093490AA0934A0AB093DB
:10B090004B0A0F94331B4091480A5091490A609122
:10B0A0004A0A70914B0A481B590B61097109409378
:10B0B000480A5093490A60934A0A70934B0A0E94C7
:10B0C000F7BA4091480A5091490A60914A0A709132
:10B0D0004B0A481B590B610971094093480A509368
:10B0E000490A60934A0A70934B0A909169138091C0
:10B0F0006813981799F0E091681387E5E89FF001CD
:10B100001124E659FC4E20E030E040E752E462A111
:10B1100073A184A195A10F9429B008C060910E027B
:10B1200070910F0280911002909111026093340A85
:10B130007093350A8093360A9093370A0F94DD0A8C
:10B1400080E1E7EFFAE0A8E3BAE001900D928A957A
:10B15000E1F78091E30A8093330A8091090280939A
:10B16000320A0E94A1B31092780B81E080934C0ABE
:10B17000789420E030E0A901C301B2010F9428AD1A
:10B1800081110AC020E030E0A901C701B6010F9487
:10B1900028AD882309F44FC061EC77E0FE013196B9
:10B1A0005F01CF010F9470B5F50101900020E9F720
:10B1B0008F01015011092091400A3091410A4091BC
:10B1C000420A5091430AC301B2010F9438AC23E004
:10B1D00048E00F9493B26EEB77E0C5010F9465B52C
:10B1E000F50101900020E9F78F010150110923E0DA
:10B1F00046E0C701B6010F9493B26BEB77E0C5014F
:10B200000F9465B5F50101900020E9F78F01015019
:10B2100011096091530270915402809155029091EE
:10B22000560223E048E00F9493B260E0C5010E940B
:10B2300017B40E94ADB5E0960FB6F894DEBF0FBE0E
:10B24000CDBFDF91CF911F910F91FF90EF90DF90D5
:10B25000CF90BF90AF907F906F905F904F90089588
:10B2600020E030E0A90160E070E080E291E4E0CE0F
:10B2700020E030E0A901CA01B901DACE2F923F9255
:10B280004F925F926F927F928F929F92AF92BF92F6
:10B29000CF92DF92EF92FF920F931F93CF93DF93A2
:10B2A000CDB7DEB728970FB6F894DEBF0FBECDBF7F
:10B2B00080910702882309F418C183E00F942D269A
:10B2C0004B015C010F949D068091910A9091920A26
:10B2D000A091930AB091940A24013501481A590AA1
:10B2E0006A0A7B0AD301C201895E9E4FAF4FBF4FEE
:10B2F0008F329240A105B10508F4F7C0C301B20135
:10B300000F94CAAD20E030E04CE853E40F942FAD29
:10B310006B017C0120E030E040E450E40F9429B060
:10B320000F9497AD69837A838B839C8309811A81FB
:10B3300020E030E040E252E4C701B6010F9429B0AA
:10B340000F9497AD6D837E838F8398878D819E81C7
:10B350002090451330904613319421943108809207
:10B36000910A9092920AA092930AB092940A109233
:10B3700046131092451314141504160417043CF4D4
:10B380002016310654F0821593056CF406C00215A0
:10B3900013051CF02816390634F48091900A8F5F4B
:10B3A0008093900A02C01092900AE2E4F4E0819146
:10B3B000882339F09091C00095FFFCCF8093C600A0
:10B3C000F6CF2AE030E0B501A4018AEA99E00E94B4
:10B3D0006534E9E4F4E08191882339F09091C0006C
:10B3E00095FFFCCF8093C600F6CF22E030E0B70196
:10B3F000A6018AEA99E00E949535EEE4F4E0819195
:10B40000882339F09091C00095FFFCCF8093C6004F
:10B41000F6CF4AE050E069817A818AEA99E00E9499
:10B420009D34E5E5F4E08191882339F09091C000E6
:10B4300095FFFCCF8093C600F6CF4AE050E06D81C7
:10B440007E818AEA99E00E949D34ECE5F4E08191E6
:10B45000882339F09091C00095FFFCCF8093C600FF
:10B46000F6CF4AE050E0B1018AEA99E00E949D34AB
:10B47000E2E6F4E08191882339F09091C00095FFD5
:10B48000FCCF8093C600F6CF6091900A70E04AE04E
:10B4900050E08AEA99E00E94A4348091900A8630B4
:10B4A00020F168E674E08AEA99E00E949034809185
:10B4B0000602882349F068E974E08AEA99E00E946C
:10B4C00090341092060211C068EB74E08AEA99E0A9
:10B4D0000E949034CDDE61E08CEF9FE00E94F5B4D5
:10B4E00081E08093950A1092070228960FB6F8948F
:10B4F000DEBF0FBECDBFDF91CF911F910F91FF90A7
:10B50000EF90DF90CF90BF90AF909F908F907F9003
:10B510006F905F904F903F902F9008958F929F92E1
:10B52000AF92BF92CF92DF92EF92FF920F931F9351
:10B53000CF93DF9300D01F92CDB7DEB79B01AC0154
:10B5400080914C0A882309F497C08091330A809334
:10B55000E30A8091340A9091350AA091360AB0919D
:10B56000370A80930E0290930F02A0931002B093BB
:10B5700011026091440A7091450A8091460A9091A7
:10B58000470A0F9437AC69837A838B839C83CE01FF
:10B5900001960F94A51A20E030E040E551E4609157
:10B5A00053027091540280915502909156020F946B
:10B5B0002FAD4B015C01E090400AF090410A0091F0
:10B5C000420A1091430A20913C0A30913D0A409171
:10B5D0003E0A50913F0A6091380A7091390A809171
:10B5E0003A0A90913B0AE3EEFAE0FF93EF93E4E42A
:10B5F000CE2EEAE0DE2E0F94580C0F94CC2580E17D
:10B60000E8E3FAE0A7EFBAE001900D928A95E1F73E
:10B6100080E1E7EFFAE0A2ECBAE001900D928A95A2
:10B62000E1F74091480A5091490A60914A0A7091A5
:10B630004B0A4093140E5093150E6093160E7093A0
:10B64000170E8FE59DE00E948B9B8091480A909198
:10B65000490AA0914A0AB0914B0A80932D10909309
:10B660002E10A0932F10B093301081E08093780BB0
:10B6700010924C0A0F900F900F900F900F900F9018
:10B68000DF91CF911F910F91FF90EF90DF90CF90BE
:10B69000BF90AF909F908F90089560E070E0CB01D5
:10B6A0003DCF60E070E0CB0139CFE6EAF7E084916E
:10B6B000882341F09091C00095FFFCCF8093C60095
:10B6C0003196F5CF4091F70A5091F80A6091F90A46
:10B6D0007091FA0A23E030E08AEA99E00E949535F9
:10B6E000E3EAF7E08491882341F09091C00095FF50
:10B6F000FCCF8093C6003196F5CF4091FB0A509164
:10B70000FC0A6091FD0A7091FE0A23E030E08AEAAB
:10B7100099E00E949535E0EAF7E08491882341F0B2
:10B720009091C00095FFFCCF8093C6003196F5CF75
:10B730004091FF0A5091000B6091010B7091020B38
:10B7400023E030E08AEA99E00E949535EEE9F7E0DF
:10B750008491882341F09091C00095FFFCCF8093A5
:10B76000C6003196F5CF8091C00085FFFCCF8AE0FE
:10B770008093C6000895E6E8F7E08491882341F0BD
:10B780009091C00095FFFCCF8093C6003196F5CF15
:10B790000F943B26AB01BC0123E030E08AEA99E03C
:10B7A0000E949535E3E8F7E08491882341F0909179
:10B7B000C00095FFFCCF8093C6003196F5CF81E0A5
:10B7C0000F943B26AB01BC0123E030E08AEA99E00C
:10B7D0000E949535E0E8F7E08491882341F090914C
:10B7E000C00095FFFCCF8093C6003196F5CF82E074
:10B7F0000F943B26AB01BC0123E030E08AEA99E0DC
:10B800000E949535EEE7F7E08491882341F090910E
:10B81000C00095FFFCCF8093C6003196F5CF809194
:10B82000C00085FFFCCF8AE08093C6000895EF92A8
:10B83000FF920F931F93CF93DF93EAE6F7E0849193
:10B84000882341F09091C00095FFFCCF8093C60003
:10B850003196F5CF0EE712E1F8E6EF2EF7E0FF2E76
:10B86000C0E0D0E0F801EC0FFD1F418152816381FF
:10B87000748123E030E08AEA99E00E949535F7016F
:10B880008491E8E6F7E0882349F09091C00095FFA5
:10B89000FCCF8093C60031968491F5CF2496CC31AD
:10B8A000D10501F7045E1F4FF3E102341F07C1F613
:10B8B000E7E6F7E08491882341F09091C00095FF7E
:10B8C000FCCF8093C6003196F5CF8091C00085FFF4
:10B8D000FCCF8AE08093C600DF91CF911F910F913A
:10B8E000FF90EF9008952F923F924F925F926F9248
:10B8F0007F928F929F92AF92BF92CF92DF92EF9200
:10B90000FF920F931F93CF93DF93CDB7DEB7C95547
:10B91000D1090FB6F894DEBF0FBECDBF82ED94E023
:10B920000E945C368823B1F08091451090914610BA
:10B930006AE270E005960F940AB6009711F0DC01F8
:10B940001C92809145109091461005960F948B554E
:10B950000C94E58B87ED94E00E945C36882309F413
:10B9600081C18DED94E00E945C36882391F0809136
:10B97000851B882311F40C94E58B0F9442A46093EB
:10B98000720B7093730B8093740B9093750B0C94E4
:10B99000E58B82EE94E00E945C36882361F0609132
:10B9A000310B7091320B4AE050E08AEA99E00E9434
:10B9B000F4340C94E58B86EE94E00E945C36882388
:10B9C000C1F08091851B882361F06091831B709189
:10B9D000841B4AE050E08AEA99E00E94A4340C9467
:10B9E000E58B69EE74E08AEA99E00E9490340C9449
:10B9F000E58B8BEF94E00E945C36882379F16091AF
:10BA00004510709146106D5F7F4F21E041E086E761
:10BA10009BE00E94D9AD8091670D9091680DA09137
:10BA2000690DB0916A0D8093140E9093150EA0933A
:10BA3000160EB093170E8FE59DE00E94C29A2091DA
:10BA4000C00025FFFCCF8093C6000A9721F760E075
:10BA500086E79BE00E9469AD0C94E58B8EEF94E045
:10BA60000E945C36882399F00E942D4381E08093E8
:10BA7000330B60914510709146106C5F7F4F21E051
:10BA800040E086E79BE00E94D9AD0C94E58B82E014
:10BA900095E00E945C36882309F44FC08091851B95
:10BAA000882309F49ECF1092300A10922F0AE5E005
:10BAB000F5E08191882339F09091C00095FFFCCF8B
:10BAC0008093C600F6CF00E010E0EE24E394F12C62
:10BAD00080912B0A90912C0A20912D0A30912E0AE8
:10BAE000821B930B8F779927892BA9F08AEA99E01B
:10BAF0000E94AA33F092300AE0922F0A9091C0007F
:10BB000095FFFCCF8093C6000F5F1F4F1092300A45
:10BB100010922F0ADDCF03311105D4F281E090E0BD
:10BB20009093300A80932F0A8091C00085FFFCCF4C
:10BB30008AE08093C6000C94E58B88E095E00E9433
:10BB40005C368823A9F0ECE0F5E08191882339F098
:10BB50009091C00095FFFCCF8093C600F6CF8091F6
:10BB6000C00085FFFCCF8AE08093C6000C94E58B73
:10BB700087E195E00E945C368823A9F0EBE1F5E0CF
:10BB80008191882339F09091C00095FFFCCF80937C
:10BB9000C600F6CF8091C00085FFFCCF8AE080937D
:10BBA000C6000C94E58B89E395E00E945C368823FF
:10BBB00021F00F9429550C94E58B8EE395E00E94BB
:10BBC0005C36882341F060E070E088EF9FE00F94DE
:10BBD000AD540C94E58B81E495E00E945C3688239B
:10BBE00059F061E475E08AEA99E00E94903440E0FF
:10BBF00052EC61E070E010C08CE495E00E945C368D
:10BC0000882381F06CE475E08AEA99E00E94903420
:10BC100040E054E961E170E08AEA99E00E9434333F
:10BC20000C945A8D88E595E00E945C36882361F07B
:10BC30000F9442A460935D0B70935E0B80935F0B37
:10BC40009093600B0C94E58B8DE595E00E945C363B
:10BC5000882311F40C94E58B61E080E00E940B3B9B
:10BC60000C94E58B8EE50E94463681110C94E58B91
:10BC700087E40E944636882311F40C94986F0E9442
:10BC8000A6360F9497AD6C34710509F434C47CF575
:10BC90006430710509F409C154F46230710509F486
:10BCA000ECC00CF0F6C077FF78C00C94E58B6C31DB
:10BCB000710509F451C17CF46A30710509F446C17B
:10BCC0006B30710511F00C94E58B60E080E00E9410
:10BCD00013480C94E58B6E31710509F451C36B3434
:10BCE000710511F00C94E58B08E210E0FAC367359A
:10BCF000710511F40C94186F14F56035710511F489
:10BD00000C944F676CF46F34710511F00C94E58B53
:10BD10000FEF10E0AFE8CA2EADE0DA2E0C943E67CC
:10BD20006135710511F40C945F6E6635710511F083
:10BD30000C94E58B86EE0E948C3A0C94E58B6C3566
:10BD4000710511F40C94216F7CF46A35710511F4BE
:10BD50000C941D6F6B35710511F00C94E58B81E02F
:10BD60008093AD0A0C94E58B6236710511F40C9446
:10BD7000836F6336710511F00C94E58B1092851B6F
:10BD80000F942E556091851B84EC9FE00F94C8B8EA
:10BD900082E00F9417570C94E58B8091970A8111DC
:10BDA0000C94E58B0E94484460912D0B70912E0BF2
:10BDB00080912F0B9091300B0F94C8AD4B015C011B
:10BDC000C090030BD090040BE090050BF090060B95
:10BDD0004090CE0A5090CF0A6090D00A7090D10A5D
:10BDE000A3019201C701B6010F9437AC20E030E007
:10BDF00048EC52E40F9429B09B01AC01C501B40199
:10BE00000F9457AF1816E4F4A7019601C301B201CD
:10BE10000F9437AC20E030E048EC52E40F9429B0A6
:10BE20009B01AC01C501B4010F9438AC0F949CADDB
:10BE300060932D0B70932E0B80932F0B9093300BF0
:10BE40008091E00A8823A9F088E50E944636811196
:10BE500010C089E50E94463681110BC08AE50E9418
:10BE60004636811106C085E40E94463681110C9445
:10BE7000E88B0E9410470C94E58B8091970A811102
:10BE80000C94E58B0E94CB4481E00E94EE490C9417
:10BE9000E58B8091970A81110C94E58B0E94CB442D
:10BEA00080E00E94EE490C94E58B80E50E944636C6
:10BEB000882339F00E94A6360F949CAD4B015C019B
:10BEC00003C0812C912C540183E50E9446368823BF
:10BED00061F00E94A63620E030E04AE754E40F9477
:10BEE00029B00F949CAD4B015C0181149104A10415
:10BEF000B10431F0E9E0F8E2859194910F949855FE
:10BF00000F94CC250F9442A42B013C01480C591CE2
:10BF10006A1C7B1C0F9442A46093A90A7093AA0A1E
:10BF20008093AB0A9093AC0A0F9442A464157505F4
:10BF30008605970510F00C94E58B0F94513780E03F
:10BF40000E94154B80E00F941757EECF60E081E020
:10BF50000E9413480C94E58B0F94CC25EDEBFEE08A
:10BF60008491882341F09091C00095FFFCCF80938D
:10BF7000C6003196F5CF99DBEFEAFEE08491882385
:10BF800041F09091C00095FFFCCF8093C6003196A0
:10BF9000F5CFF1DB81E08093620B88E50E944636A5
:10BFA000182F89E50E944636082F8AE50E944636FA
:10BFB000782E101308C0181305C07724739401E07D
:10BFC00011E001C0012F0E9476D760907E1210927E
:10BFD0007E1282E00F943B266093FF0A7093000B61
:10BFE0008093010B9093020B71100F9458004091B5
:10BFF0000E0250910F026091100270911102409355
:10C00000AE0A5093AF0A6093B00A7093B10A809160
:10C01000490290914A0290936D0B80936C0B84E6D9
:10C0200090E090934A02809349020F9442A4609357
:10C03000A90A7093AA0A8093AB0A9093AC0A81E094
:10C040000F947B1C80E1E7EFFAE0A2ECBAE00190EC
:10C050000D928A95E1F710920E0210920F02109243
:10C06000100210921102112321F080E090E00E9452
:10C07000CD3E002321F081E090E00E94CD3E88E596
:10C080000E944636882341F00E947036672B682B49
:10C09000692B11F00C94178C89E50E944636882391
:10C0A00041F00E947036672B682B692B11F00C94BD
:10C0B0002D8C772009F4F1C08091E80A882321F0C3
:10C0C0008091E90A811108C080E090E00E94CD3E95
:10C0D00081E090E00E94CD3E0E94CBD7E2E6F3E300
:10C0E00085919591A591B49189839A83AB83BC8303
:10C0F000EEE5F3E385919591A591B4918F8F98A387
:10C10000A9A3BAA326EC3AE042EC5AE0BE016F5F65
:10C110007F4FCE014F960E94AD380E943DD720E060
:10C1200030E040E451EC6091C60A7091C70A8091FA
:10C13000C80A9091C90A0F9428AD87FF0CC080E00F
:10C1400090E0A0E4B1EC8093C60A9093C70AA09354
:10C15000C80AB093C90A80E090E0A0EAB0E48093F6
:10C16000CA0A9093CB0AA093CC0AB093CD0A20E0E0
:10C1700030E040E251E460915302709154028091AA
:10C180005502909156020F942FAD60930E0270935A
:10C190000F0280931002909311021092FF0A1092E6
:10C1A000000B1092010B1092020B80E00F947B1C8D
:10C1B000E090FF0AF090000B0091010B1091020B30
:10C1C0002091FB0A3091FC0A4091FD0A5091FE0A31
:10C1D0006091F70A7091F80A8091F90A9091FA0A31
:10C1E000F3E0CF2EFBE0DF2E0F94061980900E02B5
:10C1F00090900F02A0901002B0901102E090CA0A35
:10C20000F090CB0A0091CC0A1091CD0A2091C60A79
:10C210003091C70A4091C80A5091C90A6091C20A78
:10C220007091C30A8091C40A9091C50AE3EEFAE0C6
:10C23000FF93EF93AEECCA2EAAE0DA2E0F94580CBF
:10C240000F94CC258091C20A9091C30AA091C40A90
:10C25000B091C50A8093F70A9093F80AA093F90A5F
:10C26000B093FA0A8091C60A9091C70AA091C80AB1
:10C27000B091C90A8093FB0A9093FC0AA093FD0A2F
:10C28000B093FE0A81E00F947B1C0F94631C82E044
:10C2900090E00E94CD3E0F900F908AE50E944636B6
:10C2A000882341F00E947036672B682B692B11F0B0
:10C2B0000C94438CE090FF0AF090000B0091010B6E
:10C2C0001091020B2091FB0A3091FC0A4091FD0A6B
:10C2D0005091FE0A6091F70A7091F80A8091F90A6C
:10C2E0009091FA0AE3E0CE2EEBE0DE2E0F940619D1
:10C2F00080E00F947B1C8091AE0A9091AF0AA091D0
:10C30000B00AB091B10A80930E0290930F02A093ED
:10C310001002B093110280916C0B90916D0B909371
:10C320004A02809349020F9442A46093A90A709331
:10C33000AA0A8093AB0A9093AC0A0F94631C0E94E4
:10C34000CBD70E94E7D988E50E94463681110C942C
:10C35000598C89E50E94463681110C94598C87E5E9
:10C360000E94463681110C94598C8AE50E9446360B
:10C3700081110C94598C0F94CC251092620B8FC5AF
:10C380000F94CC2581E00E94F23580915302909168
:10C390005402A0915502B091560280930E029093E0
:10C3A0000F02A0931002B093110220E030E043E0AE
:10C3B00060E070E080E291EC0E9476DAE7E5F8E276
:10C3C00085919491FC012491222341F03091C00089
:10C3D00035FFFCCF2093C6000196F4CFE6E8FEE0DF
:10C3E0008491882341F09091C00095FFFCCF809309
:10C3F000C6003196F5CF4091F70A5091F80A609146
:10C40000F90A7091FA0A25E030E08AEA99E00E9480
:10C410009535E1E8FEE08491882341F09091C000D9
:10C4200095FFFCCF8093C6003196F5CF4091FB0A73
:10C430005091FC0A6091FD0A7091FE0A25E030E0FF
:10C440008AEA99E00E949535ECE7FEE08491882322
:10C4500041F09091C00095FFFCCF8093C6003196CB
:10C46000F5CF4091FF0A5091000B6091010B709144
:10C47000020B25E030E08AEA99E00E949535EAE770
:10C48000FEE08491882341F09091C00095FFFCCF9D
:10C490008093C6003196F5CF0E9420360C94E58B30
:10C4A0009091C00095FFFCCF8093C60081918111CF
:10C4B000F7CFB801882777FD8095982F0F94CAADE4
:10C4C0000E94F34EAB01BC0122E030E08AEA99E021
:10C4D0000E9496350F5F1F4F0F36110511F40C9413
:10C4E000E58B4AE050E0B8018AEA99E00E949D3469
:10C4F000E4E2F9E0DBCF8091E80A882341F0809103
:10C50000E90A882321F08091EA0A811109C00E947A
:10C51000ADB561E083E79EE00E94F5B40C94E58B35
:10C52000E5E5FEE08491882341F09091C00095FFFD
:10C53000FCCF8093C6003196F5CF8091C00085FF77
:10C54000FCCF8AE08093C6001A82198280906C1A10
:10C5500090906D1AA0906E1AB0906F1A20E030E0A3
:10C5600040EA50E4C501B4010F942FAD0F9497AD8C
:10C5700045E0469F9001479F300D1124B90188275F
:10C5800077FD8095982F0F94CAAD2B013C0120E0D8
:10C5900030E04CE052E40F9428AD87FF06C0412CF8
:10C5A000512C9CE0692E92E4792EA5019401C301DF
:10C5B000B2010F9428AD87FF0AC020E030E040EAC6
:10C5C00050E4C301B2010F9438AC2B013C01E1E40B
:10C5D000FEE08491882341F09091C00095FFFCCF4C
:10C5E0008093C6003196F5CF22E030E0B301A2017E
:10C5F0008AEA99E00E94963520E030E040EF51E46D
:10C60000C301B2010F9437AC20E030E040E251E4C6
:10C610000F9429B020E030E040EA50E40F942FADB1
:10C6200020E030E048E452E40F9438AC0F9497AD2A
:10C630007093791A6093781A84E090E09093260BB7
:10C640008093250B81E090E09093240B8093230B43
:10C65000EBECF6E28591949121E0892B09F420E03E
:10C660002093280B80E090E0ACE8B2E48093F70AD6
:10C670009093F80AA093F90AB093FA0A80E090E048
:10C68000A0E4B0EC8093FB0A9093FC0AA093FD0A0F
:10C69000B093FE0A80E090E0A0E8BFE38093FF0A39
:10C6A0009093000BA093010BB093020B83EE9AE0E2
:10C6B0009F938F93812C912C18E4A12E12E4B12E1C
:10C6C00003E0C02E0BE0D02EE12CF12C00E81FE39C
:10C6D00020E030E040E450EC60E070E08CE892E470
:10C6E0000F94580C0F94CC250F900F90A30192013A
:10C6F00060916C1A70916D1A80916E1A90916F1AF8
:10C700000F9428AD87FF07C088EE93E00E94364D56
:10C710000E946954EBCF60E086EA9FE00F94C8B8AE
:10C7200080E090E0A0EAB0E48093FF0A9093000BD1
:10C73000A093010BB093020B2091FB0A3091FC0AED
:10C740004091FD0A5091FE0A6091F70A7091F80A33
:10C750008091F90A9091FA0AE3EEFAE0FF93EF93E1
:10C76000812C912CE8E4AE2EE2E4BE2EF3E0CF2E35
:10C77000FBE0DF2EE12CF12C00EA10E40F94580CC2
:10C78000EEE5F3E385919591A591B4918093F70A35
:10C790009093F80AA093F90AB093FA0AE2E6F3E359
:10C7A00025913591459154912093FB0A3093FC0AD1
:10C7B0004093FD0A5093FE0AE090FF0AF090000BB0
:10C7C0000091010B1091020B6091F70A7091F80A29
:10C7D0008091F90A9091FA0AE3EEFAE0FF93EF9361
:10C7E000812C912CB8E4AB2EB2E4BB2E0F94580CE4
:10C7F0000F94CC2520E030E043E060E070E080E87A
:10C800009FEB0E9476DA8091FF0A9091000BA09135
:10C81000010BB091020B24968CAF9DAFAEAFBFAFB2
:10C820002497E0E4FEE084910F900F900F900F901A
:10C830004091FF0A5091000B6091010B7091020B27
:10C84000882349F09091C00095FFFCCF8093C600EB
:10C8500031968491F5CF8091C00085FFFCCF8AE0AE
:10C860008093C600E9E3FEE08491882341F0909133
:10C87000C00095FFFCCF8093C6003196F5CF22E033
:10C8800030E08AEA99E00E949535E8E3FEE0849181
:10C89000882341F09091C00095FFFCCF8093C600A3
:10C8A0003196F5CF8091C00085FFFCCF8AE0809360
:10C8B000C6002EEAA22E2FE0B22E33E2E32EF12C98
:10C8C0000FEF1FEF4AE0D42E51E0252E5EE0352E0B
:10C8D00060E0862E6EE0962EB701882777FD809562
:10C8E000982F0F94CAAD68AF79AF8AAF9BAFE1E3E1
:10C8F000FEE08491882341F09091C00095FFFCCF29
:10C900008093C6003196F5CF4AE050E0B8016E5FE3
:10C910007F4F8AEA99E00E949D34E4E2FEE0849130
:10C92000882341F09091C00095FFFCCF8093C60012
:10C930003196F5CF8091C00085FFFCCFD092C60024
:10C94000E0E1FEE08491882341F09091C00095FFE2
:10C95000FCCF8093C6003196F5CF4AE050E0B70196
:10C960008AEA99E00E949D34F1018491E1E0FEE0C1
:10C97000882349F09091C00095FFFCCF8093C600BA
:10C9800031968491F5CF4AE050E060E070E08AEAA9
:10C9900099E00E949D34F4018491E0E0FEE0882358
:10C9A00049F09091C00095FFFCCF8093C60031966E
:10C9B0008491F5CF8091C00085FFFCCFD092C60056
:10C9C0000F3FFFEF1F0731F0BE016F5F7F4FC501C3
:10C9D0000F94AD5428AD39AD4AAD5BADC301B20182
:10C9E0000F9428AD181664F40F5F1F4F25E0E20E78
:10C9F000F11C32E0A30EB11C0530110509F06CCF1B
:10CA0000280187E2481A88EF580A440C551C38015F
:10CA100093E0690E711C85E0809F1001819F300CAE
:10CA2000112419AE18AEADE22A0E311CC3010297D3
:10CA300005970CF0C7C168AD79AD620D731D8827ED
:10CA400077FD8095982F0F94CAAD6CAF7DAF8EAFF8
:10CA50009FAFE9EFFDE08491882341F09091C00001
:10CA600095FFFCCF8093C6003196F5CF4AE050E0A9
:10CA7000B3018AEA99E00E949D34E6EFFDE08491DB
:10CA8000882341F09091C00095FFFCCF8093C600B1
:10CA90003196F5CF8091C00085FFFCCFFAE0F0938E
:10CAA000C6007092240B6092230B20E030E040EF30
:10CAB00051E46CAD7DAD8EAD9FAD0F9437AC20E0F1
:10CAC00030E040E251E40F9429B020E030E040EA49
:10CAD00050E40F942FAD20E030E048E452E40F948E
:10CAE00038AC0F9497AD7093791A6093781A80E000
:10CAF00090E0ACE8B2E48093F70A9093F80AA09330
:10CB0000F90AB093FA0A80E090E0A0E4B0EC8093D8
:10CB1000FB0A9093FC0AA093FD0AB093FE0A80E002
:10CB200090E0A0E8BFE38093FF0A9093000BA093EE
:10CB3000010BB093020BA3EEBAE0BF93AF93812C2D
:10CB4000912CA8E4AA2EA2E4BA2EB3E0CB2EBBE02F
:10CB5000DB2EE12CF12C00E81FE320E030E040E484
:10CB600050EC60E070E08CE892E40F94580C0F9465
:10CB7000CC250F900F902CAD3DAD4EAD5FAD6091CB
:10CB80006C1A70916D1A80916E1A90916F1A0F94B1
:10CB900028AD87FF07C088EE93E00E94364D0E94C3
:10CBA0006954E9CF80E090E0A0EAB0E48093FF0A06
:10CBB0009093000BA093010BB093020B2091FB0A02
:10CBC0003091FC0A4091FD0A5091FE0A6091F70AEB
:10CBD0007091F80A8091F90A9091FA0AA3EEBAE0EE
:10CBE000BF93AF93812C912CB8E4AB2EB2E4BB2E53
:10CBF00013E0C12E1BE0D12EE12CF12C00EA10E451
:10CC00000F94580CEEE5F3E385919591A591B491BD
:10CC10008093F70A9093F80AA093F90AB093FA0A5E
:10CC2000E2E6F3E325913591459154912093FB0A77
:10CC30003093FC0A4093FD0A5093FE0AE090FF0AED
:10CC4000F090000B0091010B1091020B6091F70A1C
:10CC50007091F80A8091F90A9091FA0AA3EEBAE06D
:10CC6000BF93AF93812C912CF8E4AF2EF2E4BF2E4A
:10CC70000F94580C0F94CC2520E030E043E060E0A6
:10CC800070E080E89FEB0E9476DA24962CAD3DADF3
:10CC90004EAD5FAD24976091FF0A7091000B8091BB
:10CCA000010B9091020B0F9437AC20914D193091EC
:10CCB0004E1940914F19509150190F9429B00F946B
:10CCC00097AD7A836983E5EFFDE084910F900F9033
:10CCD0000F900F90882349F09091C00095FFFCCFF2
:10CCE0008093C60031968491F5CF8091C00085FF76
:10CCF000FCCFFAE0F093C600E1EEFDE084918823DA
:10CD000041F09091C00095FFFCCF8093C600319612
:10CD1000F5CF40916C1A50916D1A60916E1A709116
:10CD20006F1A22E030E08AEA99E00E949535E2ED40
:10CD3000FDE08491882341F09091C00095FFFCCFE5
:10CD40008093C6003196F5CF24962CAD3DAD4EAD07
:10CD50005FAD24976091FF0A7091000B8091010BE9
:10CD60009091020B0F9437ACAB01BC0122E030E094
:10CD70008AEA99E00E949535E1EDFDE084918823EF
:10CD800041F09091C00095FFFCCF8093C600319692
:10CD9000F5CF8091C00085FFFCCFFAE0F093C6008C
:10CDA000BE016F5F7F4FC2010F94AD5422E0420E6F
:10CDB000511C3FEF631A730A88AD99AD059699AF80
:10CDC00088AF34CE1092260B1092250B1092280BB0
:10CDD00061E086EA9FE00F94C8B8E2E9FDE0849143
:10CDE000882341F09091C00095FFFCCF8093C6004E
:10CDF0003196F5CF8091C00085FFFCCF8AE080930B
:10CE0000C600179A1092E80A169A1092E90A149A24
:10CE1000E9ECF6E2859194910F948C5A81E00F949D
:10CE2000845882E00F9417571092791A1092781A4A
:10CE30000C94E58B84E690E00E94364D91E0E91A6F
:10CE4000F108C1F74AE050E0B8018AEA99E00E948F
:10CE50009D34F6012491EFE8FDE0211117C06091A7
:10CE60000A0B70910B0B4AE050E08AEA99E00E94AD
:10CE7000A4340550110911F40C94E58B1093E20AC7
:10CE80000093E10AF4E6EF2EF12CD4CF3091C000EC
:10CE900035FFFCCF2093C60031962491DECF81E090
:10CEA0008093360B86E50E9446368823A1F0809158
:10CEB000451090914610DC0111962C91293069F0B3
:10CEC0002F7D71F04AE050E060E070E001960F9431
:10CED0001BB468AF07C018AE05C0B1E0B8AF02C060
:10CEE000E1E0E8AF2091E80A8091891B90918A1BCC
:10CEF000222341F02091E90A222321F02091EA0A1D
:10CF000021110FC0029749F00E94ADB561E088E899
:10CF10009DE00E94F5B40C94E58B1092360B0C94B6
:10CF2000E58B1092310A029721F41092360B0C9483
:10CF3000E58BF091280B2E96FFAF2E972091250BB5
:10CF40003091260B60963FAF2EAF60978091230BF8
:10CF50009091240B62969FAF8EAF629781E0809391
:10CF6000280B81E090E09093260B8093250B83E1C2
:10CF700090E09093240B8093230B81E00F9417573C
:10CF80008EE792E10F9425010F94580080E090E025
:10CF9000A0EAB0E48093FF0A9093000BA093010BEA
:10CFA000B093020B20E030E040E752E4609153027E
:10CFB0007091540280915502909156020F942FADBA
:10CFC0004B015C012091FB0A3091FC0A4091FD0A63
:10CFD0005091FE0A6091F70A7091F80A8091F90A5F
:10CFE0009091FA0AE3EEFAE0FF93EF9313E0C12E7B
:10CFF0001BE0D12EE12CF12C00EA10E40F94580C28
:10D00000EEE5F3E385919591A591B4918093F70AAC
:10D010009093F80AA093F90AB093FA0AE2E6F3E3D0
:10D0200085919591A591B4918093FB0A9093FC0A08
:10D03000A093FD0AB093FE0A6BEF7AE087EF9AE0C7
:10D040000E94673929968FAF29970F900F9098AD5E
:10D0500019160CF45FC020E030E040EF51E460911D
:10D060004B0270914C0280914D0290914E020F94B0
:10D070002FAD4B015C01E090FF0AF090000B009196
:10D08000010B1091020B2091FB0A3091FC0A409198
:10D09000FD0A5091FE0A6091F70A7091F80A80919A
:10D0A000F90A9091FA0AE3EEFAE0FF93EF93B3E006
:10D0B000CB2EBBE0DB2E0F94580C0F94CC2520E038
:10D0C00030E040EA51E460914B0270914C02809153
:10D0D0004D0290914E020F942FAD0F9497AD8B019E
:10D0E00020E030E040E252E460915302709154023B
:10D0F00080915502909156020F942FAD0F9497ADE9
:10D100007B010E9429D78CAF0F900F90A8AD1A1603
:10D1100014F129C02996BFAD2997BB2371F0E6E62B
:10D12000FDE08491882309F496CF9091C00095FF8B
:10D13000FCCF8093C6003196F4CFECE3FDE0849100
:10D14000882309F488CF9091C00095FFFCCF80938D
:10D15000C6003196F4CF9CAD992379F1EAE1FDE068
:10D160008491811122C080E00E94F235EEE5F3E364
:10D170002696FFAFEEAF2697212C312CC701AA27A8
:10D1800097FDA095BA2F66968CAF9DAFAEAFBFAF9F
:10D190006697C801AA2797FDA095BA2F6A968CAF0B
:10D1A0009DAFAEAFBFAF6A9715C09091C00095FF1D
:10D1B000FCCF8093C6003196D3CFE4EFFCE084919E
:10D1C000882389F29091C00095FFFCCF8093C60020
:10D1D0003196F5CFA8AD1A16A4F4E3EFFCE08491E4
:10D1E000882341F09091C00095FFFCCF8093C6004A
:10D1F0003196F5CF8091C00085FFFCCF8AE0809307
:10D20000C600C10163E070E00F9407B228967FAFBB
:10D210006EAF289722969FAF8EAF22972796FFADCD
:10D220002797F0FF08C022E030E0281B390B229638
:10D230003FAF2EAF22973CAD332309F477C02114C2
:10D24000310409F473C028968EAD9FAD2897880FDE
:10D25000991F2896AEADBFAD28978A0F9B1F2296C7
:10D26000EEADFFAD22978E0F9F1F880F991F8D5334
:10D27000904F0F94C3B8BC01882777FD8095982FF5
:10D280000F94CAAD2AE037ED43E25CE30F9429B076
:10D2900020917F1230918012409181125091821220
:10D2A0000F9438AC2B013C01F8AD1F160CF041C0B7
:10D2B000EDEDFCE08491882341F09091C00095FF52
:10D2C000FCCF8093C6003196F5CF4AE050E0B10123
:10D2D0008AEA99E00E949D34EBECFCE0849188237B
:10D2E00041F09091C00095FFFCCF8093C60031962D
:10D2F000F5CF25E030E0B301A2018AEA99E00E946F
:10D300009535EAECFCE08491882341F09091C000CF
:10D3100095FFFCCF8093C6003196F5CF8091C00079
:10D3200085FFFCCF8AE08093C60003C0412C512CBE
:10D33000320180E090E0A0EAB0E48093FF0A90938D
:10D34000000BA093010BB093020B66966CAD7DAD04
:10D350008EAD9FAD66970F94CAAD2D966CAF7DAF25
:10D360008EAF9FAF2D972091FB0A3091FC0A409120
:10D37000FD0A5091FE0A6091F70A7091F80A8091B7
:10D38000F90A9091FA0AA3EEBAE0BF93AF932D96F3
:10D390008CAC9DACAEACBFAC2D97B3E0CB2EBBE05C
:10D3A000DB2EE12CF12C00EA10E40F94580C0F94C2
:10D3B000CC252696EEADFFAD269785919591A5914A
:10D3C000B4918093F70A9093F80AA093F90AB09366
:10D3D000FA0A2696EEADFFAD269734968591959183
:10D3E000A591B4918093FB0A9093FC0AA093FD0A47
:10D3F000B093FE0A6BEF7AE087EF9AE00E946739FC
:10D400000F900F90F8AD1F16A4F16A966CAD7DAD2C
:10D410008EAD9FAD6A970F94CAAD4B015C01E09051
:10D42000FF0AF090000B0091010B1091020B20916C
:10D43000FB0A3091FC0A4091FD0A5091FE0A60916E
:10D44000F70A7091F80A8091F90A9091FA0AA3EE0E
:10D45000BAE0BF93AF93A3E0CA2EABE0DA2E0F94ED
:10D46000580C0F94CC250F900F90FCADF11129C0F2
:10D4700034C04AE050E0B1018AEA99E00E949D344C
:10D4800029962FAD2997222371F0EBEBFCE08491D4
:10D49000882309F4BACF9091C00095FFFCCF809308
:10D4A000C6003196F4CFE9EAFCE08491882309F4C0
:10D4B000ACCF9091C00095FFFCCF8093C600319611
:10D4C000F4CF2114310449F020E030E040E85FE37C
:10D4D000C301B2010F9437AC04C060E070E080E299
:10D4E00091EC20E030E043E00E9476DA811103C045
:10D4F000E3E4F8E21AC08090FF0A9090000BA0903D
:10D50000010BB090020BA501940160E070E080EA8D
:10D5100090E40F9437AC2DEC3CEC4CEC5DE30F94B5
:10D5200028AD87FF05C0E1E4F8E26590749004C17E
:10D53000FCADFF2391F0A5019401C301B2010F944A
:10D5400037AC9F7720E030E040E85FE30F9457AFBF
:10D5500018161CF4E5E4F8E2E8CF28AD2A305CF4B4
:10D560000E94DA524B015C0138AD13160CF09CC0DE
:10D57000EAE8FCE05FC0E5EAFCE08491882341F042
:10D580009091C00095FFFCCF8093C6003196F5CFF7
:10D590004091F70A5091F80A6091F90A7091FA0ADD
:10D5A00025E030E08AEA99E00E949535E4EAFCE063
:10D5B0008491882341F09091C00095FFFCCF809327
:10D5C000C6003196F5CF8091C00085FFFCCF8AE080
:10D5D0008093C600E0EAFCE08491882341F09091BA
:10D5E000C00095FFFCCF8093C6003196F5CF4091E7
:10D5F000FB0A5091FC0A6091FD0A7091FE0A25E039
:10D6000030E08AEA99E00E949535EEE9FCE08491E9
:10D61000882309F4A5CF9091C00095FFFCCF80939B
:10D62000C6003196F4CF9091C00095FFFCCF809357
:10D63000C600319684918111F6CF4091FF0A509136
:10D64000000B6091010B7091020B25E030E08AEA3B
:10D6500099E00E949535E0E8FCE08491882341F050
:10D660009091C00095FFFCCF8093C6003196F5CF16
:10D6700025E030E0B501A4018AEA99E00E949535E1
:10D68000EFE7FCE08491882341F09091C00095FF82
:10D69000FCCF8093C6003196F5CF8091C00085FF06
:10D6A000FCCF8AE08093C60087E02896AEADBFAD80
:10D6B00028978A9F80018B9F100D11242296EEAD32
:10D6C000FFAD22970E0F1F1F000F111F000F111F1C
:10D6D00002581D4EA50194016091FF0A7091000B44
:10D6E0008091010B9091020B0F9437ACD8011196E9
:10D6F0006D937D938D939C9314978091230B9091C0
:10D70000240B01979093240B8093230BBFEF2B1ACC
:10D710003B0A81E00F9417572696EEADFFAD269792
:10D7200038962696FFAFEEAF2697F9E02F16310414
:10D7300009F050CD612C712C28AD2431A4F0E8E51E
:10D74000FCE08491882341F09091C00095FFFCCFCC
:10D750008093C6003196F5CF8091C00085FFFCCF45
:10D760008AE08093C60080E090E0A0EAB0E4809375
:10D77000FF0A9093000BA093010BB093020B38ADFE
:10D78000343114F1E3E4FCE08491882341F090917A
:10D79000C00095FFFCCF8093C6003196F5CF8091F5
:10D7A000C00085FFFCCF8AE08093C6004091FF0A4D
:10D7B0005091000B6091010B7091020B25E030E05D
:10D7C0008AEA99E00E949535E090FF0AF090000BFC
:10D7D0000091010B1091020B2091FB0A3091FC0A81
:10D7E0004091FD0A5091FE0A6091F70A7091F80A83
:10D7F0008091F90A9091FA0AE3EEFAE0FF93EF9331
:10D800002D968CAC9DACAEACBFAC2D97E3E0CE2E8C
:10D81000EBE0DE2E0F94580C0F94CC250F900F9058
:10D8200089E02816310421F060E0C3010C949D7654
:10D830000E942036E0E3FCE08491882341F090913F
:10D84000C00095FFFCCF8093C6003196F5CF809144
:10D85000C00085FFFCCF8AE08093C6000F94400093
:10D86000EFE1FCE08491882341F09091C00095FFA6
:10D87000FCCF8093C6003196F5CF8091C00085FF24
:10D88000FCCF8AE08093C60080EC9FE00F94B6B88E
:10D89000EE24E394813009F0E12C98AD19164CF098
:10D8A000DE0111966D01F12C2CE4622E36E4732E0C
:10D8B0001CC0EE2069F0E4E0FCE08491882381F351
:10D8C0009091C00095FFFCCF8093C6003196F5CFB4
:10D8D000E5EEFBE08491882319F39091C00095FF59
:10D8E000FCCF8093C6003196F5CF6982B2E5BA834A
:10D8F0007B8282E48C83F60181916F010E9446361F
:10D90000882319F00E9470361EC0EE2009F436C13B
:10D91000F1E0FF1528F0F11009C08FEB9FE00BC07C
:10D9200022E0F21206C08DEB9FE005C08EEB9FE077
:10D9300002C08CEB9FE00F94B6B8682F772767FD85
:10D940007095872F972F611571058105910509F451
:10D9500015C10F94CAAD2FE632E143E85AE30F94A4
:10D9600029B04B015C019F7727E139ED4EEC5DE377
:10D970000F9457AF18160CF037C0E6E4F0E184912D
:10D98000882341F09091C00095FFFCCF8093C600A2
:10D990003196F5CFE1ECFBE08491882341F0909142
:10D9A000C00095FFFCCF8093C6003196F5CF22E0F2
:10D9B00030E0B501A4018AEA99E00E949535E8EBD0
:10D9C000FBE08491882341F09091C00095FFFCCF4B
:10D9D0008093C6003196F5CF8091C00085FFFCCFC3
:10D9E0008AE08093C600CAC0F2E0FF1609F469C05D
:10D9F00023E0F21609F494C031E0F31689F120E037
:10DA000030E040E05FE3C501B4010F9429B01B0191
:10DA10002C010FE712E1A2019101D80114966D913A
:10DA20007D918D919C9117970F9438ACF801648388
:10DA3000758386839783A5019401608171818281BA
:10DA400093810F9438ACD8016D937D938D939C9303
:10DA50001397045E1F4FB2E1033D1B07E1F68EC032
:10DA600020E030E040E05FE3C501B4010F9429B04D
:10DA70001B012C0103E812E1A2019101F801608170
:10DA80007181828193810F9438ACD8016D937D931D
:10DA90008D939C931397A501940114966D917D919C
:10DAA0008D919C9117970F9438ACF801648375831E
:10DAB00086839783045E1F4FF2E1073D1F07E1F65F
:10DAC0005DC020E030E040E05FE3C501B4010F94A9
:10DAD00029B01B012C010FE712E1A2019101D8012D
:10DAE0005C966D917D918D919C915F970F9438AC70
:10DAF000F801648F758F868F978FA50194016081DF
:10DB00007181828193810F9438ACD8016D937D939C
:10DB10008D939D938D01B2E10B381B07F1F62EC05A
:10DB200020E030E040E05FE3C501B4010F9429B08C
:10DB30001B012C010BE912E1A2019101F8016081A6
:10DB40007181828193810F9438ACD8016D937D935C
:10DB50008D939D938D01A501940158966D917D91B2
:10DB60008D919C915B970F9438ACF801608F718F09
:10DB7000828F938FF2E1073A1F07F1F6F39424E0C6
:10DB8000F212B3CEE7E9FBE08491882341F0909153
:10DB9000C00095FFFCCF8093C6003196F5CF8091F1
:10DBA000C00085FFFCCF8AE08093C6008EE792E13B
:10DBB0000F944001E5E8FBE08491882341F09091C7
:10DBC000C00095FFFCCF8093C6003196F5CF8091C1
:10DBD000C00085FFFCCF8AE08093C60081E080937F
:10DBE0007E12E9E6FBE08491882341F09091C00029
:10DBF00095FFFCCF8093C6003196F5CF8091C00091
:10DC000085FFFCCF8AE08093C6000E942DF6E8E5F0
:10DC1000FBE08491882341F09091C00095FFFCCFF8
:10DC20008093C6003196F5CF8091C00085FFFCCF70
:10DC30008AE08093C600E091E30A34E0E39FF001BC
:10DC40001124EE58F54E20E030E042E053E46081CC
:10DC50007181828193810F9457AF181694F480914B
:10DC6000610B882371F086EA9FE00F94B6B8882391
:10DC700041F08091781A9091791AC29714F00C941F
:10DC8000BB8C2E968FAD2E978093280B6096AEADF1
:10DC9000BFAD6097B093260BA093250B6296EEADB7
:10DCA000FFAD6297F093240BE093230B1092360B99
:10DCB0001092350B82E00F9417570C94E58B8091EE
:10DCC0007E12882309F49EC0EEE4FBE08491882351
:10DCD00041F09091C00095FFFCCF8093C600319633
:10DCE000F5CF4AE050E067E070E08AEA99E00E94F0
:10DCF0009D34ECE4FBE08491882341F09091C000D6
:10DD000095FFFCCF8093C6003196F5CF4AE050E0F6
:10DD100067E070E08AEA99E00E949D34E9E3FBE065
:10DD20008491882341F09091C00095FFFCCF8093AF
:10DD3000C6003196F5CF4AE050E065E070E08AEA2F
:10DD400099E00E949D34E7E2FBE08491882341F052
:10DD50009091C00095FFFCCF8093C6003196F5CF1F
:10DD60008091C00085FFFCCF8AE08093C60000E070
:10DD700010E084E2A82E8BE0B82E92E2892E9BE080
:10DD8000992EE12CF12C98012A5D3C4E6901F50198
:10DD90008491E4E2FBE0882349F09091C00095FF74
:10DDA000FCCF8093C60031968491F5CFF601EE0D3D
:10DDB000FF1D418152816381748125E030E08AEA50
:10DDC00099E00E949535F4E0EF0EF11C2CE1E2168B
:10DDD000F104E9F6F4018491E2E2FBE0882349F0E2
:10DDE0009091C00095FFFCCF8093C600319684913E
:10DDF000F5CF0C5111090C33FFEF1F0709F0C1CF0C
:10DE00000C94E58BE4E0FBE08491882341F0909151
:10DE1000C00095FFFCCF8093C6003196F5CF80916E
:10DE2000C00085FFFCCF8AE08093C6000C94E58B90
:10DE300081E00E948C3A0C94E58B1092AD0A0C9410
:10DE4000E58B85E40E944636811102C00F94CC25F3
:10DE5000B0EC6B2EB6E07B2E1BEE812E1AE0912EDD
:10DE600007EFA02E0AE0B02E512CD3018D913D0179
:10DE70000E9446368823D9F1B3E05B120CC00E94A1
:10DE8000A636F501608371838283938383E09BE0F0
:10DE90000F94A51A2CC00E94A636D4012D913D9155
:10DEA0004D915C910F9438ACF5016083718382834E
:10DEB0009383E090FF0AF090000B0091010B10910A
:10DEC000020B2091FB0A3091FC0A4091FD0A50910F
:10DED000FE0A6091F70A7091F80A8091F90A909110
:10DEE000FA0AA3E0CA2EABE0DA2E0F940619539477
:10DEF000F4E08F0E911C24E0A20EB11C34E053120A
:10DF0000B4CF0C94E58B81E08093851B0F9442A4E1
:10DF10006093720B7093730B8093740B9093750BDB
:10DF20006091851B84EC9FE00F94C8B80C94E58B3E
:10DF30008DE40E944636882311F40C94D689E09132
:10DF40004510F0914610319681918032E9F3893085
:10DF5000D9F380538A30B0F0E5EFFAE0849188235A
:10DF600041F09091C00095FFFCCF8093C6003196A0
:10DF7000F5CF8091C00085FFFCCF8AE08093C6007A
:10DF80000C94E58B0E94A6360F9497AD6B3C7105FF
:10DF900011F40C94F37D0CF021C16F32710509F47A
:10DFA000AAC60CF06AC06931710509F451C3B4F511
:10DFB0006431710509F4F1C294F46131710509F419
:10DFC000E0C234F46230710508F434C20C94C189A3
:10DFD0006231710511F40C94EA790C94C1896631AF
:10DFE000710509F414C30CF40CC36731710509F40D
:10DFF00014C36831710511F00C94C18986E79BE068
:10E000000E9431A90F9442A46093A10A7093A20ABE
:10E010008093A30A9093A40A0C94E58B6E3171054A
:10E0200009F45FC38CF46B31710509F425C30CF45A
:10E0300015C36C31710509F425C36D31710511F4F7
:10E040000C94E58B0C94C1896A32710509F477C48C
:10E0500054F46F31710509F412C46032710509F48A
:10E0600078C30C94C1896C32710509F4AFC46D3268
:10E07000710509F4BAC40C94C1896D36710509F4AF
:10E08000B2C70CF064C06535710511F40C94237AA5
:10E090000CF03DC06235710511F40C94E1795CF52A
:10E0A0006135710511F00C94C1890F94EB2F0F9419
:10E0B000CC25149A0F944E261092E20A1092E10A8F
:10E0C00068EE73E080E090E00F9471A41092120269
:10E0D000E5E7F7E24591549120EB3AE06EEA7AE009
:10E0E00080E695E00E946EBB0F94985580E00F94F7
:10E0F00017570C94E58B6335710511F40C94E57991
:10E100006435710511F40C94EA790C94C18969366F
:10E11000710509F425C65CF46C35710511F40C9495
:10E120003E7A6836710509F4EAC50C94C1896A36ED
:10E13000710511F40C94B1796B36710511F00C94E2
:10E14000C1891092E20A1092E10A0C94E58B6837BB
:10E15000710511F40C94E57BFCF46237710511F440
:10E160000C94017B4CF46037710511F00C94C1895B
:10E1700063E083EB98E0E1C56337710511F40C941B
:10E18000C17A6737710511F00C94C189E1EAF7E2B1
:10E19000859194910C94F67B6E3B710509F4B9C797
:10E1A0005CF46937710511F40C94EA7B6C387105E5
:10E1B00009F4C5C50C94C189683C710511F40C942F
:10E1C000617D693C710511F00C94C18900EC16E089
:10E1D00065E3E62E69E1F62E0C94D87D673F81E079
:10E1E000780711F40C941E820CF07EC06C32A1E012
:10E1F0007A0711F40C942380C4F5603D710511F485
:10E200000C94FD7EA4F46D3C710511F40C94327EE7
:10E2100014F40C94107E6E3C710511F40C94A97EDC
:10E220006F3C710511F40C94C67E0C94C1896D3D50
:10E23000710511F40C94977F64F4613D710511F43C
:10E240000C94257F6C3D710511F40C94867F0C9421
:10E25000C189623E710511F40C94C17F603F710564
:10E2600011F40C94E58B0C94C1896036E1E07E07D3
:10E27000E4F46E35F1E07F0714F00C94E58B6E3218
:10E2800021E0720711F40C94C88114F40C945B80A3
:10E290006F3281E0780711F40C94D78160337140BC
:10E2A00011F40C9426810C94C189643FA1E07A0793
:10E2B00011F40C9410824CF46039714011F00C94FC
:10E2C000C1890F94CC250C94E58B653FF1E07F0765
:10E2D00011F40C941782663F714011F00C94C189BF
:10E2E0000E949A2A0C94E58B6E3833E0730711F480
:10E2F0000C9402870CF047C06D3B92E0790711F453
:10E300000C945388FCF46835B2E07B0711F40C944C
:10E3100032835CF46D3F714011F00C94C1890F940D
:10E320002955E0E4F0E10C942A82693522E0720775
:10E3300011F40C94BD866A35724011F40C94CB86AE
:10E340000C94C189643883E0780711F40C94D98661
:10E350006CF46E3BA2E07A0711F40C946389633588
:10E36000734011F40C943C820C94C1896B38E3E047
:10E370007E0711F40C94DC866C38734011F40C9415
:10E38000E58B0C94C189633923E0720711F40C9476
:10E390006C87D4F4603983E0780711F40C943787E4
:10E3A00014F40C9405876139A3E07A0711F40C94F6
:10E3B00069876239734011F00C94C1891092E51A93
:10E3C0000F94CE420C94E58B6639E3E07E0711F49E
:10E3D0000C9421886CF4643923E0720711F40C94D6
:10E3E00072876539734011F40C94EF870C94C189DE
:10E3F000603A83E0780709F415C2673E734011F074
:10E400000C94C1891092970A0F94C45580913110D1
:10E4100090913210A0913310B09134108093351048
:10E4200090933610A0933710B09338100E941A447E
:10E430000C94E58B00914510109146100E5F1F4F14
:10E4400080E50E944636882379F00E94A6360F9414
:10E450009CAD4B015C01FF24F394611571058105AE
:10E46000910531F4F12C04C0F12C812C912C540134
:10E4700083E50E944636882399F00E94A63620E064
:10E4800030E04AE754E40F9429B00F949CAD4B015F
:10E490005C01EE24E394611571058105910509F491
:10E4A000E12C6AE270E0C8010F940AB6009711F0FF
:10E4B000DC011C92F801CF0121912032E1F3F1102F
:10E4C00007C0E11005C0222319F00F948B5506C038
:10E4D000E5EBF6E2859194910F94985581E00F94C5
:10E4E0006B550F94CC250F9442A46093A90A7093A6
:10E4F000AA0A8093AB0A9093AC0A81149104A104F8
:10E50000B104A9F00F9442A42B013C01480C591C02
:10E510006A1C7B1C0F9442A464157505860597053B
:10E52000C8F40F949F59811115C00C94FD8C0F9461
:10E530009D59882311F40C94E58B0F949F598111F8
:10E540000CC00F94513781E00E94154B80E00F946E
:10E550001757F3CF80E00F946B558091780B882389
:10E5600041F0E3E4F7E2859194910F9498550C946F
:10E57000E58BEDE9F6E2859194910F9498550C9412
:10E58000E58BE7E7F7E2859194910F9498551798FA
:10E590001698159814980C94E58BEDE2F8E28591A5
:10E5A0009491FC012491222341F03091C00035FF69
:10E5B000FCCF2093C6000196F4CF8091C00085FF68
:10E5C000FCCF8AE08093C60086E79BE00E9402A809
:10E5D000E1E0F8E285919491FC012491222341F03D
:10E5E0003091C00035FFFCCF2093C6000196F4CFD8
:10E5F0008091C00085FFFCCF8AE08093C6000C9418
:10E60000E58B86E79BE00E9458A80C94E58B86E793
:10E610009BE00E942DA90C94E58B80914510909170
:10E6200046106AE270E004960F940AB6009711F063
:10E63000DC011C9260914510709146106C5F7F4F19
:10E6400021E041E086E79BE00E94D9AD0C94E58B88
:10E6500086E79BE00E9438A90C94E58B8091790BAA
:10E66000882311F40C94E58B83E50E9446368111D2
:10E670000C94078D0C94E58B86E79BE00E94DDAA45
:10E680000C94E58B80914510909146106AE270E001
:10E6900004960F940AB68C010097A9F080914F1050
:10E6A000909150106EE470E08C5A9F4E0F940AB611
:10E6B00060E270E00F940AB6019690934610809342
:10E6C0004510F801108260914510709146106C5F02
:10E6D0007F4F21E040E086E79BE00E94D9AD0C949B
:10E6E000E58B8091790B882311F40C94E58B60E025
:10E6F00086E79BE00E9469AD80914510909146109D
:10E700006AE270E004960F940AB68C010097A9F0B3
:10E7100080914F10909150106EE470E08C5A9F4E93
:10E720000F940AB660E270E00F940AB601969093D7
:10E73000461080934510D8011C926091451070914D
:10E7400046106C5F7F4F86E79BE00E949CA90C946B
:10E75000E58B8091780B81110F94CC2500914510A9
:10E76000109146100C5F1F4F6AE270E0C8010F94D1
:10E770000AB67C0161E270E0C8010F940AB6009706
:10E7800019F08C010F5F1F4FE114F10411F0F70134
:10E79000108280E50E944636F82E20914510309177
:10E7A00046100217130708F4F12C8091790B882387
:10E7B00011F40C94E58B21E02F2541E0B80186E7A8
:10E7C0009BE00E94D9AD83E50E9446368823B9F0CC
:10E7D00020914510309146102017310780F40E9497
:10E7E0007036AB01BC014093140E5093150E60932C
:10E7F000160E7093170E8FE59DE00E948B9B86E7A7
:10E800009BE00E9431A9F1100C94E58B0F9442A477
:10E810006093A10A7093A20A8093A30A9093A40A1A
:10E820000C94E58B80914510909146106AE270E05F
:10E8300005960F940AB68C010097A9F080914F10AD
:10E84000909150106EE470E08C5A9F4E0F940AB66F
:10E8500060E270E00F940AB60196909346108093A0
:10E860004510D8011C9260914510709146106B5F65
:10E870007F4F86E79BE00E9417B10C94E58B0F94C5
:10E8800042A460939D0A70939E0A80939F0A90937E
:10E89000A00A0091A10A1091A20A2091A30A309126
:10E8A000A40A601B710B820B930B28EE33E040E04F
:10E8B00050E00F941AB2CA01B9012CE330E040E0F5
:10E8C00050E00F941AB27F936F933F932F9386EE8D
:10E8D0009AE09F938F93CE0101969F938F930F940D
:10E8E0008AB6E0E4F0E184910FB6F894DEBF0FBE83
:10E8F000CDBFE0E4F0E1882349F09091C00095FF9E
:10E90000FCCF8093C60031968491F5CFFE013196FD
:10E910008191882339F09091C00095FFFCCF8093BE
:10E92000C600F6CF8091C00085FFFCCF8AE08093BF
:10E93000C600CE0101960F948B550C94E58B83E5B0
:10E940000E944636882311F40C94E58B0E94A6366B
:10E950000F9497ADF62EE72E862F9E2D8C0180E525
:10E960000E944636882331F00F3F110509F010F45C
:10E970000C94188D0DE010E0E8E8F6E0819191919B
:10E980008017910711F40C94E58B26E0E03CF20728
:10E99000A9F70630110539F48F2D9E2D9093E20AC8
:10E9A0008093E10A04C017FF02C00C94E58B61E07C
:10E9B000802F0F942DA66F2D802F0F9466A66F2D9C
:10E9C0007E2D802F0F9415A50C94E58B8FEF0E9460
:10E9D0008C3A60E070E088EF9FE00F94E2B80E940C
:10E9E000E3D60E9476D70C94E58B8AE50E944636E2
:10E9F000382E811112C01092791A1092781A109242
:10EA00007B1A10927A1A10927D1A10927C1A109228
:10EA10007F1A10927E1A0F94D45480E00F94845879
:10EA20008EE792E10F9425010E9476D70F94730030
:10EA30001092E80A1092E90A1092EA0A81E00E9414
:10EA4000F235EFE5F8E2859194910E947E3A0E94BA
:10EA5000EF420E94773D882309F448C10E94224377
:10EA600020E030E048E452E46091721A7091731A29
:10EA70008091741A9091751A0F9457AF181684F0FC
:10EA800020E030E048E452E46091601A7091611A2D
:10EA90008091621A9091631A0F9457AF181624F45C
:10EAA000332011F40C941F8D80E090E0A0EAB0E4D4
:10EAB0008093FF0A9093000BA093010BB093020B7D
:10EAC00020E030E040E252E4609153027091540241
:10EAD00080915502909156020F942FAD4B015C012D
:10EAE0002091FB0A3091FC0A4091FD0A5091FE0AE8
:10EAF0006091F70A7091F80A8091F90A9091FA0AE8
:10EB0000E3EEFAE0FF93EF93E3E0CE2EEBE0DE2EB0
:10EB1000E12CF12C00EA10E40F94580C0F94CC2552
:10EB200086E50E9446360F900F908823A1F08091D1
:10EB3000451090914610DC0111962C91293069F016
:10EB40002F7D71F04AE050E060E070E001960F9494
:10EB50001BB468AF07C018AE05C0B1E0B8AF02C0C3
:10EB6000E1E0E8AF3320B1F00E9420360E94CBD71D
:10EB70000E94E7D90E9493F6882309F4B5C087EF75
:10EB80009FE00F94B6B8803F09F0AEC081E00E94CC
:10EB90008C3AAAC08FEF0E948C3A60E070E088EF58
:10EBA0009FE00F94E2B81982BE016F5F7F4F88AD7E
:10EBB0000E94EAEE3C010E942036212C312C10EA02
:10EBC000412E10E4512E2092FF0A3092000B409209
:10EBD000010B5092020B20E030E040E252E46091E1
:10EBE00053027091540280915502909156020F94F5
:10EBF0002FAD4B015C012091FB0A3091FC0A409142
:10EC0000FD0A5091FE0A6091F70A7091F80A80910E
:10EC1000F90A9091FA0AA3EEBAE0BF93AF9303E02A
:10EC2000C02E0BE0D02E820171010F94580C0F946E
:10EC3000CC250F900F9077FC48C019828EE792E1A7
:10EC40000F9425010E943DD781E00E94F2350E9479
:10EC5000EF42AE014F5F5F4F68AD81E00E94ABF8BD
:10EC60003C010E9420362092FF0A3092000B409215
:10EC7000010B5092020B20E030E040E252E4609140
:10EC800053027091540280915502909156020F9454
:10EC90002FAD4B015C012091FB0A3091FC0A4091A1
:10ECA000FD0A5091FE0A6091F70A7091F80A80916E
:10ECB000F90A9091FA0AA3EEBAE0BF93AF930F94CA
:10ECC000580C0F94CC250F900F906981C3010F94BD
:10ECD000C55A77FC09C086EE0E948C3AE9E5F8E255
:10ECE000859194910F948C5A0F94CD4181E00F94AB
:10ECF00084580C94E58B0F94C16D0C94E58B88E6D9
:10ED000090E00E94CF4B81110C94E58B83E50E942B
:10ED10004636882371F00091980A0E94A63610E0CA
:10ED2000000F111F0658154E0F9497ADD8016D9323
:10ED30007C930F94EA2F0C94E58B0E94A04A83E504
:10ED40000E944636882311F40C94E58B0E94A63667
:10ED50000F9497AD7093791A6093781A0C94E58BA1
:10ED600089E690E00E94CF4B81110C94E58BE0EE98
:10ED7000FAE08491882341F09091C00095FFFCCF88
:10ED80008093C6003196F5CFE091980AB4E0EB9FEE
:10ED9000F0011124EE58F54E40815181628173815A
:10EDA00021E030E08AEA99E00E949535EDEDFAE045
:10EDB0008491882341F09091C00095FFFCCF80930F
:10EDC000C6003196F5CFE091980AF0E0EE0FFF1FF4
:10EDD000E658F54E60817181882777FD8095982FE0
:10EDE0000F94CAADAB01BC0121E030E08AEA99E0A2
:10EDF0000E949535E9EDFAE08491882341F09091E5
:10EE0000C00095FFFCCF8093C6003196F5CF4091AE
:10EE1000601A5091611A6091621A7091631A21E030
:10EE200030E08AEA99E00E949535E6EDFAE08491B7
:10EE3000882341F09091C00095FFFCCF8093C600DD
:10EE40003196F5CF6091781A7091791A882777FDFD
:10EE50008095982F0F94CAADAB01BC0121E030E042
:10EE60008AEA99E00E949535E3EDFAE084918823DF
:10EE700041F09091C00095FFFCCF8093C600319681
:10EE8000F5CF4AE050E060E070E08AEA99E00E9445
:10EE90009D34E1EDFAE08491882341F09091C00027
:10EEA00095FFFCCF8093C6003196F5CF4091721A42
:10EEB0005091731A6091741A7091751A21E030E0C4
:10EEC0008AEA99E00E949535EEECFAE08491882375
:10EED00041F09091C00095FFFCCF8093C600319621
:10EEE000F5CF60917A1A70917B1A882777FD80950B
:10EEF000982F0F94CAADAB01BC0121E030E08AEA43
:10EF000099E00E949535EAECFAE08491882341F07B
:10EF10009091C00095FFFCCF8093C6003196F5CF4D
:10EF20008091980A90E00F946B2D4AE050E0BC016C
:10EF30008AEA99E00E949D34E5ECFAE08491882306
:10EF400041F09091C00095FFFCCF8093C6003196B0
:10EF5000F5CF8FEF9FEF0F946B2D4AE050E0BC018F
:10EF60008AEA99E00E949D34E1ECFAE084918823DA
:10EF700041F09091C00095FFFCCF8093C600319680
:10EF8000F5CF40916C1A50916D1A60916E1A709184
:10EF90006F1A21E030E08AEA99E00E949535EDEBA6
:10EFA000FAE08491882341F09091C00095FFFCCF56
:10EFB0008093C6003196F5CF4091661A5091671A3A
:10EFC0006091681A7091691A21E030E08AEA99E04C
:10EFD0000E9495358091C00085FFFCCF8AE0809328
:10EFE000C6000C945A8D8DE690E00E94CF4B8111A3
:10EFF0000C94E58BEDECF7E2859194910F94985584
:10F0000081E090E090932C0B80932B0B8091851BDB
:10F01000882321F081E090E00F94065583E50E945B
:10F020004636882391F00091980A0E94A63610E097
:10F03000000F111F0658154E0F9497ADF8017183FC
:10F04000608381E08093080215C082E50E94463605
:10F05000882381F00091980A0E94A63610E0000FE4
:10F06000111F0658154E0F9497ADD8016D937C93E0
:10F07000109208020F94EA2F0F9442A46B017C01B6
:10F080000091980A10E0F801EE0FFF1FE658F54EC8
:10F0900060817181882777FD8095982F0F94CAAD84
:10F0A000F801EE0FFF1FEE0FFF1FEE58F54E11E0B7
:10F0B00020813181428153810F9457AF18160CF093
:10F0C00010E01093960A1092D20AC701B6010E946E
:10F0D000584DEBECF7E2859194910F94985582E0AE
:10F0E00090E090932C0B80932B0B8091851B8823B1
:10F0F00021F082E090E00F9406550F9442A46093B3
:10F10000A90A7093AA0A8093AB0A9093AC0A0C9454
:10F11000E58BE7E4F8E2859194910F94985583E0AC
:10F1200090E090932C0B80932B0B8091851B882370
:10F1300021F081E090E00F94065583E50E94463669
:10F14000882361F00E94A6360F9497AD7093791AC8
:10F150006093781A81E0809308020FC082E50E94D4
:10F160004636882351F00E94A6360F9497AD7093CF
:10F17000791A6093781A109208020F9442A42B0116
:10F180003C011092D20A6091781A7091791A8827FE
:10F1900077FD8095982F0F94CAAD11E02091601AE9
:10F1A0003091611A4091621A5091631A0F9457AFCF
:10F1B00018160CF010E01093960A0AEB1AE096EB82
:10F1C000E92E9AE0F92E22EBA22E2AE0B22E3AE0A6
:10F1D000D32E8091960A6091781A7091791A8823BB
:10F1E00009F490C08091D20A81118CC0882777FDE4
:10F1F0008095982F0F94CAAD2091601A3091611AB2
:10F200004091621A5091631A0F9457AF18160CF080
:10F2100090C00F9442A46419750986099709693E44
:10F2200073408105910508F464C08091851B8111AC
:10F230005CC0E091E30A24E0E29FF0011124EE5863
:10F24000F54E4081518162817381F8018491EAEB2E
:10F25000FAE0882349F09091C00095FFFCCF80939D
:10F26000C60031968491F5CF22E030E08AEA99E039
:10F270000E949535F7018491E6EBFAE0882349F086
:10F280009091C00095FFFCCF8093C6003196849189
:10F29000F5CF6091E30A70E04AE050E08AEA99E035
:10F2A0000E949D34F5018491E2EBFAE0882349F055
:10F2B0009091C00095FFFCCF8093C6003196849159
:10F2C000F5CF4091601A5091611A6091621A709165
:10F2D000631A21E030E08AEA99E00E949535809136
:10F2E000C00085FFFCCFD092C6000F9442A42B0132
:10F2F0003C010F94513780E00E94154B80E00F9441
:10F30000175767CF882777FD8095982F0F94CAAD40
:10F310002091601A3091611A4091621A5091631ADB
:10F320000F9428AD87FF05C080910802882309F457
:10F3300070CFE9E4F8E2859194910F94985584E0B8
:10F3400090E090932C0B80932B0B0F9442A460932E
:10F35000A90A7093AA0A8093AB0A9093AC0A0C9402
:10F36000E58B83E50E944636882319F10E94A63674
:10F3700020E030E0A9010F9428AD87FD0FC00E9466
:10F38000A63620E030E04FE753E40F9457AF18164D
:10F3900044F00E94A6360F9497AD05C060E070E07F
:10F3A00002C06FEF70E07093E20A6093E10A0C9480
:10F3B000E58B8FEF90E09093E20A8093E10A0C9442
:10F3C000E58B1092710B0C94E58B81E08093710BAF
:10F3D0000C94E58B83E50E944636882399F00E94C1
:10F3E000A63620E030E04AE754E40F9429B00F94A9
:10F3F0009CAD60930A0270930B0280930C02909371
:10F400000D021DC088E50E94463681110C943B8D8B
:10F4100089E50E94463681110C943B8D8AE50E9455
:10F42000463681110C943B8D85E40E94463681114D
:10F430000C943B8D0F94CC25149A0F944E26109269
:10F44000220B0C94E58B83E50E944636882311F449
:10F450000C94E58B0E94A63620E030E04AE754E4A5
:10F460000F9429B00F949CAD6093A50A7093A60ADF
:10F470008093A70A9093A80A0C94E58B20EC36E0C1
:10F4800039AF28AF05E419E1B5E5EB2EB9E1FB2E64
:10F4900085E0282E89E1382ED12CA8ADB9AD8D910B
:10F4A000B9AFA8AF0E944636882309F45CC0B3E028
:10F4B000DB1252C00E94A6362B013C0120E030E056
:10F4C00040EA51E40F9428AD87FF3FC0A3019201A9
:10F4D000F80160817181828193810F942FAD4B017E
:10F4E0005C019B01AC0160912519709126198091F6
:10F4F0002719909128190F9429B0609325197093BA
:10F5000026198093271990932819A5019401D701F2
:10F510006D917D918D919C910F9429B0F70160833D
:10F52000718382839383D1016D917D918D919C91A3
:10F530000F94C8ADA50194010F9429B00F949CAD10
:10F54000F1016083718382839383D8014D925D9230
:10F550006D927C92139707C00E94A636F8016083D3
:10F56000718382839383D3940C5F1F4FF4E0EF0E7B
:10F57000F11C24E0220E311C34E0D3128ECF0C9407
:10F58000E58B86E50E9446368823B9F00F948FA05C
:10F59000FC012491222341F03091C00035FFFCCFC3
:10F5A0002093C6000196F4CF8091C00085FFFCCF68
:10F5B0008AE08093C6000C94E58B85E50E94463670
:10F5C000882369F0809145109091461001969093A0
:10F5D0004610809345100F9400A30C94E58BE3EA4A
:10F5E000F7E285919491FC012491222311F40C946B
:10F5F000E58B3091C00035FFFCCF2093C60001960B
:10F60000F2CFEBEAFAE08491882341F09091C000B8
:10F6100095FFFCCF8093C6003196F5CF4091F70A55
:10F620005091F80A6091F90A7091FA0A22E030E0EC
:10F630008AEA99E00E949535E7EAFAE08491882306
:10F6400041F09091C00095FFFCCF8093C6003196A9
:10F65000F5CF4091FB0A5091FC0A6091FD0A709130
:10F66000FE0A22E030E08AEA99E00E949535E3EA5A
:10F67000FAE08491882341F09091C00095FFFCCF7F
:10F680008093C6003196F5CF4091FF0A5091000B50
:10F690006091010B7091020B22E030E08AEA99E060
:10F6A0000E949535EFE9FAE08491882341F090912A
:10F6B000C00095FFFCCF8093C6003196F5CF4091F6
:10F6C000030B5091040B6091050B7091060B22E027
:10F6D00030E08AEA99E00E949535E3E1F8E285910D
:10F6E0009491FC012491222341F03091C00035FF18
:10F6F000FCCF2093C6000196F4CF80E00F942D2616
:10F700000F94CAAD2091451930914619409147197F
:10F71000509148190F942FADAB01BC0122E030E0AD
:10F720008AEA99E00E949535EBE9FAE08491882312
:10F7300041F09091C00095FFFCCF8093C6003196B8
:10F74000F5CF81E00F942D260F94CAAD2091491971
:10F7500030914A1940914B1950914C190F942FAD8B
:10F76000AB01BC0122E030E08AEA99E00E949535C5
:10F77000E7E9FAE08491882341F09091C00095FF79
:10F78000FCCF8093C6003196F5CF82E00F942D26F2
:10F790000F94CAAD20914D1930914E1940914F19D7
:10F7A000509150190F942FADAB01BC0122E030E015
:10F7B0008AEA99E00E9495358091C00085FFFCCFD0
:10F7C0008AE08093C6000C94E58B80E00F947B1C4C
:10F7D0000C94E58B81E00F947B1C0C94E58B3091AD
:10F7E000C00035FFFCCF2093C6000196FC01249198
:10F7F0002111F5CF8091C00085FFFCCF8AE0809376
:10F80000C600EBEAF6E285919491FC012491222353
:10F8100041F03091C00035FFFCCF2093C600019627
:10F82000F4CF8091060182FF10C0E5E0F8E28591F7
:10F830009491FC0124912223C1F03091C00035FF46
:10F84000FCCF2093C6000196F4CFE3E0F8E2859167
:10F850009491FC012491222341F03091C00035FFA6
:10F86000FCCF2093C6000196F4CF8091C00085FFA5
:10F87000FCCF8AE08093C600EDEAF6E28591949190
:10F88000FC012491222341F03091C00035FFFCCFD0
:10F890002093C6000196F4CF8091060182FF10C02C
:10F8A000E5E0F8E285919491FC0124912223C1F0D6
:10F8B0003091C00035FFFCCF2093C6000196F4CFF5
:10F8C000E3E0F8E285919491FC012491222341F038
:10F8D0003091C00035FFFCCF2093C6000196F4CFD5
:10F8E0008091C00085FFFCCF8AE08093C600E5EAE6
:10F8F000F6E285919491FC012491222341F030910C
:10F90000C00035FFFCCF2093C6000196F4CF809154
:10F91000060187FF10C0E5E0F8E285919491FC01B3
:10F9200024912223C1F03091C00035FFFCCF2093F9
:10F93000C6000196F4CFE3E0F8E285919491FC01D2
:10F940002491222341F03091C00035FFFCCF209359
:10F95000C6000196F4CF8091C00085FFFCCF8AE0FD
:10F960008093C600E7EAF6E285919491FC01249128
:10F97000222341F03091C00035FFFCCF2093C60018
:10F980000196F4CF8091060187FF10C0E5E0F8E210
:10F9900085919491FC0124912223C1F03091C00003
:10F9A00035FFFCCF2093C6000196F4CFE3E0F8E2E8
:10F9B00085919491FC012491222341F03091C00063
:10F9C00035FFFCCF2093C6000196F4CF8091C00094
:10F9D00085FFFCCF8AE08093C600EFE9F6E28591CF
:10F9E0009491FC012491222341F03091C00035FF15
:10F9F000FCCF2093C6000196F4CF1C9B10C0E5E01D
:10FA0000F8E285919491FC0124912223C1F0309178
:10FA1000C00035FFFCCF2093C6000196F4CFE3E091
:10FA2000F8E285919491FC012491222341F03091D8
:10FA3000C00035FFFCCF2093C6000196F4CF809123
:10FA4000C00085FFFCCF8AE08093C600E1EAF6E2C1
:10FA500085919491FC012491222341F03091C000C2
:10FA600035FFFCCF2093C6000196F4CF019910C05A
:10FA7000E5E0F8E285919491FC0124912223C1F004
:10FA80003091C00035FFFCCF2093C6000196F4CF23
:10FA9000E3E0F8E285919491FC012491222341F066
:10FAA0003091C00035FFFCCF2093C6000196F4CF03
:10FAB0008091C00085FFFCCF8AE08093C6000C9443
:10FAC000E58B8091E30A8093980A84E50E9446368C
:10FAD000882329F10E94A6360F949CAD6093980A62
:10FAE0006623E9F0E0E4F0E18491882341F090910D
:10FAF000C00095FFFCCF8093C6003196F5CFEFE9AB
:10FB0000F7E2A591B4918D91882311F40C94E58BC3
:10FB10009091C00095FFFCCF8093C600F4CF84E4A1
:10FB20000E944636882311F40C94E58B0E94A63679
:10FB300020E030E0A9010F9428AD811103C010929C
:10FB4000070B32C00091980A10E00E94A636F80117
:10FB5000EE0FFF1FEE0FFF1FE15CFD4F608371830F
:10FB600082839383E0903F02F09040020091410233
:10FB70001091420220E030E0A901B701C8010F94C2
:10FB800028AD811104C0E12CF12C00E410E4C70180
:10FB9000D80180933F0290934002A0934102B0931A
:10FBA000420281E08093070B0E94244D0C94E58B68
:10FBB000D8018D918D010E944636882349F00E941C
:10FBC000A6360F949CADF701608371838283938383
:10FBD000F4E0EF0EF11C26E0043C120749F70F9405
:10FBE000CB1A0C94E58B00EC16E055E5E52E59E1B7
:10FBF000F52ED8018D918D010E944636882339F06B
:10FC00000E94A636F7016083718382839383F4E0B8
:10FC1000EF0EF11C26E0043C120759F70C94E58B1B
:10FC200083E50E944636882351F00E94A6366093F1
:10FC30002D1970932E1980932F199093301984E504
:10FC40000E944636882311F40C94E58B0E94A63658
:10FC50006093291970932A1980932B1990932C196A
:10FC60000C94E58B83E50E944636882351F00E9470
:10FC7000A63660933119709332198093331990939B
:10FC8000341984E50E944636882351F00E94A63636
:10FC9000609315197093161980931719909318197A
:10FCA00082E40E944636882361F00E94A6360F94B3
:10FCB0009CAD609365197093661980936719909352
:10FCC000681988E50E944636882391F00E94A6367E
:10FCD00060931D1970931E1980931F19909320191A
:10FCE0006093191970931A1980931B1990931C191A
:10FCF00089E50E944636882351F00E94A63660931B
:10FD00001D1970931E1980931F19909320198AE56D
:10FD10000E944636882351F00E94A636609321192E
:10FD200070932219809323199093241985E40E94DB
:10FD30004636882311F40C94E58B0E94A636609316
:10FD400025197093261980932719909328190C94DC
:10FD5000E58B00EC16E04BEEE42E4AE0F42ED801E1
:10FD60008D918D010E944636882339F00E94A63677
:10FD7000F7016083718382839383F4E0EF0EF11CBB
:10FD800026E0033C120759F70C94E58B83E50E94AB
:10FD90004636882351F00E94A63660931F02709366
:10FDA0002002809321029093220286E40E9446362C
:10FDB000882381F00E94A63620E030E040E752E43C
:10FDC0000F942FAD6093170270931802809319025D
:10FDD00090931A028AE50E944636882311F40C9407
:10FDE000E58B0E94A6366093DB0A7093DC0A809351
:10FDF000DD0A9093DE0A0C94E58B83E50E9446367B
:10FE0000882351F00E94A6366093D70A7093D80ACF
:10FE10008093D90A9093DA0A86E40E9446368823B2
:10FE200011F40C94E58B0E94A63620E030E040E708
:10FE300052E40F942FAD60931302709314028093D9
:10FE40001502909316020C94E58B83E50E944636CA
:10FE5000882311F40C94E58B0E94A6360F9497AD7D
:10FE60006115710551F06130710569F481E080938D
:10FE7000E00A1092DF0A0C94E58B1092E00A1092CF
:10FE8000DF0A0C94E58BE0E4F0E18491882341F0F3
:10FE90009091C00095FFFCCF8093C6003196F5CFBE
:10FEA000EDEBF6E285919491FC012491222341F03F
:10FEB0003091C00035FFFCCF2093C6000196F4CFEF
:10FEC000E0914F10F0915010EC5AFF4E8191882331
:10FED00039F09091C00095FFFCCF8093C600F6CF1B
:10FEE000E2E9FAE08491882341F09091C00095FF07
:10FEF000FCCF8093C6003196F5CF8091C00085FF7E
:10FF0000FCCF8AE08093C6000C94E58B83E50E94C9
:10FF10004636882311F40C94E58B0E94A6360F9484
:10FF200097AD70934A02609349020C94E58B83E588
:10FF30000E944636882311F40C94E58B0E94A63665
:10FF40000F9497AD6B017C0184E50E9446368823AF
:10FF500091F08DED90E00E94CF4B81110C94E58BD8
:10FF6000E091980AF0E0EE0FFF1FEB5BFD4FD182AE
:10FF7000C0820C94E58BD0924802C09247020C9448
:10FF8000E58B80E50E944636882311F40C94E58BBE
:10FF90000E94A6360F9497ADD62E062F172F83E515
:10FFA0000E944636882331F00E94A6360F9497AD02
:10FFB0007B0103C0EE24EA94FE2CC701019603974F
:10FFC00010F00C94E58BE8E8F6E0819191918017B0
:10FFD000910711F40C94E58B26E0E03CF207A9F7B9
:10FFE00017FF02C00C94E58B0F94CC25CD2C60E05C
:10FFF0008D2D0F942DA63FEFE316F30631F0EA9412
:020000021000EC
:10000000EF2871F000E010E00DC08D2D0F949BA63D
:1000100031E020E0892B09F030E0032F122F02C0DD
:1000200001E010E08C2D0F949BA68017910711F42E
:100030000C94E58B0F94513780E00E94154B80E0C3
:100040000F941757EFCF83E50E944636882331F08F
:100050000E94A6360F9497AD8B0102C00EE610E009
:1000600080E50E944636882331F00E94A6360F9420
:1000700097ADCB0102C088EE93E06C01EE24D7FC73
:10008000E094FE2C1016110684F420E030E0A90163
:10009000B80184E50F9490A8C701B6010F9471A42C
:1000A00084E50F94B6AB0C94E58BC701B6010F94B1
:1000B00071A40C94E58B80E50E944636882351F0AC
:1000C0000E94A63660939C0270939D0280939E02CC
:1000D00090939F0289E40E944636882361F00E9433
:1000E000A6360F940D3E6093980270939902809308
:1000F0009A0290939B0284E40E944636882361F022
:100100000E94A6360F94193E609394027093950254
:10011000809396029093970283E40E944636882348
:1001200051F00E94A63660939002709391028093E2
:100130009202909393020F943E2DE3E7F7E28591AC
:100140009491FC012491222341F03091C00035FFAD
:10015000FCCF2093C6000196F4CFEDE6F5E0819147
:10016000882339F09091C00095FFFCCF8093C600A2
:10017000F6CF40919C0250919D0260919E02709139
:100180009F0222E030E08AEA99E00E949535E1E79B
:10019000F5E08191882339F09091C00095FFFCCF64
:1001A0008093C600F6CF6091980270919902809179
:1001B0009A0290919B020F94133EAB01BC0122E086
:1001C00030E08AEA99E00E949535E5E7F5E0819113
:1001D000882339F09091C00095FFFCCF8093C60032
:1001E000F6CF609194027091950280919602909161
:1001F00097020F941F3EAB01BC0122E030E08AEA77
:1002000099E00E949535E9E7F5E08191882339F07E
:100210009091C00095FFFCCF8093C600F6CF40912F
:10022000900250919102609192027091930222E0AB
:1002300030E08AEA99E00E9495358091C00085FF00
:10024000FCCF8AE08093C6000C94E58B80E50E9489
:100250004636882351F00E94A63660938C02709334
:100260008D0280938E0290938F0289E40E9446361D
:10027000882361F00E94A6360F940D3E6093880299
:100280007093890280938A0290938B0284E40E9487
:100290004636882361F00E94A6360F94193E60937B
:1002A00084027093850280938602909387020F9454
:1002B0003E2DE3E7F7E285919491FC0124912223FE
:1002C00041F03091C00035FFFCCF2093C60001966D
:1002D000F4CFEDE6F5E08191882339F09091C000EC
:1002E00095FFFCCF8093C600F6CF40918C025091D1
:1002F0008D0260918E0270918F0222E030E08AEAD6
:1003000099E00E949535E1E7F5E08191882339F085
:100310009091C00095FFFCCF8093C600F6CF60910E
:1003200088027091890280918A0290918B020F94C9
:10033000133EAB01BC0122E030E08AEA99E00E9462
:100340009535E5E7F5E08191882339F09091C0007B
:1003500095FFFCCF8093C600F6CF60918402709128
:10036000850280918602909187020F941F3EAB0117
:10037000BC0122E030E08AEA99E00E949535809144
:10038000C00085FFFCCF8AE08093C6000C94E58B0B
:1003900083E50E944636882319F00E94A63603C0E2
:1003A00060E070E0CB010F94C21A0C94E58B85E4F9
:1003B0000E944636882341F00E94A6360F9497ADDE
:1003C0008B0177FF03C009C000E010E0812C912C65
:1003D00096E1A92E93E4B92E06C0812C912C8CE8CD
:1003E000A82E82E4B82E83E50E944636882321F0A9
:1003F0000E94A6364B015C0183E40E9446368823A6
:1004000031F00E94A6360F9497AD9B0102C025E003
:1004100030E0A801C501B4010F94FE2F0C94E58BC8
:1004200060E084E190E00E9497240C94E58B60E00A
:1004300084E190E00E94262C0C94E58B80E00E94E1
:10044000B7250C94E58B9091C00095FFFCCF80936D
:10045000C600319684918111F6CFE2E8FAE08491EA
:10046000882311F40C94E58B9091C00095FFFCCF8C
:100470008093C6003196F3CF8AE50E9446368823E2
:1004800009F4B0C00E94A6364B015C0120E030E0C8
:1004900040E751EC0F9457AF87FD4EC020E030E0AD
:1004A00040EA50ECC501B4010F9428AD18160CF4C5
:1004B00043C0B7FAB094B7F8B0948092E40A90922F
:1004C000E50AA092E60AB092E70AE0E4F0E184913E
:1004D000882341F09091C00095FFFCCF8093C60027
:1004E0003196F5CFE3E7F7E245915491E3EAF6E27E
:1004F0008591949121E83AE065E279E00E946EBB33
:10050000FC012491222341F03091C00035FFFCCF43
:100510002093C6000196F4CF8091C00085FFFCCFE8
:100520008AE08093C6008091C00085FFFCCF8AE0FE
:100530008093C6000C94E58BE0E4F0E1849188237D
:1005400041F09091C00095FFFCCF8093C60031969A
:10055000F5CFE3EAF6E285919491FC012491222300
:1005600041F03091C00035FFFCCF2093C6000196CA
:10057000F4CFEFE9F6E285919491FC0124912223D6
:1005800041F03091C00035FFFCCF2093C6000196AA
:10059000F4CF4AE050E061EF7FEF8AEA99E00E94F1
:1005A0009D34E1EAF6E285919491FC0124912223A5
:1005B00041F03091C00035FFFCCF2093C60001967A
:1005C000F4CF4AE050E06BEF7FEF8AEA99E00E94B7
:1005D0009D348091C00085FFFCCF8AE08093C600E7
:1005E0000C94E58BE0E4F0E18491882341F0909154
:1005F000C00095FFFCCF8093C6003196F5CFE3EAAB
:10060000F6E2859194916DE77AE00E944DBBFC0182
:100610002491222341F03091C00035FFFCCF20937C
:10062000C6000196F4CF8091C00085FFFCCF8AE020
:100630008093C6004091E40A5091E50A6091E60A71
:100640007091E70A705822E030E08AEA99E00E944F
:1006500095358091C00085FFFCCF8AE08093C6006D
:100660000C94E58B6DE775E08AEA99E00E9490347E
:100670000F94CC258091851B882321F086E190E0A2
:100680000F9406558091490290914A02909344023A
:1006900080934302C090F70AD090F80AE090F90ADC
:1006A000F090FA0ACF8ED8A2E9A2FAA20091FB0A32
:1006B0001091FC0A2091FD0A3091FE0A0BA31CA3A5
:1006C0002DA33EA34091FF0A5091000B6091010BB6
:1006D0007091020B4FA358A769A77AA78091030BCB
:1006E0009091040BA091050BB091060B8BA79CA7D2
:1006F000ADA7BEA7C982DA82EB82FC820D831E837E
:100700002F83388749875A876B877C878D879E8799
:10071000AF87B88B85E40E944636882359F00E9443
:10072000A6369B01AC016BA57CA58DA59EA50F945B
:1007300038AC0AC020E030E040E050E46BA57CA576
:100740008DA59EA50F9437AC6BA77CA78DA79EA700
:10075000EFA0F8A409A51AA52BA13CA14DA15EA16B
:100760006F8D78A189A19AA1E3EEFAE0FF93EF9350
:10077000812C912CB8ECAB2EB3E4BB2EDE019B9602
:100780006D010F94580C8AE50E9446360F900F9029
:10079000882349F00E94A6369B01AC016FA178A581
:1007A00089A59AA51EC020E030E040E050E46FA18A
:1007B00078A589A59AA50F9438AC4B015C016FA36D
:1007C00078A789A79AA720E030E040E251E40F948F
:1007D00028AD87FF0CC020E030E040E251E4C501C5
:1007E000B4010F9438AC6FA378A789A79AA7EFA09C
:1007F000F8A409A51AA52BA13CA14DA15EA16F8D5E
:1008000078A189A19AA1E3EEFAE0FF93EF93812CFE
:10081000912CA0E7AA2EA1E4BA2EFE01BB966F018F
:100820000F94580C88E50E9446360F900F9088234D
:1008300079F00E94A6369B01AC016F8D78A189A149
:100840009AA10F9438AC6F8F78A389A39AA308C09C
:1008500080E090E0A3E5B3E48F8F98A3A9A3BAA3A7
:1008600089E50E944636882339F00E94A6366BA39C
:100870007CA38DA39EA304C01BA21CA21DA21EA22A
:10088000EFA0F8A409A51AA52BA13CA14DA15EA13A
:100890006F8D78A189A19AA1E3EEFAE0FF93EF931F
:1008A000812C912CF8E4AF2EF2E4BF2EDE019B9652
:1008B0006D010F94580C0F94CC2581E08093280B88
:1008C000EBEBF6E2859194910F9498558CE40E949D
:1008D00046360F900F90882359F00E94A6369B0150
:1008E000AC016BA57CA58DA59EA50F9438AC0AC064
:1008F00020E030E040EA52E46BA57CA58DA59EA5E2
:100900000F9437AC6BA77CA78DA79EA7EFA0F8A488
:1009100009A51AA52BA13CA14DA15EA16F8D78A1BF
:1009200089A19AA1E3EEFAE0FF93EF93812C912C39
:10093000E8ECAE2EE3E4BE2EFE01BB966F010F94F1
:10094000580C0F94CC25149A64E670E080E090E097
:100950000F9471A40F9425720F9442A46093370BE7
:100960007093380B8093390B90933A0B0F900F9044
:1009700000E010E0F12C0F949F5981112AC0F394EC
:100980000F94513781E00E94154BF110F4CF043FD2
:10099000F1E01F0711F400E010E080910101846094
:1009A000809301010115110531F49FB7F8948091EE
:1009B0000201846008C00431110541F49FB7F89426
:1009C000809102018B7F809302019FBF0F5F1F4FB9
:1009D000D2CF9FB7F894809102018B7F8093020160
:1009E0009FBF20E030E04CE852E46BA57CA58DA5CC
:1009F0009EA50F9438AC6BA77CA78DA79EA7EFA0F0
:100A0000F8A409A51AA52BA13CA14DA15EA16F8D4B
:100A100078A189A19AA1F3EE6F2EFAE07F2E7F9242
:100A20006F92812C912CA0EAAA2EA1E4BA2EDE01AD
:100A30009B966D010F94580C20E030E048E452E49E
:100A40006BA57CA58DA59EA50F9438AC6BA77CA744
:100A50008DA79EA7EFA0F8A409A51AA52BA13CA1DC
:100A60004DA15EA16F8D78A189A19AA17F926F920D
:100A7000812C912CA12CB0E4BB2E0F94580C109219
:100A80005A0B1092590B0F948D720F900F900F907C
:100A90000F908091590B90915A0B019709F48CC0DB
:100AA00010925A0B1092590B0F94CD728091590BE2
:100AB00090915A0B8230910571F1039709F076C03D
:100AC00020E030E048E452E46BA57CA58DA59EA50E
:100AD0000F9438AC6BA77CA78DA79EA7EFA0F8A4B6
:100AE00009A51AA52BA13CA14DA15EA16F8D78A1EE
:100AF00089A19AA17F926F92812C912CA12CA0E4C4
:100B0000BA2EDE019B966D010F94580C0F944D7216
:100B10000F900F90BECF20E030E04CE852E46BA580
:100B20007CA58DA59EA50F9438AC6BA77CA78DA73F
:100B30009EA7EFA0F8A409A51AA52BA13CA14DA141
:100B40005EA16F8D78A189A19AA17F926F92812C6D
:100B5000912CB0EAAB2EB1E4BB2EDE019B966D0169
:100B60000F94580C20E030E048E452E46BA57CA5DB
:100B70008DA59EA50F9438AC6BA77CA78DA79EA7CB
:100B8000EFA0F8A409A51AA52BA13CA14DA15EA137
:100B90006F8D78A189A19AA17F926F92812C912C5F
:100BA000A12CE0E4BE2E0F94580C6DCF0F943F7231
:100BB00081E00F9484586DCF20E030E040EA50E4AB
:100BC0006BA57CA58DA59EA50F9438AC6BA77CA7C3
:100BD0008DA79EA7EFA0F8A409A51AA52BA13CA15B
:100BE0004DA15EA16F8D78A189A19AA1E3EE6E2E31
:100BF000EAE07E2E7F926F92812C912CA12CF0E462
:100C0000BF2EFE01BB966F010F94580CA5019401F5
:100C10006BA57CA58DA59EA50F9437AC6BA77CA773
:100C20008DA79EA7EFA0F8A409A51AA52BA13CA10A
:100C30004DA15EA16F8D78A189A19AA17F926F923B
:100C4000812C912CA8ECAA2EA3E4BA2E0F94580C58
:100C5000EFA0F8A409A51AA52D813E814F815885E2
:100C600069817A818B819C817F926F92812C912CFA
:100C7000B8E4AB2EB2E4BB2E0F94580CE984FA848E
:100C80000B851C852D813E814F81588569817A8134
:100C90008B819C817F926F92812C912CE0E7AE2E0C
:100CA000E1E4BE2E0F94580C20E030E040E050E428
:100CB0006BA57CA58DA59EA50F9438AC6BA77CA7D2
:100CC0008DA79EA7E984FA840B851C852D813E8122
:100CD0004F81588569817A818B819C817F926F9247
:100CE000812C912CF8ECAF2EF3E4BF2E0F94580C0E
:100CF000CE010D960F94A51A809143029091440263
:100D00008093490290934A029F938F9384E79AE0DD
:100D10009F938F938E01015D1F4F1F930F930F942D
:100D20008AB660E0C8010E9417B4EDE9F6E2859149
:100D300094910F9498551092280B1092260B1092B4
:100D4000250B0FB6F894DEBF0FBECDBF8091950A7C
:100D5000882309F43AC50E9441B30F94CC250E9420
:100D6000B1B5811105C00E94735C0E9441B3F7CFF9
:100D70000E94D53A0E94515B28C58091891B9091B1
:100D80008A1B892B09F021C585E090E090938A1B8E
:100D90008093891B1AC58091891B90918A1B892B8E
:100DA00009F013C586E090E090938A1B8093891B1D
:100DB0000CC50E94283C09C588E50E944636882358
:100DC00039F00E94A6360F9497AD80E00F94442727
:100DD0008AE50E944636882339F00E94A6360F9491
:100DE00097AD81E00F94442785E40E94463688231E
:100DF00009F4EBC40E94A6360F9497AD82E00F94DD
:100E00004427E3C40F94CE42E0C488E50E944636EE
:100E1000882339F00E94A6360F949CAD80E00F9491
:100E20004C4289E50E944636882339F00E94A63656
:100E30000F949CAD81E00F944C428AE50E944636A7
:100E4000882339F00E94A6360F949CAD82E00F945F
:100E50004C4285E40E944636882309F4B6C40E94B9
:100E6000A6360F949CAD83E00F944C42AEC488E547
:100E70000E944636882339F00E94A6360F949CAD16
:100E800080E00F948D4289E50E944636882339F030
:100E90000E94A6360F949CAD81E00F948D428AE5A6
:100EA0000E944636882339F00E94A6360F949CADE6
:100EB00082E00F948D4285E40E944636882309F42F
:100EC00084C40E94A6360F949CAD83E00F948D429B
:100ED0007CC40F94D93E79C481E08093E51A0F94C5
:100EE000CE4273C488E50E944636882331F00E94C2
:100EF000A6360F949CAD6093A50289E50E94463604
:100F0000882331F00E94A6360F949CAD6093A60210
:100F10008AE50E944636882331F00E94A6360F9457
:100F20009CAD6093A70285E40E944636882331F089
:100F30000E94A6360F949CAD6093A802EAE8F5E003
:100F40008191882339F09091C00095FFFCCF809368
:100F5000C600F6CF4AE050E06091A5028AEA99E027
:100F60000E94E234EDE9F5E08191882339F0909117
:100F7000C00095FFFCCF8093C600F6CF4AE050E05A
:100F80006091A6028AEA99E00E94E234E0EBF5E083
:100F90008191882339F09091C00095FFFCCF809318
:100FA000C600F6CF4AE050E06091A7028AEA99E0D5
:100FB0000E94E234E3ECF5E08191882339F09091CE
:100FC000C00095FFFCCF8093C600F6CF4AE050E00A
:100FD0006091A8028AEA99E00E94E234F6C388E5AB
:100FE0000E944636882339F00E94A6360F949CADA5
:100FF00080E00F944D4089E50E944636882339F001
:101000000E94A6360F949CAD81E00F944D408AE576
:101010000E944636882339F00E94A6360F949CAD74
:1010200082E00F944D4085E40E944636882309F4FF
:10103000CCC30E94A6360F949CAD83E00F944D4024
:10104000C4C388E50E944636882339F00E94A6363C
:101050000F949CAD80E00F94A44089E50E94463631
:10106000882339F00E94A6360F949CAD81E00F943E
:10107000A4408AE50E944636882339F00E94A636AD
:101080000F949CAD82E00F94A44085E40E94463604
:10109000882309F49AC30E94A6360F949CAD83E07E
:1010A0000F94A44092C3159881E08093280B82E0AE
:1010B00090E09093260B8093250BEFEAF7E2859161
:1010C00094910F94985520E030E04CE852E4609100
:1010D000030B7091040B8091050B9091060B0F94FC
:1010E00038AC6093030B7093040B8093050B9093C3
:1010F000060BE090FF0AF090000B0091010B10919D
:10110000020B2091FB0A3091FC0A4091FD0A50919C
:10111000FE0A6091F70A7091F80A8091F90A90919D
:10112000FA0AE3EE6E2EEAE07E2E7F926F92812C19
:10113000912CF0ECAF2EF0E4BF2EA3E0CA2EABE072
:10114000DA2E0F94580C20E030E048EC51E4609126
:10115000030B7091040B8091050B9091060B0F947B
:1011600038AC6093030B7093040B8093050B909342
:10117000060BE090FF0AF090000B0091010B10911C
:10118000020B2091FB0A3091FC0A4091FD0A50911C
:10119000FE0A6091F70A7091F80A8091F90A90911D
:1011A000FA0A7F926F92812C912CB0E8AB2EBFE3AC
:1011B000BB2E0F94580C0F94CC250F900F900F90CE
:1011C0000F908091851B8823A9F081E00F948458AB
:1011D00082E00F941757EDE9F6E2859194910F9410
:1011E00098551092270B1092280B1092260B1092F4
:1011F000250BEBC28091270B882339F303EE602E79
:1012000007E2702EF3018591949141E060E00F9424
:10121000357C91E0811101C090E013EE412E1AE07F
:10122000512E9111D2CF81E00F94845882E00F9417
:10123000175720E030E048EC51E46091030B7091C7
:10124000040B8091050B9091060B0F9438AC6093C2
:10125000030B7093040B8093050B9093060BE090A7
:10126000FF0AF090000B0091010B1091020B2091EE
:10127000FB0A3091FC0A4091FD0A5091FE0A6091F0
:10128000F70A7091F80A8091F90A9091FA0A5F9230
:101290004F92812C912CA0E8AA2EAFE3BA2EB3E096
:1012A000CB2EBBE0DB2E0F94580C0F94CC25F30112
:1012B0008591949141E060E00F94357C0F900F9000
:1012C000811183CFB0CF81E08093280B82E090E042
:1012D0009093260B8093250BEBEBF6E2859194918E
:1012E0000F94985520E030E040EA52E46091030BFF
:1012F0007091040B8091050B9091060B0F9437AC05
:101300006093030B7093040B8093050B9093060B73
:10131000E090FF0AF090000B0091010B1091020B7E
:101320002091FB0A3091FC0A4091FD0A5091FE0A7F
:101330006091F70A7091F80A8091F90A9091FA0A7F
:10134000E3EEFAE0FF93EF93812C912CE8EEAE2EC2
:10135000E2E4BE2EF3E0CF2EFBE0DF2E0F94580C1C
:101360000F94CC25EDE9F6E2859194910F94985570
:101370001092280B1092260B1092250B0F900F90B5
:1013800024C2E4E6FAE08491882341F09091C00001
:1013900095FFFCCF8093C6003196F5CF8091C000B9
:1013A00085FFFCCF8AE08093C6000FC284E50E94CF
:1013B0004636882309F4D1C0E0914510F0914610DB
:1013C000319681918032E9F38930D9F390ED980F0D
:1013D0009A30E0F08F33A9F0E4E5FAE084918823B5
:1013E00041F09091C00095FFFCCF8093C6003196EC
:1013F000F5CF8091C00085FFFCCF8AE08093C600C6
:10140000E4C10F94859F8093980A06C00E94A63677
:101410000F949CAD6093980A2091980A81E090E027
:10142000022E01C0880F0A94EAF79091220B982BA4
:101430009093220B222309F442C0E0E4F0E184916E
:10144000882341F09091C00095FFFCCF8093C600A7
:101450003196F5CFE2E5FAE08491882341F090914E
:10146000C00095FFFCCF8093C6003196F5CF609108
:10147000980A70E04AE050E08AEA99E00E949D34C0
:101480008091C00085FFFCCF8AE08093C600E7EB27
:10149000F7E285919491FC012491222341F030914F
:1014A000C00035FFFCCF2093C6000196F4CF809199
:1014B000C00085FFFCCF8AE08093C60086C186E429
:1014C0000E9446368823D9F00E94A6364B015C0163
:1014D0006093B20A7093B30A8093B40A9093B50AEA
:1014E00020E030E0A9010F9457AF181644F4809221
:1014F0000E0290920F02A0921002B0921102E0E44C
:10150000F0E18491882341F09091C00095FFFCCFD9
:101510008093C6003196F5CFE5E6F8E28591949187
:10152000FC012491222341F03091C00035FFFCCF13
:101530002093C6000196F4CF6091E30A70E04AE080
:1015400050E08AEA99E00E949D348091C00085FFB6
:10155000FCCF8AE08093C60038C184E40E944636FE
:10156000882309F4F1C00E94A6360F9497AD663027
:10157000710509F4BBC0ACF462307105B1F154F4EB
:101580006115710579F16130710509F01EC10E9484
:10159000EC2D1BC16430710559F16CF50E94C42E0D
:1015A00014C16A30710509F450C054F467307105F4
:1015B000B1F06830710509F008C1E6EDF5E0B6C09C
:1015C000683EF3E07F0709F480C0693E23E07207BC
:1015D00009F481C0673E734009F0F7C03AC0E3EEFA
:1015E000F5E08FC00E94D62DF0C00E94032EEDC002
:1015F0000E948E2FEAC061EF75E08AEA99E00E94AE
:10160000903480E50E944636882341F00E94A63639
:101610000F9497AD7093300A60932F0AEBEFF5E0CB
:101620008191882339F09091C00095FFFCCF809381
:10163000C600F6CF60912F0A7091300A4AE050E060
:101640008AEA99E00E94A434C0C086EE0E948C3AD7
:10165000BCC061E176E08AEA99E00E9490340F9480
:10166000CC2581E00F9484580F94815482E00F942C
:101670001757E9E4F7E28591949140E060E00F9418
:10168000357C182F81E00F94845882E00F9417570F
:10169000EDE9F6E2859194910F94985561E011235C
:1016A00079F08CE49AE00E9417B461E086E49AE055
:1016B0000E9417B461E080E49AE00E9417B485C0EC
:1016C0008AE39AE00E9417B480C00E944D5B81E0DB
:1016D0008093A0027AC01092780B60E086E79BE0CE
:1016E0000E9469AD81E08093A0026FC081E090E02C
:1016F0000E94CD3E6AC09091C00095FFFCCF8093C0
:10170000C60081918111F7CF68EC88EC0F94FD063B
:101710004AE050E0BC018AEA99E00E94A43455C036
:101720009091C00095FFFCCF8093C60081918111FC
:10173000F7CF85E70F9493294AE050E0BC018AEA8D
:1017400099E00E94A43441C0E0E4F0E18491882350
:1017500041F09091C00095FFFCCF8093C600319678
:10176000F5CFEDEBF6E285919491FC0124912223D3
:1017700041F03091C00035FFFCCF2093C6000196A8
:10178000F4CFE0914F10F0915010EC5AFF4E819140
:10179000882339F09091C00095FFFCCF8093C6005C
:1017A000F6CFE5E3FAE08491882341F09091C00000
:1017B00095FFFCCF8093C6003196F5CF8091C00095
:1017C00085FFFCCF8AE08093C6000E94EF4372C180
:1017D0008090CE0A9090CF0AA090D00AB090D10A03
:1017E0002091030B3091040B4091050B5091060B97
:1017F000C501B4010F9437AC2DEC3CEC4CEC5DE32F
:101800000F9457AF181614F00C94395F8092030BA5
:101810009092040BA092050BB092060B83E09BE024
:101820000F94A51A60E080E00E94134843C10E9413
:10183000A6362091EB0A3091EC0A4091ED0A5091C6
:10184000EE0A0F9438AC6093F70A7093F80A80930D
:10185000F90A9093FA0A0C944C600E94A6362091E3
:10186000EF0A3091F00A4091F10A5091F20A0F9478
:1018700038AC6093FB0A7093FC0A8093FD0A909346
:10188000FE0A0C9459600E94A6362091F30A30910A
:10189000F40A4091F50A5091F60A0F9438AC60931F
:1018A000FF0A7093000B8093010B9093020B0C9432
:1018B0005A61711028C0662031F181E080937E1258
:1018C0000F943B266B017C0180E00F943B26AB011B
:1018D000BC01970186018EE792E10E94AF369B0121
:1018E000AC016091FF0A7091000B8091010B909107
:1018F000020B0F9437AC6093FF0A7093000B809338
:10190000010B9093020B8091851B882321F084E1C9
:1019100090E00F9406551092620BE3EAFEE084918A
:10192000882341F09091C00095FFFCCF8093C600C2
:101930003196F5CF0E94555BE7E9FEE0849188235C
:1019400041F09091C00095FFFCCF8093C600319686
:10195000F5CF0E94BB5BEBE8FEE08491882341F069
:101960009091C00095FFFCCF8093C6003196F5CFD3
:101970000E94175C2ACF20E030E040E85FE36091EE
:10198000030B7091040B8091050B9091060B0F9443
:1019900038AC6093030B7093040B8093050B90930A
:1019A000060BE090FF0AF090000B0091010B1091E4
:1019B000020B2091FB0A3091FC0A4091FD0A5091E4
:1019C000FE0A6091F70A7091F80A8091F90A9091E5
:1019D000FA0AE3EEFAE0FF93EF93812C912CA8EC46
:1019E000AA2EA3E4BA2EB3E0CB2EBBE0DB2E0F94DD
:1019F000580C0F900F900C94416E0F94513781E06A
:101A00000E94154B80E00F9417570C948A720E9425
:101A10007036AB01BC014093140E5093150E6093C9
:101A2000160E7093170E8FE59DE00E948B9BCDCE16
:101A30000E94A6360F9497AD8B010C94BC740F9442
:101A40001D68E1E7F7E2859194910F948C5AEBEDD4
:101A5000F7E2859194910E947E3A41E050E062E085
:101A600080E00F948C54E9EDF7E2859194910F9406
:101A700080690C9454750F94CC2588E50E944636F5
:101A8000882319F0179A1092E80A89E50E944636D1
:101A9000882319F0169A1092E90A8AE50E944636C0
:101AA00085E40E944636882311F40C941F7A149A18
:101AB0000C941F7AC75ADF4F0FB6F894DEBF0FBEE3
:101AC000CDBFDF91CF911F910F91FF90EF90DF90ED
:101AD000CF90BF90AF909F908F907F906F905F90CE
:101AE0004F903F902F9008950F931F93CF93DF93C4
:101AF0001F92CDB7DEB780915B0B90915C0B892B69
:101B0000A1F00F9442A40091990A10919A0A209191
:101B10009B0A30919C0A601B710B820B930B693EF0
:101B200073408105910508F0B1C080915B0B9091E5
:101B30005C0B892B11F41092630B8091330B88237B
:101B400019F00E9444437EC00E94BAB560E086E767
:101B50009BE00E9473AC80914B1090914C10892BAC
:101B600009F470C010924A108091760B8823B1F06E
:101B700000914F10109150100C5A1F4E60ED7EE0F6
:101B8000C8010F94B5B5892B09F5B80186E79BE02C
:101B90000E94C2AB8091770B882319F00E94735C7E
:101BA00031C0E3E7F7E285919491FC01249122236F
:101BB00041F03091C00035FFFCCF2093C600019664
:101BC000F4CF8091C00085FFFCCF19C060E086E7AC
:101BD0009BE00E9469ADEFEDF7E285919491FC01E5
:101BE0002491222341F03091C00035FFFCCF209397
:101BF000C6000196F4CF8091C00085FFFCCF8AE03B
:101C00008093C60080914A1081111CC080914B10B6
